:020000040800F2
:100000000000011049660308C9360208595F01085B
:100010004D6703084D6703084D67030800000000A3
:10002000000000000000000000000000153D020874
:10003000113D0208000000000D3D020831EA0008F1
:100040004D6703084D6703084D6703084D670308B4
:100050004D6703084D6703089D8F00088D900008C9
:100060004D670308519000081590000855AC000832
:1000700045AC000835AC000825AC000815AC0008FC
:1000800001AC0008EDAB00084D6703084D6703089D
:100090004D6703084D6703084D670308D98F0008B3
:1000A0004D6703084D6703084D6703084D67030854
:1000B00019DF000809DF0008F9DE00084D670308B2
:1000C0004D6703084D6703084D6703084D67030834
:1000D0004D67030891EC00084D670308F5EB000835
:1000E000618F00084D670308313D02084D67030822
:1000F0004D6703084D6703084D670308D9AB000837
:100100004D6703084D6703084D6703084D670308F3
:1001100059EB00084D6703084D6703084D67030856
:10012000C5AB0008B1AB00089DAB000889AB000867
:1001300075AB00084D6703084D6703084D6703085A
:100140004D6703084D6703084D670308CD36020865
:1001500061AB00084DAB000839AB0008BDEA0008F0
:100160004D6703084D6703084D6703084D67030893
:100170004D6703084D6703084D6703084D67030883
:080180004D6703084D670308F9
:1001880002020300881D0020841D002000000000DA
:100198000000000014000200042300205C2300205B
:1001A80000000000980500080B100C00401F0020FC
:1001B80060230020000000009A05000827000400C2
:1001C800902400209025002000000000A6050008CB
:1001D80016000800942500209C250020000000003F
:1001E800AA05000803123200AE2800207C2800204F
:1001F800000000000000000025005A00C827002069
:10020800222800200000000000000000F60108007D
:10021800C0270020B82700200000000000000000D0
:1002280001010400E4290020A03C00200000000097
:100238000000000008020900183C0020A43C00202F
:100248000000000001800008FA010100403C002085
:10025800B03C002000000000B205000802000C00BD
:10026800243C0020B43C00200000000000000000F6
:1002780003010600303D0020743D0020000000000E
:10028800B4050008000205007C3D0020A8400020BD
:1002980000000000000000001E000400843D002053
:1002A800B040002000000000BA05000822000C0041
:1002B80024400020B440002000000000BE050008D3
:1002C8000400C00098500020585100200000000091
:1002D80000000000F9010400CC450020185200205D
:1002E80000000000DDD5000818002C00984500200B
:1002F8001C520020000000005564020806001A0085
:10030800C440002048520020000000001DD502080B
:100318000E00DE0078520020A460002000000000DB
:10032800FDD4020813000400C85300208461002093
:1003380000000000CC0500080201030067520020FD
:10034800886100200000000021B00108150070003D
:100358007C7500206476002000000000000000008A
:100368000300010078750020D4760020000000000A
:10037800000000002A00600088740020D876002061
:1003880000000000853D02082C001000DC780020E9
:10039800CC78002000000000AD6002082B0024008B
:1003A80010790020EC780020000000007D60020831
:1003B80005000500F27900202C7B002000000000D9
:1003C800D005000812001600CA790020347B0020EE
:1003D80000000000D60500080C0024009C790020CD
:1003E8004C7B002000000000F9AF0108FD011E0051
:1003F800987D0020F47D0020000000006DD50008E5
:10040800FE010800847D0020147E0020000000000A
:10041800E95B0108290050006C810020F881002068
:10042800000000000000000001000A00A888002069
:10043800B488002000000000EC0500081A0008003D
:1004480094880020C088002000000000F6050008FD
:100458001B00F400E0880020708A002000000000E3
:1004680005D8010810000300548D0020588D002085
:1004780000000000FE05000828000C00488D002040
:100488005C8D00200000000002060008260008001D
:10049800408D0020688D0020000000000E06000836
:1004A80023000E00308D0020708D00200000000019
:1004B800F9BA020819000500288D0020808D002057
:1004C8000000000016060008F8010100248D002035
:1004D800888D0020000000001C06000800010400B0
:1004E800208D00208C8D0020000000001E060008D2
:1004F80034001000689300203C94002000000000A5
:10050800AD3D0208FB010100449200204C940020FC
:1005180000000000A15B0108FC0109000C9100200B
:1005280050940020000000006D5B0108F7010600F0
:10053800049100205C9400200000000022060008BE
:100548001F000E002C950020D4950020000000000C
:10055800280600080502010054950020E4950020B3
:1005680000000000360600080A0012000C9C00205B
:1005780054A4002000000000380600080D002C00DC
:10058800E09B002068A4002000000000D978020841
:1005980003002B21231E0101000001000A01200392
:1005A8000000C409000019012828230004010100E3
:1005B800000000000100C800141E010064002C01A6
:1005C80028000000080100000101030001000000EC
:1005D8000001000000000000000000000000000012
:1005E800000000000A0AE8030000640001007E051C
:1005F800EA05B40532000001050000000001000012
:1006080000000000000001155802D903C5030000CE
:1006180028010000040090010000240100000000EF
:1006280000000000000001000000000500000000BC
:1006380000300100005A0000000090012C01C800A1
:0206480064004C
:10064A005001000007000000020000000000000046
:10065A000000000001020304060708090101000066
:10066A00D8BA030840CD03080000000000000000CB
:10067A00E8BA0308F0BA03080000000001200000ED
:10068A00F4BA0308FCBA03080000000001400000A5
:10069A0000BB030868E60308000000000120000010
:1006AA000CBB030818BB030800000000040000008C
:1006BA001CBB030828BB030800000000040000005C
:1006CA002CBB03089CDD03080000000001000000A9
:1006DA00020000000000803F0000803FFF00000091
:1006EA00FFFFFFFF749C03080508040000000000D8
:1006FA00B49D0308509D0308609C03080000000095
:10070A00A09C030805080A0000000000B49D030825
:10071A00509D0308A0A70308000000000101010082
:10072A0024CC03080E00000069C60108000000007E
:10073A000000000060020020E8CB0308000000006F
:10074A0000000000000000000000000040CD030887
:10075A000000000000000000CC020020040000009D
:10076A0074CB03080C00000079CF01081807002099
:10077A000000000098CA03080C0000004DCF0108D1
:10078A000C0700200000000008CC03080800000045
:10079A00000000000007002004000000F8CB030856
:1007AA000C00000079D00108F406002000000000C7
:1007BA0084CA0308030000007D910208DC060020B9
:1007CA000000000000CC0308030000007D9102082D
:1007DA00C40600200000000088CA030801000000C7
:1007EA0000000000000000000000000000000000FF
:1007FA000D000000000000000000000000000000E2
:10080A00E8CB030800000000000000000000000020
:10081A000000000040CD03080000000000000000B6
:10082A00CC0200200400000018CB030803000000DB
:10083A0051C80108AC06002008000000F8CB0308E4
:10084A000C00000079D00108F40600200000000026
:10085A0084CA0308030000007D910208DC06002018
:10086A000000000000CC0308030000007D9102088C
:10087A00C40600200000000088CA03080100000026
:10088A00000000000000000000000000000000005E
:10089A000D00000000000000000000000000000041
:1008AA0010CC030800000000000000000000000057
:1008BA000000000040CD0308000000000000000016
:1008CA00CC0200200400000020CB03080300000033
:1008DA007D910208240700200000000088CA03084E
:1008EA0001000000000000000000000000000000FD
:1008FA00000000000D0000000000000000000000E1
:10090A000000000000FFFF00000000002D202D2D38
:10091A00202D2D2D2D202D2D2D0000000000000052
:10092A0000000000000000000000002D202D2D20F6
:10093A002D2D2D2D202D2D2D2D0000000000000025
:10094A00000000000000000000000000010000009C
:10095A00C0120000000000000102030401020304A7
:10096A0006070809EC3C002088130C170100000058
:10097A00EE3C002088130C17000000005CCA030834
:10098A00000000000000000000000000000000005D
:10099A006CCA0308080000000000000030030020B1
:1009AA000400000078CA03080800000000000000E4
:1009BA00240300200000000084CA03080400000089
:1009CA0075CE0108000000000000000088CA030874
:1009DA00010000000000000000000000000000000C
:1009EA00000000000D0000000000000000000000F0
:1009FA0000000000EA3C002088130C1701000000E8
:100A0A00E83C002088130C1700000000C8CA03083D
:100A1A000E000000BDC60108000000000000000032
:100A2A003C030020FB3C002001000000749D0308E9
:100A3A00E73C002001000000809D0308F03C0020F4
:100A4A0002000000889D03080A73002000000000CD
:100A5A0000000000087300200000000000000000F1
:100A6A00067300200000000000000000047300204C
:100A7A0000000000000000000273002000000000D7
:100A8A0000000000007300200000000000000000C9
:100A9A00100300200000000000000000E63C0020D7
:100AAA0002000000949D0308D0CA03080000000059
:100ABA000000000000000000000000006CCA0308EB
:100ACA000800000000000000C0030020040000002D
:100ADA0078CA03080800000000000000B4030020E0
:100AEA000000000084CA0308040000009DC6010833
:100AFA00000000000000000088CA0308010000008E
:100B0A0000000000000000000000000000000000DB
:100B1A000D000000000000000000000000000000BE
:100B2A00E0CA030800000000000000000000000006
:100B3A0000000000F0CA03080C000000CDCE010836
:100B4A00FC03002004000000FCCA03080C0000009B
:100B5A00E1C60108F00300200400000008CB0308E6
:100B6A000C00000091CE0108E40300200000000000
:100B7A0014CB03080300000071C80108CC0300204D
:100B8A000800000020CB0308030000007D91020842
:100B9A00240700200000000088CA030801000000A2
:100BAA00000000000000000000000000000000003B
:100BBA000D0000000000000000000000000000001E
:100BCA0028CB03080000000000000000000000001D
:100BDA000000000030CB030804000000FDCF01082C
:100BEA00000000000000000088CA0308010000009D
:100BFA0000000000000000000000000000000000EB
:100C0A000D000000000000000000000000000000CD
:100C1A007CCB030800000000000000000000000078
:100C2A000000000098C803080C0000000000000043
:100C3A005C040020040000008CCB030808000000BC
:100C4A0000000000500400200400000098CB0308B4
:100C5A000800000000000000440400200400000016
:100C6A00A0CB0308080000000000000038040020A0
:100C7A0004000000A8CB03080800000000000000E0
:100C8A002C04002004000000B0CB03080800000078
:100C9A00000000002004002004000000B8CB030874
:100CAA0008000000000000001404002004000000F6
:100CBA00C0CB030808000000000000000804002060
:100CCA000400000088CA03080100000000000000B8
:100CDA000000000000000000000000000D000000FD
:100CEA00000000000000000000000000C8CB03085C
:100CFA000E000000ADC60108000000000000000060
:100D0A0068040020D0CB03080E0000000000000099
:100D1A000000000000000000E0040020D8CB030817
:100D2A000E000000000000000000000000000000AB
:100D3A0080050020403D002004000000A09D03081B
:100D4A00E23C0020E0150C1700000000E53C002002
:100D5A0008000000509D0308E43C00200500000044
:100D6A00B49D0308E0CB03080E0000000000000059
:100D7A000000000000000000D00500200000803FB5
:100D8A0004030904120100020202004083044057CE
:100D9A00000201020301000009024300020100C02F
:100DAA0032090400000102020100052400100105B5
:100DBA002401000104240202052406000107058219
:100DCA00030800FF09040100020A000000070501E8
:100DDA00024000000705810240000000FF000000F9
:100DEA00615C0208815B020885560208015202080A
:100DFA0035550208115202082D520208E12F020845
:100E0A00D12F0208000000000000000001000000CD
:100E1A007D32020835320208093602080000000055
:100E2A00A92F02088931020809320208F1300208A2
:100E3A0000000000000000009D2F02081D2F02087C
:100E4A00192F0208152F0208092F0208052F020878
:100E5A00112F02080D2F0208912F0208852F020870
:100E6A005D2F0208712F0208492F0208352F020848
:100E7A00212F020820700020702D7200000000004F
:100E8A0000010000000000000000000074D4030804
:100E9A000E0000000000000000000000000000003A
:100EAA0048150020FFFFFFFFFA00000001000000C4
:100EBA000100000028CB0308000000000000000029
:100ECA0000000000000000002FD00308040000000A
:100EDA0039CA0108000000000000000088CA03089F
:100EEA0001000000000000000000000000000000F7
:100EFA00000000000D0000000000000000000000DB
:100F0A0000000000EE2200200100C40900000000D9
:100F1A00EC2200200100C40900000000EA2200209F
:100F2A000100C40900000000E82200200100C409F1
:100F3A0000000000E42200200100C40900000000B3
:100F4A00E62200200100C40900000000E22200207D
:100F5A000100C40900000000E02200200100C409C9
:100F6A00000000005CD003080E0000000000000032
:100F7A000000000000000000740800202C3D002042
:100F8A009CFF2C0100000000DC0000200A00000089
:100F9A00A0A70308D03C0020E0150C1700000000B1
:100FAA00DE00002008000000509D0308DD0000203C
:100FBA0005000000B49D0308D23C00200200000096
:100FCA00B8A70308F879002001200100F77900206A
:100FDA0002000000C4A703085E5300200000F401C9
:100FEA00010000005C5300200000F4010100000031
:100FFA005A5300200000F401010000005853002059
:10100A000000F401010000005653002000FF010017
:10101A009A790020E803D0070A0000009879002096
:10102A00006401000A0000009979002000640100B0
:10103A000A00000092790020006401000A00000002
:10104A0097790020006401000A00000096790020C8
:10105A00006401000A000000957900200064010084
:10106A000A0000009179002000FF01000A00000038
:10107A009079002000FF01000A000000745200204D
:10108A000000F40101000000725200200000F40187
:10109A0001000000705200200000F401010000006D
:1010AA006E5200200000F401010000008D7900203A
:1010BA0000C801008C79002000C801008B7900204B
:1010CA0000C801008A790020006401000A000000BB
:1010DA008979002000FF01000A000000C979002078
:1010EA0000C80100C879002000C80100C7790020A3
:1010FA0000C80100C679002000C80100C579002097
:10110A0000C80100C479002000C80100C37900208A
:10111A0000C80100C279002000C80100C17900207E
:10112A0000C8010064D003080000000000000000AD
:10113A00000000000000000074D00308090000004D
:10114A000000000018090020040000007CD00308F9
:10115A0009000000000000000C0900200400000043
:10116A0024D3030809000000000000000009002041
:10117A000400000084D003080900000000000000F9
:10118A00F40800200400000088D0030809000000C9
:10119A0000000000E80800200400000090D00308C6
:1011AA000900000000000000DC0800200400000024
:1011BA0098D003080900000000000000D0080020B1
:1011CA0004000000A0D0030809000000000000008D
:1011DA00C40800200400000088CA030801000000B7
:1011EA0000000000000000000000000000000000F5
:1011FA000D000000000000000000000000000000D8
:10120A00A8D0030800000000000000000000000051
:10121A0000000000B8D0030805000000000000002C
:10122A006D5200200000000088CA03080100000077
:10123A0000000000000000000000000000000000A4
:10124A000D00000000000000000000000000000087
:10125A00C0D00308000000000000000000000000E9
:10126A000000000040CD030800000000000000005C
:10127A00EB02002004000000CCD003080C000000A0
:10128A00D1CA0108780900200000000074CB0308C5
:10129A000C000000ADC501086C0900200000000028
:1012AA0098CA03080C00000091C5010860090020D3
:1012BA000000000008CC030808000000000000003D
:1012CA005409002004000000F8CB03080C000000B9
:1012DA00FDC401084809002000000000D0D003081E
:1012EA0009000000000000003C0900200400000082
:1012FA0084CA0308030000007D9102082409002023
:10130A000000000088CA0308010000000000000075
:10131A000000000000000000000000000D000000B6
:10132A00000000000000000000000000D8D0030800
:10133A0000000000000000000000000000000000A3
:10134A00E8D003080C000000000000008C0900200F
:10135A0000000000F0D003080A00000000000000AE
:10136A00547A002000000000FCD003080A000000A4
:10137A00000000005C7A00200000000004D103088D
:10138A000A00000000000000647A0020000000004B
:10139A000CD10308070000000000000084090020A7
:1013AA000000000018D1030804000000B9920208E6
:1013BA00000000000000000088CA030801000000C5
:1013CA000000000000000000000000000000000013
:1013DA000D000000000000000000000000000000F6
:1013EA0024D10308000000000000000000000000F3
:1013FA000000000038D103080700000000000000C8
:10140A00C80900200000000044D1030808000000B9
:10141A0000000000BC0900200000000050D10308B1
:10142A000800000000000000B009002000000000D1
:10143A005CD103080800000000000000A409002095
:10144A000000000068D10308080000000000000046
:10145A00980900200000000088CA03080100000063
:10146A000000000000000000000000000000000072
:10147A000D00000000000000000000000000000055
:10148A0074D10308000000000000000037080020A3
:10149A000000000080D103080B00000000000000DB
:1014AA00300A00200000000088D103080B00000069
:1014BA0000000000240A00200000000094D1030864
:1014CA000B00000000000000180A002000000000C5
:1014DA00A0D103080B000000000000000C0A002045
:1014EA0000000000ACD103080B000000000000005F
:1014FA00000A002000000000B8D103080B00000019
:10150A0000000000F409002000000000C0D1030818
:10151A000B00000000000000E809002000000000A5
:10152A00CCD103080B00000000000000DC090020F9
:10153A0000000000D8D103080800000000000000E5
:10154A00D00900200000000088CA0308010000003A
:10155A000000000000000000000000000000000081
:10156A000D00000000000000000000000000000064
:10157A00E4D10308000000000000000000000000A1
:10158A0000000000F8D10308080000000000000075
:10159A00600A00200000000004D2030808000000CE
:1015AA0000000000540A00200000000010D20308C6
:1015BA000800000000000000480A002000000000A7
:1015CA001CD2030808000000000000003C0A0020AA
:1015DA000000000088CA03080100000000000000A3
:1015EA000000000000000000000000000D000000E4
:1015FA0000000000000000000000000024D20308E0
:10160A000000000000000000340800200000000074
:10161A0034D203080B00000000000000900A0020EA
:10162A000000000040D203080B0000000000000088
:10163A00840A0020000000004CD2030807000000C2
:10164A00000000007C0A00200000000058D20308B5
:10165A000700000000000000740A002000000000DB
:10166A0064D2030807000000000000006C0A002092
:10167A000000000088CA0308010000000000000002
:10168A000000000000000000000000000D00000043
:10169A0000000000000000000000000070D20308F3
:1016AA0000000000000000003408002000000000D4
:1016BA007CD203080700000000000000DC0A0020BA
:1016CA000000000084D203080700000000000000A8
:1016DA00D40A0020000000008CD203080700000092
:1016EA0000000000CC0A00200000000094D2030889
:1016FA000700000000000000C40A002000000000EB
:10170A009CD203080700000000000000BC0A002069
:10171A0000000000A4D20308070000000000000037
:10172A00B40A002000000000ACD203080700000041
:10173A0000000000AC0A002000000000B4D2030838
:10174A000700000000000000A40A002000000000BA
:10175A00BCD2030807000000000000009C0A002019
:10176A000000000088CA0308010000000000000011
:10177A000000000000000000000000000D00000052
:10178A00000000000000000000000000C4D20308AE
:10179A000E00000000000000091E02080000000000
:1017AA00E40A00206B5200200A3201006A5200202B
:1017BA0001FA01006652002000C8010064520020AC
:1017CA00E803D0070100000046465F464F525449DD
:1017DA004E49463400000000CCD203080E00000037
:1017EA001F1E020800000000AB230208C00B0020E5
:1017FA00D4D203080E00000039C501080000000019
:10180A0000000000100C0020DCD203080E000000CB
:10181A0099920208919002085D8F0208EC0C002050
:10182A00E4D203080E000000E98D0208891E0208AE
:10183A0000000000A00D0020ECD203080E000000FA
:10184A00698E02089D8E020800000000400E0020EA
:10185A008E79002001030100F8D203080E0000006F
:10186A00651E0208411E020800000000300F002019
:10187A0000D303080E000000258E0208BF8F02085D
:10188A0000000000BC0F00200CD303080E0000006B
:10189A00C18E020805900208000000005C100020BA
:1018AA00887900200103010014D303080000000016
:1018BA0000000000000000000000000020D3030820
:1018CA0008000000000000007C1100200000000059
:1018DA0028D303080700000000000000741100204C
:1018EA000000000038D303080700000000000000D1
:1018FA006C1100200000000044D303080700000018
:10190A0000000000641100200000000050D303080A
:10191A00030000007D9102084C1100200000000025
:10192A0088CA03080100000000000000000000004F
:10193A0000000000000000000D0000000000000090
:10194A00000000000000000058D303080000000057
:10195A0000000000000000000000000068D3030837
:10196A000A0000000000000038BB03080000000065
:10197A0070D303080A0000000000000078D30308AF
:10198A000000000080D303080A00000000000000E5
:10199A00E07900200000000088D303080A00000054
:1019AA0000000000881100200000000088CA030817
:1019BA00010000000000000000000000000000001C
:1019CA00000000000D000000000000000000000000
:1019DA000000000090D3030800000000000000008F
:1019EA00000000000000000058BC030803000000CB
:1019FA007D910208C811002000000000A4D303084A
:101A0A00030000007D910208E000002000000000B1
:101A1A00ACD30308030000007D910208B011002036
:101A2A0000000000B4D30308030000007D910208FF
:101A3A00981100200000000088CA03080100000075
:101A4A00000000000000000000000000000000008C
:101A5A000D0000000000000000000000000000006F
:101A6A00C0D30308000000000000000000000000CE
:101A7A0000000000CCD303080700000051900208C0
:101A8A00601200200000000070EC03080300000050
:101A9A007D9102084812002000000000D8D30308F4
:101AAA00030000007D9102083012002000000000AF
:101ABA00E0D30308030000007D91020818120020F9
:101ACA0000000000E8D30308070000003590020870
:101ADA00101200200000000090CB03080300000051
:101AEA007D910208F811002000000000F4D30308D9
:101AFA00030000007D910208E011002000000000B0
:101B0A0088CA03080100000000000000000000006D
:101B1A0000000000000000000D00000000000000AE
:101B2A00000000000000000000D403080E000000BE
:101B3A00DD1D0208AF1D0208000000006812002027
:101B4A0008D403080E000000318F020800000000CC
:101B5A00000000000813002014D403080E0000003F
:101B6A0000000000000000000000000094130020A4
:101B7A0024D403080E000000098F0208719002089D
:101B8A0000000000201400202CD4030800000000EC
:101B9A0000000000000000000000000038D4030824
:101BAA00030000007D9102083015002000000000AB
:101BBA0018D40308030000007D91020818150020BC
:101BCA000000000040D40308030000007D910208D1
:101BDA0000150020000000004CD403080300000098
:101BEA007D910208E81400200000000054D4030884
:101BFA000200000005930208000000000000000037
:101C0A005CD40308020000000593020801000000EA
:101C1A000000000068D403080200000005930208CF
:101C2A000200000000000000000000000D0000009B
:101C3A0000000000000000000000000000600240F8
:101C4A001060024000000000000B000000002000AD
:101C5A00000000000000000000600240286002400E
:101C6A0000000000060C0000000020000000000038
:101C7A0000000000006002404060024000000000D6
:101C8A00100D00000000200000000000000000000D
:101C9A00006002405860024000000000160E00007A
:101CAA000000200000000000000000000060024068
:101CBA007060024000000000200F000000002000B9
:101CCA00000000000000000000600240886002403E
:101CDA0000000000261000000000200000000000A4
:101CEA000000000000600240A06002400000000006
:101CFA003011000000002000000000000000000079
:101D0A0000600240B860024000000000362F000068
:101D1A0000002000000000000000000000640240F3
:101D2A00106402400000000000380000000040007B
:101D3A000000000000000000006402402864024025
:101D4A00000000000639000000004000000000000A
:101D5A0000000000006402404064024000000000ED
:101D6A00103A0000000040000000000000000000DF
:101D7A00006402405864024000000000163B000064
:101D8A000000400000000000000000000064024063
:101D9A007064024000000000203C00000000400087
:101DAA000000000000000000006402408864024055
:101DBA00000000002644000000004000000000006F
:101DCA000000000000640240A0640240000000001D
:101DDA003045000000004000000000000000000044
:101DEA0000640240B8640240000000003646000069
:101DFA000000400000000000000000000101000097
:101E0A006DC102080000000000000000010000008F
:101E1A000000803F00000101FFFF00004CC60308DC
:101E2A00000000000000000035B00108A086010093
:101E3A000400000000000000000000000000000094
:101E4A000000000000000000000000000000000088
:101E5A0070EC0308B0C503080000000099090108E6
:101E6A007D000000060000000000000000000000E5
:101E7A000000000000000000000000000000000058
:101E8A0000000000DCEA0308000000000000000077
:101E9A0039560308E80300000300000000000000B0
:101EAA000000000000000000000000000000000028
:101EBA000000000000000000E4EA0308000000003F
:101ECA00000000001DD602081027000003000000D1
:101EDA0000000000000000000000000000000000F8
:101EEA00000000000000000000000000F0EA030803
:101EFA000000000059C502082D710108204E00009B
:101F0A0005000000000000000000000000000000C2
:101F1A0000000000000000000000000000000000B7
:101F2A00A4C703080000000000000000F5500308E1
:101F3A00102700000100000000000000000000005F
:101F4A000000000000000000000000000000000087
:101F5A0000000000F4EA030800000000000000008E
:101F6A00395B0108E80300000500000000000000DA
:101F7A000000000000000000000000000000000057
:101F8A00000000000000000000EB03080000000051
:101F9A0000000000FDB20108204E0000030000000E
:101FAA000000000000000000000000000000000027
:101FBA0000000000000000000000000010EB030811
:101FCA000000000000000000F5B00108204E0000EB
:101FDA0003000000000000000000000000000000F4
:101FEA0000000000000000000000000000000000E7
:101FFA0020EB03080000000000000000554F030812
:10200A00400D030003000000000000000000000073
:10201A0000000000000000000000000000000000B6
:10202A0000000000E0BB0308000000000000000000
:10203A00C58B020810270000010000000000000004
:10204A000000000000000000000000000000000086
:10205A000000000000000000BCC5030800000000EA
:10206A000000000039ED01081027000003000000FD
:10207A000000000000000000000000000000000056
:10208A0000000000000000000000000024BC03085B
:10209A000000000000000000595A0308A00F0000C9
:1020AA000100000000000000000000000000000025
:1020BA000000000000000000000000000000000016
:1020CA0030EB030800000000000000001DF40208C5
:1020DA0010270000010000000000000000000000BE
:1020EA0000000000000000000000000000000000E6
:1020FA000000000004C803080000000000000000FF
:10210A00D13203081027000001000000000000007F
:10211A0000000000000000000000000000000000B5
:10212A000000000000000000A4C503080000000031
:10213A0000000000499402081A4100000100000052
:10214A000000000000000000000000000000000085
:10215A000000000000000000000000003CEB030843
:10216A000000000000000000355A0308400D03007B
:10217A000000000000000000000000000000000055
:10218A000000000000000000000000000000000045
:10219A0044EB03080000000000000000697902080F
:1021AA00A0860100030000000000000000000000FB
:1021BA000000000000000000000000000000000015
:1021CA000000000001000000000101010101AA5500
:1021DA0003009FAA5505010000AA550B010000AA99
:1021EA005507010000AA550902000000430000003B
:1021FA0000000000000000000000000000000000D5
:10220A000000000000000000000000004300000081
:10221A0000000000000000000000000000000000B4
:10222A000000000000000000000000004300000061
:10223A000000000000000000000000000000000094
:10224A000000000000000000000000004300000041
:10225A000000000000000000000000000000000074
:10226A000000000000000000000000004300000021
:10227A000000000000000000000000000000000054
:10228A000000000000000000000000004300000001
:10229A000000000000000000000000000000000034
:1022AA0000000000000000000000000043000000E1
:1022BA000000000000000000000000000000000014
:1022CA00000000000000000000000000396C030854
:1022DA00796A0308000000001EEF03082AD00308E9
:1022EA0052CE030852CE030852CE030852CE030838
:1022FA0052CE030852CE030852CE030852CE030828
:10230A0052CE0308FFFFFFFFFFFFFFFFFFFFFFFFA4
:10231A00FFFF00000100415343494900000000004B
:10232A0000000000000000000000000000000000A3
:10233A00000000000000415343494900000000002A
:10234A000000000000000000000000000000000083
:10235A0000000000000000001C1D0020000000001A
:10236A000000000000000000000000000000000063
:10237A000000000000000000000000000000000053
:10238A000000000000000000000000000000000043
:10239A000000000000000000000000000000000033
:1023AA000000000000000000000000000000000023
:1023BA000000000000000000000000000100000012
:10800000152303701623C370172383713A238370DB
:108010003B2343713C230372704740F2E93300E095
:10802000A3B10289013B12F0020F9BB2F8D089B2D2
:10803000818140F2E93300E043B10289013B12F053
:10804000010F9BB2F8D08089C0B27047094A9042B4
:1080500005D0094B984201D0FF2070470223074A00
:1080600002EB03135A89013292B25A815889C0B285
:10807000704700BF00300140003C0040707B002092
:10808000F0B5446814B12568A4886C8341F0800180
:10809000046840F2E93501E0002D54D02689013D05
:1080A00016F0020FADB2F7D089B2A18140F2E931EA
:1080B00001E0002958D02589013915F0010F89B256
:1080C000F7D0A189A1894FF0000C4FF47A714FF6D7
:1080D000FF764FF0FF0E624502D12DE0B1421BD07A
:1080E0002589013915F0020589B2F7D0A4F80CE012
:1080F0004FF47A7102E0B9B2B1420DD0258915F082
:10810000010501F1FF37F6D0A589ADB20BB11D70A5
:1081100001330CF1010CDEE71B4B9C4204D0A3F5AC
:1081200074439C4208D10225184B03EB05156B895B
:1081300001339BB26B816B89436813B11A689B88CA
:1081400013830120F0BD10498C4204D0A1F5744185
:108150008C42B7D102250D4901EB05156989013122
:1081600089B269816989ADE7074DAC4203D00849FE
:108170008C42A7D10221054D05EB01114D89013536
:10818000ADB24D8149899DE700300140707B0020F0
:10819000003C004030B4446814B12368A5885D8376
:1081A000036840F2E93001E0002832D01D8901382F
:1081B00015F0020F80B2F7D089B2998140F2E9310F
:1081C00001E0002947D01889013910F0010F89B268
:1081D000F7D0998940F2E93100E059B318890139A3
:1081E00010F0020F89B2F8D092B29A8140F2E932CF
:1081F00001E0002A3FD01989013A11F0010F92B233
:10820000F7D09B8914B12368A2881A83012030BC5F
:10821000704721498B4204D0A1F574418B42D9D1DA
:1082200002201E4901EB00104189013189B24181D0
:108230004189CFE7184A934204D0A2F57442934291
:10824000E0D10221154B03EB01114B8901339BB2A5
:108250004B814B89D6E71048834203D010498B42AB
:10826000B8D102210D4800EB01114889013080B2DC
:1082700048814989AEE708498B4203D0084A9342B6
:10828000C0D10222054B03EB0212538901339BB28A
:1082900053815389B6E700BF00300140707B002056
:1082A000003C0040002870B51EDB0928044620DD94
:1082B000012303EB83035B00B0FBF3F2092AF8D838
:1082C0007BB10E4EB4FBF3F00928CCBF572230220D
:1082D000A6FB03E5024403FB1044EB0801F8012B65
:1082E000F0D100230B7070BD2D230B704042013183
:1082F000DBE7303001F8010BF3E700BFCDCCCCCC8D
:10830000884230B44FF001042ED301FB04F4B0FBDB
:10831000F4F58D42F9D284B1AAB901E0B0FBF4F5CD
:10832000092DCCBF572230222A4404FB150003F844
:10833000012BB4FBF1F4002CF0D100221A7030BCF8
:108340007047B0FBF4F5092DCCBF372230222A4408
:1083500004FB150003F8012BB4FBF1F4002CF0D161
:1083600000221A7030BC70470546002AEBD1D7E7CF
:1083700003685A1C0260197070472DE9F047089C89
:108380002578002B804689460CBF4FF0200A4FF01D
:10839000300A661C35B3002A29DD334601E0024667
:1083A00098B113F8011B501E0029F8D1971E60B137
:1083B0003D46013D51464046C8476B1C002BF8DC4A
:1083C000257827EAE770013055B1041B294640465D
:1083D000C847301916F8015B002DF7D1BDE8F087CA
:1083E000BDE8F087002A04DC2846BDE8F0870020BD
:1083F000EBE7571EDCE70A44914251D030B441F21A
:10840000210411F8013B80EA0320430010F4004FDF
:1084100084EA03059BB2ADB208BF1D466B0015F49C
:10842000004F84EA03009BB280B208BF18464300A5
:1084300010F4004F84EA03059BB2ADB208BF1D469D
:108440006B0015F4004F84EA03009BB280B208BFB2
:108450001846430010F4004F84EA03059BB2ADB206
:1084600008BF1D466B0015F4004F84EA03009BB261
:1084700080B208BF1846430010F4004F84EA030599
:108480009BB2ADB208BF1D466B0084EA030015F431
:10849000004F85B298B218BF28468A42B1D130BC8D
:1084A000704783684268D0ED037A00EB83010133A3
:1084B000934281ED040A836004BF0023836000EBD4
:1084C000830393ED047A036870EE277A9A42C0ED35
:1084D000037A77EEC77AC0ED037A0CDA013307EE40
:1084E000103AF8EEC76AB7EE007A87EEA60A036084
:1084F00030EE070A704707EE102AB8EEC77A87EE0B
:10850000870A704790ED097A90ED004AD0ED0A6A2B
:10851000D0ED014AD0ED047A90ED035AD0ED025A25
:10852000A4EE007AB0EE406AB0EE470AB0EE667A8A
:10853000A6EE247A67EEC07AA0EE457AE6EE257ABA
:1085400080ED097AC0ED0A7A7047D0ED057A90ED9A
:10855000013AD0ED003AD0ED064A90ED024A90ED96
:10856000077A90ED035A90ED086AD0ED045AC0EDF9
:10857000067AF0EE406A27EE830AC0ED056AA3EEA4
:10858000A60A80ED087AA4EE240AA5EE470AA5EE15
:10859000C60A80ED070A7047D0ED007A90ED017AA7
:1085A00030EE670AE7EE007AB0EE670AC0ED007AB7
:1085B000704770474FF40063038270474FF40063C5
:1085C000038270474FF40063038270474FF4805377
:1085D00003827047BFF34F8F0549064BCA6802F408
:1085E000E0621343CB60BFF34F8F00BFFDE700BFD6
:1085F00000ED00E00400FA0570B4037B04681F2B53
:1086000008D9203B2021626801FA03F31A421CD1E9
:1086100070BC70472021226801FA03F31A42F7D098
:1086200042691449582000FB021251685689CD68EE
:108630000868296821F001012960828992B222EA42
:1086400006028281A36070BC7047426909495820C4
:1086500000FB021251685689CD680868296821F02C
:1086600001012960828992B222EA06028281E360D6
:1086700070BC7047F040002030B4094B1C786CB1DE
:10868000084A002502EBC404116893884D6288896A
:10869000083203439BB2A2428B81F5D130BC7047B4
:1086A000104500201445002010B4037B01681F2BE7
:1086B00009D9203B20224C6802FA03F31C4214D152
:1086C0005DF8044B704720220C6802FA03F31C4249
:1086D000F6D00C4A40680024147002685DF8044B20
:1086E00022F0010202608B607047064A4068002455
:1086F000147002685DF8044B22F001020260CB6046
:10870000704700BFE389002090F8493013B1002280
:1087100080F849201846704770B5044682B018307A
:10872000256D94F85C106B460622A847A8B19DF809
:1087300004009DF800609DF801109DF802509DF81E
:1087400003209DF8053041EA062143EA002342EA6E
:108750000522A184E2842385012002B070BD70B59A
:10876000044682B00830256A6B4606223B21A847A2
:10877000A8B19DF804009DF800609DF801109DF8D7
:1087800002509DF803209DF8053041EA062143EA96
:10879000002342EA05226182A282E382012002B024
:1087A00070BD50F8043C012280F83520143803B124
:1087B00018477047F8B50468C4F30D0405460E4623
:1087C00004B32F681DF01CFC092840F08880454C3C
:1087D000236923F440732361236943F40073236105
:1087E000236943F0010323613E601DF009FC236906
:1087F000092823F00103236171D12B6804332B6016
:108800000020F8BD384B394A93422BD902F58042FB
:10881000934226D902F5804293422AD902F580423A
:10882000934228D902F58032934226D902F50032CC
:10883000934224D902F50032934222D902F5003244
:10884000934220D902F5003293421ED902F58022CC
:1088500093421CD9B3F1016F1BD3052005F054FDE1
:10886000FBE708241DF0CCFB092814D04FF0FF30A3
:10887000F8BD1024F6E71824F4E72024F2E72824B2
:10888000F0E73024EEE73824ECE74024EAE7482418
:10889000E8E75824E6E7134F3B6923F440733B6154
:1088A0003B6943F400733B613B6923F0F8033B6190
:1088B0003B6943F002031C433C613B6943F4803352
:1088C0003B611DF09DFB3B6923F002033B613B696B
:1088D000092823F0F8033B613FF473AFC6E76FF05C
:1088E0000100F8BD003C024000400008FF3F0008C6
:1088F000F8B504460D468E180027B54201D120690F
:10890000F8BDE368591CE160234415F8012B1A7285
:108910000429F2D1206918B9A1682046FFF74AFF5F
:108920002061E760E9E7024B186806F063BA00BF10
:1089300098A40020F8B5027B466903681F2A2DD948
:10894000A2F120055F682024AC402742114617D0D1
:108950001022AA40DC60DA605A68EA40D40749D4A1
:10896000716B756A0A68B46A22F00102A5420A6056
:1089700037D1012286F84C20027B11461F2A20D9CC
:108980002039082258688A40024200D0DA60042266
:10899000586802FA01F1014221D1F8BD20241D6876
:1089A0009440254211460CD0102191409C60996062
:1089B0001968D140C907D3D5012101FA02F29A60A2
:1089C000CEE7082218688A40024200D09A6004224A
:1089D000186802FA01F101420BD09960F8BDD96024
:1089E000F8BD0446304606F0A1F9227B2368114603
:1089F000C4E7F8BD012202FA05F5DD60B0E770B505
:108A000082B004466946183021F026FCA8B19DF8D2
:108A100005009DF801609DF802109DF803509DF837
:108A200004209DF8063041EA062143EA002342EA89
:108A30000522A184E2842385012002B070BD0028B4
:108A400055D0026802F13F4303F57E032DE9F04F54
:108A50009B0A544DEB5C03F01F055B090124032BBB
:108A600004FA05F444D0042B00F09780022B44D084
:108A700001F00306731E012BC1F3810CC1F3001832
:108A80008588C1F341113DD90024234601274FF0C9
:108A9000030E03E0102B04F1020426D007FA03F0C2
:108AA000A84303F10103F5D1D2F800C00EFA04F097
:108AB000C04300EA0C0CC2F800C0D2F8008006FAED
:108AC00004FC4CEA080CC2F800C0D2F80CC000EA62
:108AD0000C00D060D2F80CC001FA04F040EA0C009F
:108AE000102BD06004F10204D8D1BDE8F08F70479C
:108AF0002D4B1D6C2C431C64BAE72B4B5D6C2C4337
:108B00005C64B5E7002003464FF0010E4FF0030907
:108B100004E00133102B00F102003CD00EFA03F701
:108B200037EA0504F5D1D2F800A009FA00F4E443CD
:108B30000AEA040AC2F800A0D2F800B006FA00FA65
:108B40004AEA0B0AC2F800A0D2F808A004EA0A0A0E
:108B5000C2F808A0D2F808B00CFA00FA4AEA0B0AE8
:108B6000C2F808A0D2F804A02AEA07075760D2F892
:108B700004A008FA03F747EA0A075760D7683C40A1
:108B8000D460D76801FA00F401333C43102BD46061
:108B900000F10200C2D1BDE8F08F034B1D6B2C43E6
:108BA0001C6365E7D8A703080038024010B10368CA
:108BB00082885A83704710B1036882881A8370478D
:108BC00010B5014600BF064C2068FFF7EFFF0548CF
:108BD000FFF723FA2068FFF7EEFF00BF10BD00BFCC
:108BE000443C0020003C004018B10368828809B969
:108BF0005A8370471A83704730B1036882881B69B3
:108C00001A4214BF01200020704738B590F84D304B
:108C100003B938BD0446184605F048F90546FFF784
:108C2000EBFF01460028F4D1D5B12023E871AB71E8
:108C30002846FFF704FF21460F4B41F8143F284612
:108C400021F09CFAAB88B3FA83F3C3F11F0301222E
:108C500012FA03F3DDD009490A6813430B6038BDEB
:108C60002946FFF7ECFE2146034B41F8143F284606
:108C7000BDE8384021F082BAA3870008003C0140DB
:108C800038B5044600F11805FFF7BFFF636D802279
:108C90006B2128469847642005F02CFE636D07225F
:108CA000682128469847642005F024FE636D002261
:108CB0006B2128469847642005F01CFE636D012255
:108CC0006B21284698470F2005F014FE94F84720A2
:108CD000636D022A8CBF1A2218221B21284698474E
:108CE0000F2005F007FE636D18221C2128469847C7
:108CF0000F2005F0FFFD636D94F846201A212846E9
:108D000098470F2005F0F6FD636D94F8482019216F
:108D100028469847642005F0EDFD636D1022372149
:108D2000284698470F2005F0E5FD2846636D01228F
:108D3000382198470F20BDE8384005F0DBBD10B55D
:108D400004460120A269138823F040031B041B0C76
:108D5000138013889BB223F0380343F03003138051
:108D600013889BB243F04003138005F069FD204651
:108D7000FFF786FF10226A2104F11800FFF70AFAB4
:108D8000642005F0B7FDA06921F05AF80120BDE884
:108D9000104005F055BD38B505460446FFF735FFD0
:108DA00055F8180F21F074F8636D80226B21284666
:108DB0009847642005F09EFD636D032268212846D4
:108DC0009847642005F096FD636D01226B212846CB
:108DD00098470F2005F08EFD94F84720636D022A16
:108DE0008CBF1A2218221B21284698470F2005F015
:108DF00081FD636D18221C21284698470F2005F03D
:108E000079FD636D94F846201A21284698470F2073
:108E100005F070FD636D94F84820192128469847A5
:108E2000642005F067FD636D1022372128469847BE
:108E30000F2005F05FFD2846636D01223821984719
:108E4000A069BDE8384021F00FB8F8B5434E04469C
:108E5000FFF7DBFE3778C7B104F11805A06921F0F0
:108E600017F894F846201A212846FFF793F90120B5
:108E700005F0E6FCA06920F0E3FF2046FFF74CFC7C
:108E800094F9263001335FD0F8BD254655F8180F08
:108E900020F0FEFF80226B212846FFF77BF9962009
:108EA00005F028FD032268212846FFF773F9962074
:108EB00005F020FD03226B212846FFF76BF90F20F8
:108EC00005F0BEFC10226A212846FFF763F90F2047
:108ED00005F0B6FC3A466C212846FFF75BF90F20F7
:108EE00005F0AEFC94F8482019212846FFF752F906
:108EF0000F2005F0A5FC18221B212846FFF74AF990
:108F00000F2005F09DFC10221C212846FFF742F996
:108F10000F2005F095FC102237212846FFF73AF97B
:108F20000F2005F08DFC012238212846FFF732F989
:108F30000F2005F085FCA06920F082FF012005F0DC
:108F40007FFC0123337089E794F9243001339BD1EE
:108F50000620BDE8F84005F0D7B900BF801D00200D
:108F60002DE9F0410B4E346873691C400FD0DFF8D7
:108F700028800127B4FA84F3C3F11F0307FA03F52D
:108F800058F8230003689847AC437561F2D1BDE8F7
:108F9000F08100BF003C0140287D00202DE9F04118
:108FA0000B4E346873691C400FD0DFF8288001270E
:108FB000B4FA84F3C3F11F0307FA03F558F823004A
:108FC00003689847AC437561F2D1BDE8F08100BFFA
:108FD000003C0140287D00202DE9F0410B4E346813
:108FE00073691C400FD0DFF828800127B4FA84F39E
:108FF000C3F11F0307FA03F558F8230003689847E5
:10900000AC437561F2D1BDE8F08100BF003C014086
:10901000287D00202DE9F0410B4E346873691C4017
:109020000FD0DFF828800127B4FA84F3C3F11F03BF
:1090300007FA03F558F8230003689847AC437561B5
:10904000F2D1BDE8F08100BF003C0140287D002046
:109050002DE9F0410B4E346873691C400FD0DFF8E6
:1090600028800127B4FA84F3C3F11F0307FA03F53C
:1090700058F8230003689847AC437561F2D1BDE806
:10908000F08100BF003C0140287D00202DE9F04127
:109090000B4E346873691C400FD0DFF8288001271D
:1090A000B4FA84F3C3F11F0307FA03F558F8230059
:1090B00003689847AC437561F2D1BDE8F08100BF09
:1090C000003C0140287D0020084A094808B5536C3F
:1090D00043F480435364002140222FF05EFF054B90
:1090E0004FF0FF321A60C3F8032008BD0038024079
:1090F000287D0020687D002003685B6A18472DE901
:10910000F041044618460D46164698462CF0DEFD02
:109110002768E6722844A07229467D694346324694
:109120002046AC46BDE8F0416047036810B50446F0
:109130001B689847236820469B689847A37B0133A8
:10914000A37310BD10B5036804469B689847FF23BE
:1091500001226373227310BD08B504F0A7FE38B175
:109160002C2282710022C2712021BDE8084066E4F1
:1091700008BD10B5044682B04068FFF717FD2068AF
:1091800041F08001FEF749FF0DF10701206820F052
:1091900093FE6068FFF70FFD9DF8070002B010BD59
:1091A000F8B5654C0601A7190546387A20F03EFF50
:1091B0003B7A03F01F015B090122032B02FA01F243
:1091C0006DD0042B66D0022B5CD0A3190135187921
:1091D00004F06CFEEDB2074610B11223C571837125
:1091E000A319587904F062FE10B11323C57183717D
:1091F000A319987904F05AFE10B11423C571837134
:10920000A5190A21EA79384604F084FD687904F04A
:109210004DFEEA790A2104F07DFDA87904F046FEAE
:10922000EA790A2104F076FDA359444A934247D0D3
:10923000434A934250D0434A934259D0424A9342C0
:1092400062D0424A93426BD0414A93422CD034447C
:10925000227BE2B901200222198801F4415141F434
:1092600045710A4302431A809A8B22F40062120469
:10927000120C07219A8319821A8892B242F0400296
:109280001A80F8BD334B596A0A435A629DE70020A1
:109290000246E1E72F4B19690A431A6195E72D4B06
:1092A000196A0A431A6290E702F564424FF400100B
:1092B000536A43F40013536214F0ABF9A359C6E7A1
:1092C00002F584324FF48050536A43F48053536262
:1092D00014F09FF9A359BAE702F500324FF4804029
:1092E000136A43F48043136214F09CF9A359AEE768
:1092F00002F5FE324FF40040136A43F40043136258
:1093000014F090F9A359A2E702F582324FF400500D
:10931000536A43F40053536214F07BF9A35996E760
:1093200002F568424FF48010536A43F4801353628D
:1093300014F06FF9A3598AE7707B002000300140D8
:1093400000380040003C0040003401400050014023
:109350000054014000380240427A02B9704710B50B
:1093600004460368406804F10A01984700236372C9
:1093700010BD437A5A1C0344D2B242729972037AE6
:10938000934200D802B9704710B50446036840689C
:1093900004F10A0198470023637210BD302827D0DA
:1093A000312827D0322827D0332827D0342827D077
:1093B000352827D0202827D0212827D0102827D0AB
:1093C000112827D0122827D0132827D0142827D0D7
:1093D000152827D0162805D0172808BF0F2202D03D
:1093E000002070470E22104B03EB42035878704761
:1093F0000022F8E70122F6E70222F4E70322F2E76F
:109400000422F0E70522EEE70622ECE70722EAE76E
:109410000822E8E70922E6E70A22E4E70B22E2E76E
:109420000C22E0E70D22DEE70491030870B54488C2
:1094300006460D46C4F30B042246002128462FF0B1
:10944000ACFD3369094A934209D3094A934206D2D3
:10945000224628461946BDE870402DF01FBB23B1B7
:1094600021462846BDE87040184770BD98050008A1
:109470004A060008064B07498B4202D300231846D0
:1094800070471A88C2F30B029042F8D01433F3E706
:109490008801000898050008024A136823EA0000C2
:1094A00010607047C8530020F8B51A4D2B789F2BD9
:1094B0002ED16B78BE2B2BD105221749A81C2FF07B
:1094C000B7FD28BB072229464FF6FF70FEF793FF32
:1094D000124FEC1D22884AB1A618BE4218D2052AA6
:1094E00016D92146FEF787FF3446F3E721460222CC
:1094F000FEF781FF0222A118FEF77DFF0634084B1C
:10950000641B1C8041F60F53C31A58425841F8BDE2
:109510000020F8BD004000088CBA03080080000855
:10952000AC2600202DE9F04FDFF85891504F8DB058
:109530000326A7EB090718220DEB020000212FF0EC
:109540002CFD4C4BCDF8189007971A69002A04DAC5
:10955000494A5A6002F188325A6001228DF82C2063
:10956000F322DA60454B464C18689A8804909B7940
:10957000ADF8142004A9072206A88DF81630FFF7CD
:10958000B7F9072204A94FF6FF70FEF734FFDFF8A2
:10959000F8B080464FF0000A5C4539D30CAC00258A
:1095A00024F82C5D0222214606A8FFF7A1F9022229
:1095B00021464046FEF71FFF40BAC043ADF8080001
:1095C000022202A906A8FFF793F9099878B108AB1F
:1095D000C0F10402294618442FF0DFFC0A9818B99C
:1095E000089906A8FFF7E6F800230A9009939DF86A
:1095F0002C300A9A23B11F490B6943F000430B61D9
:10960000013E2DD0002A96D1FFF74EFF50B32CE03B
:1096100065888DF80DA0C5F30B05AA1DADF80820CF
:109620002288C2F30B01120BADF80A108DF80C2042
:1096300002A9062206A8FFF75BF9062202A9404606
:10964000FEF7D9FE616880462A4606A8FFF750F962
:10965000616840462A46FEF7CEFE143480469BE7FA
:10966000002AD1D0052004F04FFE0DB0BDE8F08FE8
:1096700000800008003C0240230167452491030854
:109680008801000800400008980500080378202B96
:10969000024600F10100F9D0092BF7D02D2B2CD078
:1096A0002B2B03BF5378B7EE000A0246B7EE000A31
:1096B000A3F13001C8B209289FED467A10D8F2EE26
:1096C000046A07EE901AF8EEE77A12F8013FE7EE27
:1096D000267AA3F13001C8B20928B0EE677AF0D932
:1096E0002E2B4CD003F0DF03452B0BD0F7EE007A86
:1096F00067EE276A20EE260A70475378BFEE000A0D
:109700000246D5E710B451782D2959D02B290ABF2C
:109710009178501C901C0024A1F13003092B53D8E0
:10972000002303EB830301EB430310F8011FA1F1B6
:109730003002092AA3F13003F3D9B3F59A7F28BF89
:109740004FF49A73072B42D9DFED236A1A46F7EEDE
:10975000007A083A072A67EEA67AFAD803F00703D8
:109760002BB1F2EE046A013B67EEA67AFBD124B37B
:10977000C7EE276A5DF8044B20EE260A704753783F
:10978000A3F13001C8B2092802F10102AAD8F2EE11
:10979000046AF0EE665A07EE901AF8EEE77A12F8CD
:1097A000013F87EEA66AA3F13001C8B2092866EE30
:1097B000A56A37EE067AEED994E767EE276AD9E70D
:1097C000901C91780124A7E7F7EE007ACFE7F7EE37
:1097D000007AC5E70000000020BCBE4CB5EEC00A10
:1097E000DFED317AF1EE10FACCBF30EE270A30EE21
:1097F000670ADFED2E7A20EE270A30B5FDEEC07A3B
:1098000087B017EE904A054684EAE470002303A966
:10981000A0EBE47001930093029317F0D9FE002CA3
:10982000ACBF20232D2303A88DF800302CF04EFA76
:10983000012803A924D002282DD0032805BF3023F6
:10984000684668468DF801302FF0CDFB68462CF055
:109850003DFA0338C4B22246694628462FF021FC5F
:1098600000232B5528462CF031FA2E22431C2A5473
:109870000DEB0401E8182FF0D3FB284607B030BDEC
:10988000302368468DF801308DF802308DF80330B2
:109890002FF0A9FBDAE7302368468DF801308DF808
:1098A00002302FF0A0FBD1E76F12033A00007A4498
:1098B0002DE9F041064615460846B6FBF2F43CB9E0
:1098C00005FB1464124B1B5D00F8013BBDE8F08101
:1098D000B4FBF2F767B90E4B05FB174705FB1464A1
:1098E000DA5D00F8012B1B5D00F8013BBDE8F0815B
:1098F000B7FBF2F8B8F1000F02D04046FFF7D8FFEF
:1099000005FB1878024B13F8082000F8012BE3E759
:1099100094BA030830B402681146531C036011F86E
:10992000024B0160D31C517803609378151D0560CC
:109930001B0443EA0123D078234343EA006030BC90
:1099400070470368591C1A46016012F8021B026036
:10995000587841EA0020704738B50446006815463B
:109960002DF09CF822682A44226038BD036810B4A8
:109970000A0E5C1C04601A7003680A0C5C1C04600C
:109980001A7003680A0A5C1C04601A7003685A1C87
:10999000026019705DF8044B7047036810B40A0A3E
:1099A0005C1C04601A7003685A1C026019705DF830
:1099B000044B704703685A1C026010B419700368A6
:1099C0000A0A5C1C04601A7003680A0C5C1C0460C0
:1099D0001A700368090E5A1C026019705DF8044B76
:1099E000704703685A1C026019700368090A5A1C00
:1099F0000260197070472DE9F047002488B0804656
:109A00000F461E46A14605AD531C0393117839B38A
:109A1000252933D1931CCDF810900393507830282A
:109A20004ED04FF0000AA0F13003DBB2092B42D92F
:109A30006C2819D0642800F0938024D825281CD0E5
:109A400063D9582876D063281BD131784046B8476F
:109A5000039A531C03931178043601340029D7D19B
:109A6000204608B0BDE8F087039B5A1C03921B7880
:109A7000642B7CD02AD8252B54D125214046013493
:109A8000B847039AC0E7732833D044D975284FD11B
:109A900006F1040E30682B4600220A217646FEF7B6
:109AA0002FFC049A0095534639464046FEF765FC64
:109AB000039A0444A8E704AA03A917F065FDB7E7D1
:109AC000D31C039390784FF0010AACE7732B10D0AE
:109AD0005BD9752B3AD0782B96D1A3F15802B2FA04
:109AE00082F2306852092B4610210436FEF708FC3A
:109AF000D7E73368049A0093394600234046FEF7BF
:109B00003CFC04360444039A7EE70028B9D1204681
:109B100008B0BDE8F0876E28B3D1039A33680436E5
:109B20001C6071E72AD9582BD7D0632B8DD06BE7F7
:109B30007828A6D1A0F15802B2FA82F23068520910
:109B40002B461021FEF7DCFB0436AAE706F1040ED3
:109B500030682B4600220A217646FEF7D1FBA0E7AB
:109B6000331D306829461E46FEF79CFB99E7331DDE
:109B7000306829461E46FEF795FB92E7002B7FF4DE
:109B800043AF204608B0BDE8F0876E2BC6D03BE758
:109B90000EB400B584B005AB019053F8042B064910
:109BA000039301A8FFF727FF019B00221A7004B05E
:109BB0005DF804EB03B07047718300080FB430B553
:109BC00083B006AB0A490B4853F8042B09680068B8
:109BD0000193FFF710FF084C0546206805F0F6F8E2
:109BE0000028FAD0284603B0BDE8304004B07047E2
:109BF000F43B0020F83B002098A40020DFED2B7AF6
:109C0000B4EEE70AF1EE10FA4ADDDFED296A9FEDC6
:109C1000297A01E0B0EE670AB4EEC70AF1EE10FA55
:109C200070EE667AF6DC9FED247AF4EEC77AF1EEF8
:109C300010FA38D5DFED1E6A9FED207A01E0F0EED4
:109C4000407AF4EEC77AF1EE10FA37EEA60AF6D4AF
:109C5000DFED1B7AB4EEE70AF1EE10FA14DDDFED6A
:109C6000137A37EEC00A60EE006A9FED166A9FED28
:109C7000167ADFED167AA6EE867A20EE266AE6EEF2
:109C8000877AA6EE270A7047DFED117AB4EEE70A6D
:109C9000F1EE10FA44BFDFED087A37EEC00AE2E7D2
:109CA000F0EE407ABFE7B0EE670AD1E7DB0F49403C
:109CB000DB0FC940E4CB1641DB0F49C0E4CB16C132
:109CC000DB0FC93F92E741B99730083C15A82ABE7F
:109CD000DB0FC9BF41404A0011F0800F82F0D5036D
:109CE000D2B2DBB208BF1346590013F0800F81F0E7
:109CF000D502C9B2D2B208BF0A46510012F0800F95
:109D000081F0D503C9B2DBB208BF0B46590013F08E
:109D1000800F81F0D502C9B2D2B208BF0A46510005
:109D200012F0800F81F0D503C9B2DBB208BF0B4639
:109D3000590013F0800F81F0D502C9B2D2B208BF2A
:109D40000A46510012F0800F81F0D503C9B2DBB290
:109D500008BF0B465A0082F0D50013F0800FD2B234
:109D6000C0B208BF1046704709B909E0194690FB18
:109D7000F1F301FB13030846002BF7D108467047A7
:109D80000146FBE7F0EEC07AB0EEE07AB4EEE77A97
:109D9000F1EE10FAB4BFB0EE676AB0EE476AB5EE06
:109DA000406AF1EE10FA46D0B4EEE77AF1EE10FA1E
:109DB0008CBFF0EE675AF0EE475AC5EE866A9FED0B
:109DC0001F3A9FED1F6A9FED1F4A9FED1F5ADFED5F
:109DD0001F3ADFED1F4ADFED1F5AA6EEC36AE6EE1B
:109DE000A34AA6EE864AB7EE006AA6EE845AA6EE0D
:109DF000A46AE6EE855AC5EE866AB4EEE77AF1EE1D
:109E000010FA48BFDFED147AF5EEC00A48BF77EECE
:109E1000E66AF1EE10FA48BFDFED107AB5EEC00A3F
:109E200048BF77EEE66AF1EE10FA48BFF1EE666AD7
:109E3000B0EE660A7047DFED076ADEE739094E3D8E
:109E4000E3B59E3E88FA163E45FE7F3F99FB243FD0
:109E500069A2163EA7DFA834DB0FC93FDB0F4940DC
:109E6000DFED317A30EE277AFDEEC76A16EE903AD2
:109E70002033402B02D99FED2D0A7047B4EEE70A3C
:109E8000F1EE10FA4DDD9FED2A6ADFED2A6A01E05E
:109E9000B0EE677AB4EEE67AF1EE10FA77EE467A33
:109EA000F6DC9FED257AF4EEC77AF1EE10FA35D59F
:109EB000DFED1F6A9FED217A01E0F0EE407AF4EECB
:109EC000C77AF1EE10FA37EEA60AF6D4DFED167A6D
:109ED000B4EEE70AF1EE10FA1BDCDFED197AB4EE0E
:109EE000E70AF1EE10FA44BFDFED137A37EEC00A4D
:109EF00060EE006A9FED136A9FED137ADFED137A2F
:109F0000A6EE867A20EE266AE6EE877AA6EE270A85
:109F10007047DFED0F7A37EEC00AE9E7B0EE670A67
:109F2000D4E7F0EE477ABCE7DB0FC93F0000000042
:109F3000DB0FC940E4CB1641DB0F49C0E4CB16C1AF
:109F4000DB0FC9BF92E741B99730083C15A82ABE7C
:109F5000DB0F4940FDEEC07A17EE903A2033402BDC
:109F600051D8DFED2D7AB4EEE70AF1EE10FA50DDAC
:109F7000DFED2A6A9FED2A7A01E0B0EE670AB4EEBF
:109F8000C70AF1EE10FA70EE667AF6DC9FED257ADC
:109F9000F4EEC77AF1EE10FA38D5DFED206A9FEDC6
:109FA000227A01E0F0EE407AF4EEC77AF1EE10FA90
:109FB00037EEA60AF6D4DFED1D7AB4EEE70AF1EE2D
:109FC00010FA1BDCDFED1A7AB4EEE70AF1EE10FAB4
:109FD00044BFDFED147A37EEC00A60EE006A9FEDF1
:109FE000156A9FED157ADFED157AA6EE867A20EEDA
:109FF000266AE6EE877AA6EE270A7047DFED067A34
:10A0000037EEC00AE9E79FED0E0A7047B0EE670A27
:10A01000D1E7F0EE407AB9E7DB0F4940DB0FC940EA
:10A02000E4CB1641DB0F49C0E4CB16C1DB0FC93FBF
:10A03000DB0FC9BF92E741B99730083C15A82ABE8B
:10A040000000000010B507EE901A2DED028BB8EE5F
:10A05000678ADFED227A28EE008A044628EE278AF6
:10A06000B0EE480A2CF0DAFEF0EE408AB0EE480A74
:10A070002CF036FEF7EE007A9FED197AF0EE675A73
:10A08000E8EE875A0023A361B0EE676AC7EEA56ABF
:10A0900063612362E361A3626362A8EEC76ABDECF9
:10A0A000028B77EEC07AB6EE007AF8EE005A27EE11
:10A0B000877A20EE250A27EE267A26EE266A67EEB4
:10A0C000A67A20EE260A84ED046AC4ED017A84EDB6
:10A0D000007A84ED027A84ED030A10BD27D4D236CB
:10A0E000F304353F10B44C09012250F8243001F03C
:10A0F0001F0102FA01F10B4340F824305DF8044BD4
:10A1000070474B0901F01F0150F82320012303FA87
:10A1100001F1114214BF184600207047074A084B4E
:10A1200010781B78074A834296BFC31AC3F1800395
:10A130000020126818441044704700BF287B00209C
:10A14000A57A002068810020064A074B10781B780A
:10A1500083428ABFC3F18003C01AC018C0F17F00D8
:10A16000704700BF287B0020A57A002010B582B080
:10A1700000249F2332208DF804308DF805408DF89F
:10A1800006408DF8074004F0B5FB8DF8014000BF94
:10A19000334C2068FEF70AFD01A9042268461FF02F
:10A1A000C5FE2068FEF707FD00BF9DF802309DF850
:10A1B00001009DF803102B4A1B0243EA00430B43A6
:10A1C000934246D01ADD284A93423AD02FDD274ADF
:10A1D00093422FD00132934222D1254B4FF480720B
:10A1E0001A805A809A881988224C120202FB01F1C7
:10A1F00001209A60D960607002B010BD1E4A93427F
:10A2000018D001329342E8D0A2F51A42033A9342A1
:10A2100006D1174B20214FF4807219805A80E1E754
:10A22000134B0020188058809860D860E4E7023A09
:10A230009342F5D10E4B80214FF4807219805A80E1
:10A24000D0E70B4B4FF400714FF4807219805A80A5
:10A25000C8E7074B40214FF4807219805A80C1E74C
:10A26000443C00201620C2001920C2001740EF0015
:10A270003C080020801D002017BA200030B5124C89
:10A28000637883B01BB90120637003B030BD052231
:10A2900000238DF800208DF8013000BF0B4D286899
:10A2A000FEF784FC6946022201A81FF03FFE2868E1
:10A2B000FEF781FC00BF9DF8053003F0010383F039
:10A2C0000100637003B030BD801D0020443C0020BD
:10A2D00070B5064C0646256803E023685B1BB34255
:10A2E00003D8FFF7CBFF0028F7D070BDEC7D00202E
:10A2F0002DE9F04F89B0B2F100080190039102936B
:10A3000040F39F800B46002201EB880153F8040BB9
:10A310008B420244FAD1029B0592002B00F0898007
:10A32000059B002B5ED04B4BDDF814B01B685FFA29
:10A3300083FA0AEB0B02B2F5807F474AD2688CBFE2
:10A34000CAF5807ADA469A425ED9190C1A0A4FF099
:10A35000020406208DF81F308DF81E208DF81D1088
:10A360008DF81C40FFF7B4FF0620FEF729FC3B4A9E
:10A370000123537000BF3A4B1868FEF717FC07A97A
:10A38000042200201FF0D2FD0024039D019E5746A9
:10A39000A1462968A30000200A46013459B1B942F8
:10A3A00024D231681FF0C2FD2A6833681344336039
:10A3B000BF1AC5F80090A04505F1040506F1040692
:10A3C000E7D1274B1868FEF7F6FB00BF214B214A67
:10A3D0001B6853441360029AABEB0A0B0AB3BBF140
:10A3E000000FA4D1059809B0BDE8F08F019C04933B
:10A3F0003A46E1581FF09AFD049B2A68E158394417
:10A40000D71BE1502F60DCE705981649164AA0EBF0
:10A410000B000590059800230B70137009B0BDE880
:10A42000F08F059BA3EB0B030593059809B0BDE8DE
:10A43000F08FFFF723FF00287FF472AF029B059394
:10A44000D0E7029C1CB9FFF719FF0594CAE7002367
:10A450000593C7E7688100203C080020801D00208C
:10A46000443C0020287B0020A57A002070B5104DC8
:10A47000104E2B7831788B4284B016D00E4A03925E
:10A480001A4402928CBF0C46CA1A04A98CBFC3F1AD
:10A4900080020024012341F8102D02A80222019419
:10A4A000FFF726FF002333702B7004B070BD00BF90
:10A4B000A57A0020287B0020A87A002070B5194CCE
:10A4C000194D23782978994284B027D0174A0392EE
:10A4D0001A44029234BF0E46CA1A04A934BFC3F10B
:10A4E00080020026002341F8102D02A802220196C6
:10A4F000FFF7FEFE23781844C0B203062B7848BF4E
:10A5000080F080008342207002D0002004B070BD33
:10A51000002301202B70237004B070BD012004B013
:10A5200070BD00BFA57A0020287B0020A87A0020FB
:10A5300008B545F20820FFF7CBFE0620FEF740FBEA
:10A54000064B0122C7205A70FEF73AFB0448054922
:10A55000054A002303700B70136008BD801D0020A6
:10A56000287B0020A57A0020688100202DE9F04199
:10A5700082B00346060C050A032406208DF8073036
:10A58000884617468DF805608DF806508DF8044012
:10A59000FFF79EFE98B100BF0A4C2068FEF706FB4D
:10A5A00001A9042200201FF0C1FC3A4600214046C8
:10A5B0001FF0BCFC2068FEF7FEFA00BF384602B070
:10A5C000BDE8F081443C0020F0B5124BDD6885B059
:10A5D0000DB905B0F0BDED0A14D0002704AE7C190A
:10A5E0006410E00210226946FFF7C0FF0F2809DD62
:10A5F0006B4653F8042B01320AD1B342F9D12546F8
:10A60000AF42ECDBFFF732FF034BED021D60E0E7EA
:10A61000671CF5E73C080020688100200C4B98423D
:10A6200013D0A3F5806398420FD003F5804398427E
:10A630000BD003F58063984207D003F580639842FE
:10A6400003D0044B186840087047024B18687047E5
:10A650000004014038940020F0B5774B774A87B06A
:10A660001968914200AF00F0DB800023744A3B6020
:10A670007B60136843F48033136003E03B68B3F5F9
:10A68000A04F09D0136803F400337B603B680133AB
:10A690003B607B68002BF1D0694B1B6813F40033DF
:10A6A00018BF01237B607B68012B7BD0654D644B19
:10A6B000654AEA606549586F654A0860AA605E6B42
:10A6C000644C654A654826F080065E635E6F46F01E
:10A6D00080765E67196B0C431C63596B5963996BE9
:10A6E0009963196C41F05B5141F47B1141F41F6196
:10A6F00041F00F011964596C07F118040A4348F23C
:10A70000FF715A6444F8101D002621460123FB7393
:10A710003E737E73BE7312F031FF21464FF6FF7316
:10A720004F48BB6012F02AFF4FF6FF7321464D4899
:10A73000BB6012F023FF21464B4812F01FFF214659
:10A740004A4812F01BFF2146494812F017FF2146E4
:10A75000484812F013FF2146474812F00FFF2146E8
:10A76000464812F00BFF204612F064FF444B454C64
:10A770001B68BA6844484549A4FB03439B09A0FBF6
:10A780000202013B920CB3F1807F0A6007D2404A7B
:10A79000F0200721536085F82300966011601C3774
:10A7A000BD46F0BD264B3B4D1A6C3B4842F08052F3
:10A7B0001A642C684268816844F440442C609C68A8
:10A7C0009C609C6844F400449C609C6844F4A054E1
:10A7D0009C600068120642EA801242F48002490836
:10A7E00042F00802013942EA01425A601A6842F016
:10A7F00080721A601A689201FCD52849104A40F20A
:10A8000005700860996821F003019960996841F02A
:10A8100002019960936803F00C03082BFAD145E715
:10A8200000221A6062B61E4B1B6883F308881D4B1A
:10A830001B689847FEE700BFFCFF0120EFBEADDEBE
:10A840000038024000ED00E00005FA05C445002094
:10A8500000000008FF916700335F0700000002401E
:10A860000004024000080240000C024000100240B8
:10A870000014024000180240001C02400020024068
:10A8800038940020D34D621083DE1B43F07D0020FE
:10A8900010E000E00070004000000020003C02409A
:10A8A0000000FF1F0400FF1F08B5054B1B6803B124
:10A8B0009847044B044A1A6072B6FDF78BFE00BF3E
:10A8C000B88D0020FCFF0120EFBEADDE08B5034BC4
:10A8D0001B6803B1984772B6FDF77CFEB88D002067
:10A8E000084B10B507281B68C8BF143818440C461D
:10A8F000007D03F0DBFA20B12146BDE81040FEF7F1
:10A9000073B910BD947D002038B50D4B07281B6826
:10A91000CCBFA0F11404044623440546187D03F07F
:10A92000C5FA58B101342722C47182710121FEF7A2
:10A9300086F828460021BDE83840D1E738BD00BF81
:10A94000947D002070B50F4C0F4DC0EBC00004EBA0
:10A950008004286B26693043286382B09209667BA5
:10A96000A1600025012101A863618DF804608DF8C4
:10A9700005208DF806508DF807101FF0DDFB02B0A2
:10A9800070BD00BFFC15002000380240074BC0EB33
:10A99000C00030B403EB8000054C0569236B2B43EA
:10A9A00023630176427630BC704700BFFC1500205F
:10A9B000003802402DE9F04F5B4C54F8204083B042
:10A9C000002C00F0AC80E66D002E00F0AA809046CE
:10A9D000564A35692260994604F2622204F1620304
:10A9E0006361A2614FF400737268A1600746E3607F
:10A9F0002361A265A246B5B14D4B00205A6895422D
:10AA000003F11C0376D001301028F7D100207A1C06
:10AA1000D2B20C21FFF7BAFFA36DB168326922638D
:10AA20000433A1636365F068E8B1414B00215A68C3
:10AA3000904203F11C035BD001311029F7D10025AE
:10AA40007A1CD2B20B212846FFF7A0FF2346F27FE3
:10AA500038492846FFF776FFA36DB168F268626354
:10AA60000433E163236594F8610003F01FFA05469F
:10AA700094F8600003F01AFA8346307F00284BD127
:10AA800019F0080F38D118F0020F09D045B10B2288
:10AA90007B1CAA71EB712846727F222103F03AF9E0
:10AAA00018F0010F15D1A36B7BB996F82020B17F68
:10AAB0008DF8063001A8930901228DF805308DF834
:10AAC00004108DF807201FF037FB504603B0BDE897
:10AAD000F08FBBF1000FE6D001370C238BF8077025
:10AAE0008BF806305846727F222103F013F9DAE71B
:10AAF000CDB2A5E7C0B28AE70137FFB215B10B238B
:10AB0000EF71AB7119F0100F284614BF022112210A
:10AB1000727F03F0FFF8C6E71FF088FAB0E7A2469D
:10AB2000D3E7B246D1E700BF003C00202C910308D8
:10AB3000FC150020358900080348D0F8AC3113B16A
:10AB400000F5D27018477047FC1500200348D0F874
:10AB5000903113B100F5C47018477047FC15002000
:10AB60000348D0F8743113B100F5B6701847704738
:10AB7000FC1500200348D0F8583113B100F5A87037
:10AB800018477047FC1500200348D0F83C3113B13A
:10AB900000F59A7018477047FC1500200348D0F85C
:10ABA000203113B100F58C7018477047FC15002058
:10ABB0000348D0F804310BB1FC301847704700BF90
:10ABC000FC1500200348D0F8E8300BB1E0301847FE
:10ABD000704700BFFC1500200348D0F8CC300BB103
:10ABE000C4301847704700BFFC1500200348D0F858
:10ABF000B0300BB1A8301847704700BFFC150020DB
:10AC00000348D0F894300BB18C301847704700BF20
:10AC1000FC1500200248836F0BB170301847704755
:10AC2000FC1500200248C36D0BB154301847704723
:10AC3000FC1500200248036C0BB1383018477047F0
:10AC4000FC1500200248436A0BB11C3018477047BE
:10AC5000FC1500200248836803B11847704700BF05
:10AC6000FC1500201549164B16480A6810B48C686C
:10AC70001549B2FBF4F203FB02F30360D1F888201C
:10AC8000124B134C42F47002C1F888201A6800205D
:10AC900042F001021A6098601A6822F0847222F46D
:10ACA00080321A605C601A684FF0006422F48022DF
:10ACB0001A60D8608C605DF8044B7047000000207B
:10ACC00040420F003894002000ED00E000380240C0
:10ACD00010300024044B4FF4F0700A21022283E864
:10ACE0000700FFF7BFBF00BF000000202DE9F04FB5
:10ACF000A34CDFF8C09294F85C312DED028B8346B3
:10AD00008FB0002B40F05A8194F8DD31002B39D000
:10AD1000D4F8E0319B4AABEB0303934200F2348456
:10AD200094F84862002E00F0B780D4F850324BB34C
:10AD3000D4F8583240F6B732ABEB0303934221D933
:10AD400094F85432002B00F061858F4F013BDBB249
:10AD500084F85432002B00F06985D4F8505294F8EE
:10AD60005C2215F8011B94F85D323868C4F8505223
:10AD70000A44013384F85C2284F85D3204F03AF826
:10AD8000C4F858B294F85E32D9F8005043B17F4EFF
:10AD9000306828B194F85F32013B012B40F2F38414
:10ADA00094F8A03353B17A4E33683BB1D9F80070B0
:10ADB000D4F8A433FB1A632B00F22A8294F8DC3314
:10ADC000022B00F0D482734D95F87430032B00F001
:10ADD000488794F8F8336BB1D4F8FC3353B103F0DF
:10ADE000E3FCD4F8003444F61F62C31A93420746CA
:10ADF00000F2E88294F87A35002B40F08B8194F8C9
:10AE00008B3533B1D4F88C3503F5C333A0339B4570
:10AE100078D294F8C235BBB15F4D2E46D4F8C40544
:10AE200003F0E4FF80B1D4F8C40503F0D7FF94F831
:10AE3000C83507465A1E63B1D4F8C40584F8C8253E
:10AE400003F0D4FF0028EED10FB0BDEC028BBDE8BB
:10AE5000F08F0322514928462EF085F894F8CC351E
:10AE600094F8CD2584F8CF7583F47F4383F0FF03F6
:10AE70009B1ABFB29BB2B7EB132FCFD194F8CE255C
:10AE8000DBB29A42CAD1304628F088FE94F8C83521
:10AE9000184484F8C805C1E73B4F386803F0A6FFA3
:10AEA000C0B201280FD902283A4D40F0CE842B7849
:10AEB000002B41F0A087D4F84C32ABEB0303B3F581
:10AEC0007A6F81F09A85D4F85032002B3FF45AAF54
:10AED00094F84832002B7FF42BAF314B1B689B78E2
:10AEE00001211E3B00228B4284F8481284F85C2228
:10AEF00041F2D28738680221043028F074FF94F8B8
:10AF0000543223E794F89035264AC4F88CB502EB06
:10AF10008302526C42B3244F244E0EADFB1C45F805
:10AF2000203D07F1150300210793A523318084F804
:10AF300094358021152384F89635284684F8951594
:10AF4000904728463188FEF74CFD069DED1B152DD8
:10AF5000A8BF15252A46394607F118002BF09EFD9B
:10AF600094F8903584F8C155114A013382FB0312DD
:10AF7000A2EBE37202EB42029B1A84F8903548E799
:10AF80008C1D00203F0D03007C9500205095002073
:10AF9000749500201C000020582300205923002015
:10AFA0008095002054910308202300203A9500202A
:10AFB00056555555EC7D002000007A44D4F8603198
:10AFC000D9F80020D31A7C2B7FF69EAE94F864311A
:10AFD0001FED078AC4F86021013384F8643104F559
:10AFE000CE772425284628F075FFB4F87831F7ECA1
:10AFF000016A07EE103AF8EEE66AB8EEC77A013554
:10B00000C6EE877AEDB267EE887AFDEEE77ACDED8F
:10B01000007ABDF90060F0B228F032FFC6F30720D5
:10B0200028F02EFF272DDDD1302028F053FFD94EF8
:10B03000002028F025FF002028F022FF30685E2144
:10B0400003F0D8FE94F8643113F0030528D1D4F846
:10B05000602141F288339A4201F2C987142028F016
:10B0600039FFCD4AB4F9B031DD1782FB0323C5EBBC
:10B07000A3052DB2E8B228F003FFC5F3072028F09E
:10B08000FFFE1C2028F026FF002028F0F9FE0020FB
:10B0900028F0F6FE5E21306803F0ACFE94F86431CF
:10B0A00013F0070501F02E85282B7FF42DAE002527
:10B0B0001720D9F8008084F8645128F00BFF284647
:10B0C00028F0DEFEB54BB64FA3FB08239B0BA7FB76
:10B0D00003125209C2EB0212A3EB8203D8B228F08A
:10B0E000CFFE182028F0F6FEAE4BA3FB08239B09E9
:10B0F000A7FB03125209C2EB0212A3EB8203D8B2E0
:10B1000028F0BEFE284628F0BBFE30685E2103F022
:10B1100071FEF9E5A44D2A7832B1A449D4F87C0532
:10B1200003F030FE00232B70D4F8803503F5C333D1
:10B13000A0339B45FFF463AE94F88935C4F880B51D
:10B14000234493F88455E80701F10B86A90701F120
:10B15000CD856A0701F191852A074DD5944B079358
:10B160000EAA1046A3F1210240F8202DA3F12402DB
:10B1700006460090002003F8240C11250223557088
:10B180009370D4F8C8113046FEF7F0FB3046D4F87F
:10B19000CC11FEF7EBFBB4F8D6317F4903EBC303C8
:10B1A0009B00053381FB0321DB17C3EBA10189B2AF
:10B1B0003046FEF7F2FBB4F8D83103EB83035900B5
:10B1C00089B23046FEF7E9FB94F8C231009D9B0737
:10B1D00043BFB4F8D01101F57A7189B24FF47A7196
:10B1E0002846FEF7DAFB069B94F8C421591C069109
:10B1F00028461A7028F0D7FE94F8893594F88A15F5
:10B20000013393FBF1F201FB123384F88935F6E543
:10B21000412028F099FD604DB4F9AE31DFF8A081EE
:10B2200085FB0320DB17C3EBA00080B228F070FD84
:10B23000B4F9AC3185FB0320DB17C3EBA00080B26F
:10B2400028F066FDB4F9B03185FB0320DB17C3EBB2
:10B25000A00080B228F05CFD98F80010306803F080
:10B26000C9FD94F8A85315F0010200F0B585514BC3
:10B270001B689A0668D594F8C2319B0701F1B58323
:10B280000125472028F060FDD4F8C80128F00CFD06
:10B29000D4F8CC0128F008FD474AB4F8D63130681C
:10B2A000A2FB0323C3F3471A514603F0A3FDB4F8EE
:10B2B000D02198F80030642000FB02F08AEA0303F2
:10B2C00088F8003028F0F0FC94F8C431306845EA82
:10B2D0008305EDB2294603F08DFD98F80030306803
:10B2E0005D40294688F8005003F084FD94F8A85387
:10B2F00055BB4F2028F028FDD4F8D40328F0D4FC07
:10B30000D4F8D80328F0D0FC284628F0CDFC012141
:10B31000306803F06FFD94F8C25198F8003030683F
:10B3200005F00105294683F0010388F8003003F099
:10B3300061FD98F8003030685D40294688F800507B
:10B3400003F058FD94F8A8531C4AC4F8A4736B1C6E
:10B35000DBB2A2FB0312D20802EB8202A3EB420390
:10B3600084F8A83394F8DC33022B7FF42CAD03F07F
:10B370001BFAD4F8E06340F6B833861B9E4201F214
:10B380004E8294F8EC333A2B01F03A85002384F88E
:10B39000DC331EE5849500206766666673B2E74578
:10B3A00089888888D34D6210D0950020AC95002004
:10B3B000AC950020BC8D00201F85EB51CDCCCCCCB2
:10B3C0007895002094F80634002B40F0CB846A4B2B
:10B3D0001B6848F6034113F0080F49F607464FF083
:10B3E000190208BF0E46580784F8062403D546F410
:10B3F000005646F00806990648BF46F4804694F881
:10B40000B85148BF46F02006C6F30908002D41F0A8
:10B410001B8394F8B931002B41F024861D4664202B
:10B420004FF0FF3A4FF0000C06960796ADF8265005
:10B43000CDF82080ADF828A08DF83600ADF824C0F6
:10B44000ADF82AC0ADF82CC0ADF82EC0ADF830C0B4
:10B45000ADF832C0ADF834C00DF1180EBEE80F00E3
:10B46000464E35460FC59EE80F0007C525F8023B3E
:10B47000180C0121FE221F23287084F8531084F831
:10B480004E2084F84F3094F8162484F851C0511897
:10B49000C82084F8161484F85020311F84F8520014
:10B4A0004FF6FF7501E011F8013B6B4083EA03138F
:10B4B000DBB21A0982EA152242EA03228E4282EAAC
:10B4C000C305F0D12D49A4F84C5001F11F0011F82B
:10B4D000013B6B4083EA0313DBB21A0982EA1522AF
:10B4E00082EA032282EAC3031BB29DB28142A4F81E
:10B4F0004C50ECD183F07C0383EA0313DBB21A09CE
:10B5000082EA152282EA032282EAC3031BB29AB2BC
:10B510004FEA122C5FFA83FE194EA4F84C2084F8EF
:10B5200074C084F873E004F14E0804F16E0AD8F890
:10B530000000D8F80410D8F80820D8F80C303546A8
:10B540000FC508F11008D0452E46F0D1D8F80000FC
:10B5500028600C4D98F80430337105F1270684F803
:10B5600065E484F866C415F8011FD4F8FC0303F001
:10B5700041FCAE42F7D1F8E3BC8D0020E01D002075
:10B58000CC210020CB210020D94ADA4BD07AD9F83F
:10B590000010D4F810221B88891A4FF47A7202FB2B
:10B5A00000F2DDB200201B0A914284F8025284F8B6
:10B5B000F85184F8033284F8F93184F8E60184F80C
:10B5C000E80181F0F480CC4BCC491A689B6894F870
:10B5D000C20181FB026581FB0361D217DB17C2EB5D
:10B5E000A502C3EBA10315121912F42684F8002258
:10B5F000012284F8015284F80432302584F80512BF
:10B6000084F8FE617521782384F8FF21860794F879
:10B61000C42184F8065284F8071284F8083284F8AA
:10B62000322241F1BF80D4F8C851B549D4F8CCC119
:10B63000B448B54BDFF8E8A281FB0567EE1781FB44
:10B640000CE1C6EBA7564FEAEC77C7EBA15100FB24
:10B65000065707EB47077F0000FB01C083FB07E8A5
:10B6600000EB400040004FEAA848052A4FEAD57594
:10B670004FEAE77201EB810183FB00E301EB8101FB
:10B6800006EB860684F82152A8EB02054FEAA34E8A
:10B6900000912A464FEAE0716DB206EB860605EB93
:10B6A0008606B4F8D631AEEB010529464FEADC7CBC
:10B6B0000AFB127203EBC303944FDFF868E284F8CD
:10B6C00026C24FFA81FC00990AFB15054FEA830355
:10B6D000B4F8D0010CEB81018EFB03CE87FB028C0A
:10B6E0004FEAE27287FB0587C2EB6C12B6B289B2F1
:10B6F0004FEAE373B4F844C284F8226200F5FA70AA
:10B700004FEAE5754FEA112AC3EBAE1EC5EB67158C
:10B710004FEA162380B24FEA222884F828A284F840
:10B7200023324FEA252784F82712CEF307264FEA63
:10B73000102184F8242234BF4FF0320A4FF0330A2C
:10B740004FEA1C22B4F8463284F8258284F8295244
:10B7500084F82A7284F81FE284F8206284F82D02AB
:10B7600084F82E1284F833A284F82BC284F82C2299
:10B7700084F8343294F84862C4F8E0B1002E7FF4C3
:10B78000D4AAFFF789BB624F4FF0010A4FF00008BF
:10B7900008E01B2B00F07B820D2B00F0878187F8DF
:10B7A00001A0306803F022FB00285BD0306803F072
:10B7B00015FB83B27E2BD9F800204CD07A78002A72
:10B7C000EFD194F860120029E3D07D2B00F046827F
:10B7D00094F864E2BEF1000F04D080F02003DBB2E5
:10B7E00084F864224A1CD2B2092A635484F8602285
:10B7F00000F02A82082AD4D8B4F86222134403EB5A
:10B80000132303F0FF03A4F86232CAE7C4F85032EE
:10B8100084F8483228F01AFB94F854323D4F013B2B
:10B82000DBB284F85432002B7FF497AA94F85C12B0
:10B8300094F85D3238684A1C013384F85C2284F83D
:10B840005D3203F0D7FAFFF79BBA28F0EFFA012335
:10B850002B70FFF738BB84F8608284F8618287F828
:10B8600001809EE794F865322BB1637884F8650215
:10B87000302B01F0398394F86122274B274FDFF8F2
:10B88000A8E0DFF86CC00126002A3FF489AAD9F8A5
:10B890000000401B012825D894F87883B8F1000FE8
:10B8A00040F0068294F890A303EB4A000089002838
:10B8B0003CD184F8906338688106E5D594F8C201DC
:10B8C0008007E1D5B4F8D62110494FF4F36303FBA8
:10B8D00002F381FB0321DB17C3EB61114FF403601B
:10B8E00028F067FA002384F86132FFF759BA00BFE5
:10B8F0002C9500203C9500204095002067666666E8
:10B900006BCA5F6B806967FF83DE1B431F85EB514A
:10B910001C0000207C95002054910308BC8D002061
:10B9200040420F00D34D6210C84500200AF1010AC1
:10B930005FFA8AFAB0F5E06F84F890A300F099807E
:10B940001AD8B0F5047F00F0318136D8B0F5887F81
:10B9500000F00981B0F5007F00F0EF80B0F5807F46
:10B9600092D1396849078FD5002128F022FA0023A7
:10B9700084F86132FFF714BAB0F5026F00F001816C
:10B980006CD8B0F5E46F00F08380B0F5006F00F084
:10B990009380B0F5E26F7FF477AFD4F8A021B4F8CC
:10B9A0007811642303FB02F393FBF1F128F001FA11
:10B9B000002384F86132FFF7F3B9B0F5826F00F02D
:10B9C0002481B0F5C06F00F01081B0F5806F7FF476
:10B9D0005BAF94F891330133DBB2032B00F2628149
:10B9E00042F2107184F8913301FB03F1B4F8923301
:10B9F000002B40F055810131D24B1B78DF07B4F8A2
:10BA0000943348BF0431DD0748BF0A31980748BF67
:10BA100014311A0648BF2831DF0548BF28315D07B9
:10BA200048BF6431180748BFC8319A0548BF01F5BF
:10BA3000C8719F0648BF01F57A71DD0648BF01F560
:10BA4000FA61580648BF01F57A614FF4806028F02A
:10BA5000B0F9002384F86132FFF7A2B9B0F5046FA2
:10BA600019D0B0F5116F4DD0B0F5036F7FF40CAF66
:10BA700021E7D4F89C21B4F87811642303FB02F386
:10BA800093FBF1F128F095F984F86182FFF788B90A
:10BA9000D4F8A421EFE7B4F9B01101EB810149001A
:10BAA00028F087F984F86182FFF77AB984F860A2F8
:10BAB0002370A4F8621274E6386881067FF5E4AE5C
:10BAC00094F8C20180077FF5DFAE1AF0010F40F055
:10BAD0007887D4F8C8219C4982EAE273A3EBE27329
:10BAE00003EB5303A1FB0331C908002AB8BF41F09F
:10BAF00080414FF4006028F05CF9002384F8613243
:10BB0000FFF74EB994F8B80100283FF4BDAE8F4955
:10BB1000087800283FF4B8AE8D4B1B8803EB8303F5
:10BB2000590080464FF4116091FBF8F128F041F97B
:10BB3000002384F86132FFF733B994F8B901002883
:10BB40003FF4A2AE834B84491B6881FB0321DB17C2
:10BB5000C3EBA1014FF4007028F02BF9002384F807
:10BB60006132FFF71DB9386841077FF58DAE0021BE
:10BB70004FF4887028F01DF9002384F86132FFF734
:10BB80000FB9396889067FF57FAE94F8C2A11AF023
:10BB9000020F3FF479AEB4F8D031642101FB03F118
:10BBA00028F007F984F86182FFF7FAB894F8B80131
:10BBB00000283FF469AE6549087800283FF464AE78
:10BBC000664B5B7B002B01F04982614B198891FB2E
:10BBD000F0F101EB810149004FF4047028F0E9F81D
:10BBE000002384F86132FFF7DBB894F8B90100282C
:10BBF0003FF44AAE574B4FF4C060996828F0D9F82B
:10BC0000002384F86132FFF7CBB83868810640F131
:10BC1000F18594F8C22194F8C41112F0020F0CBF00
:10BC200000234FF47A7312F0010F0CBF00224FF47F
:10BC3000FA62134419444FF4826028F0BAF80023E2
:10BC400084F86132FFF7ACB8B4F86222C2F1FF02A7
:10BC500093427FF4A4AD84F865A2A0E584F864A2C1
:10BC60009FE5D4F8F40303685B69984700283FF424
:10BC7000B0A8D4F8F403036801219B699847022215
:10BC8000002385F8742084F8DC33FFF7A2B830680D
:10BC900003F0ACF800287FF482AD84F861A280E55F
:10BCA0000231A9E6012384F8913342F210719DE636
:10BCB000D4F868322A4E94F88E23B34201F0B08152
:10BCC000511C94F88F03D4F86C7284F88E1302F030
:10BCD0000F028DF818200DF11902F91A002941F30D
:10BCE000008306A900910DF11E0502E0002E40F32D
:10BCF000A0850133C4F8683213F8011C02F8011B57
:10BD0000AA42A7EB030680EA0100EFD384F88F0371
:10BD100001F0E182531CAB42107038BF002203D205
:10BD200003F8012BAB42FBD10099322028F026F812
:10BD30004FF00008002384F8788384F86132FFF71D
:10BD40002FB800BF6F3D00201F85EB516395002089
:10BD50003C95002040950020676666662C95002083
:10BD600004200020013B84F8063494F80734002BAB
:10BD700040F0958094F84815D9F800E00A2284F83C
:10BD80000724002900F059850129B4F854A541F28F
:10BD900021830229B4F8568501F06A810329B4F899
:10BDA00058C501F04283B4F85A250092042901F0E5
:10BDB00037830529B4F85C5501F02E830629B4F8C1
:10BDC0005E0501F026830729B4F8602500F03D8563
:10BDD000B4F8623500F039BDB4F89433D80513D403
:10BDE000D90601F1EF809D0601F14981580601F164
:10BDF0006F82190701F17B82DD0701F1D78213F011
:10BE0000020F0CBF04220C22B24994F8AF3391F810
:10BE100000A00AF0010A0BB14AF0020A5320009276
:10BE200027F092FFAC4B1B8803EB830303EB8303E8
:10BE3000980080B227F06CFF002027F069FFB4F86B
:10BE4000D033A6493068C3EBC3135B0081FB0321E9
:10BE50001944DD17C5EB6125EDB2294602F0CAFF92
:10BE600098F80030009A306842EA0A0A5D400021E2
:10BE700088F8005002F0BEFF5146306802F0BAFF69
:10BE800098F8003030688AEA0303DBB2194688F874
:10BE9000003002F0AFFF94F8A853FFF729BA013B36
:10BEA00084F8073494F80A34002B40F06E848C4BED
:10BEB0001B68192284F80A249A0640F11A8294F821
:10BEC000C2319B0700F1B885012602F06DFCB4F881
:10BED000D811B4F8D051D4F8C831069001EB8101E3
:10BEE000019349004FF47A70ADF83210D4F8CC21A8
:10BEF000B4F8D68194F8C4C101998DF8346000FB80
:10BF000005F04FF0000E06AB4FF6FF75ADF8308030
:10BF10008DF835C0CDF81CE00A9008910992ADF873
:10BF20002C50ADF82E5098460093B8E80F006D4E97
:10BF3000B446ACE80F0098E80F00ACE8070094F8AE
:10BF40001624ACF8003084F851E0A6F1040A02F19E
:10BF5000010E1820FE211E234FF0C80CD04684F895
:10BF6000502084F816E484F8530084F84E1084F8C6
:10BF70004F3084F852C001E018F8013B6B4083EA6F
:10BF80000313DBB21A0982EA152242EA032246456C
:10BF900082EAC305F0D1534AA4F84C5002F11E01C5
:10BFA00012F8013B6B4083EA0313DBB2180980EA05
:10BFB000152080EA032080EAC3031BB29DB28A42A7
:10BFC000A4F84C50ECD183F0180383EA0313DBB2DE
:10BFD0001A0982EA152585EA032282EAC3031BB205
:10BFE0009AB2DBB24FEA122E019384F87230DFF876
:10BFF00000C1A4F84C2004F16E0384F873E004F14E
:10C000004E060293F36830687168B26865460FC5E2
:10C01000029B10369E42AC46F4D13068CCF800004A
:10C02000314D9DF8043084F8643484F865E42E467C
:10C0300016F8011FD4F8FC0302F0DCFE2B4BB342D0
:10C04000F6D102F0B1FBB4F9B011DFF8A8E0B4F812
:10C05000D06106908EFB010EC9174FF47A7000FB79
:10C0600006F0D4F8C821D4F8CC31009E0990C1EB79
:10C07000AE014FF0000EADF82CE0ADF82EE0ADF8BB
:10C0800030E0ADF832100A90079208930FCE04F119
:10C09000540CACE80F0096E8070021231C268CE81E
:10C0A000070084F85330C8226FF0010384F851E090
:10C0B00084F84E3084F84F6084F8522094F8163497
:10C0C00084F850305A1C84F8162433464FF6FF7E0D
:10C0D000564613E06F3D00203C9500200308208069
:10C0E000BC8D0020E01D0020CB210020F12100208C
:10C0F000CC2100206766666616F8013B83EA0E03D2
:10C1000083EA0313DBB21A0982EA1E2242EA0322FF
:10C11000B04582EAC30EEFD1D248A4F84CE000F15A
:10C120001C0110F8013B83EA0E0383EA0313DBB220
:10C130001A0982EA1E2282EA032282EAC3031BB2A0
:10C140001FFA83FE8842A4F84CE0EAD183F068032A
:10C1500083EA0313DBB21A0982EA1E2282EA03226F
:10C1600082EAC3031BB29AB2DBB2110A019384F8CC
:10C170007030DFF800C3029104F16E03A4F84C2084
:10C1800084F8711004F14E080393D8F80C30D8F8F5
:10C190000000D8F80410D8F80820E646AEE80F00F2
:10C1A000039B08F110089845F446EED1B8F800302A
:10C1B000AEF800309DF8043084F862349DF8083001
:10C1C00084F86334A84618F8011FD4F8FC0302F081
:10C1D00011FEA54B4345F6D1D4F8D433D4F8D82377
:10C1E00006934FF0000E009BCDF820E0079293E8F5
:10C1F000070004F1540383E8070094F8162484F838
:10C2000051E0312002F1010EFE210C2384F8502070
:10C21000C82284F816E484F8530084F84E1084F899
:10C220004F3084F852204FF6FF7E01E01AF8013BB0
:10C2300083EA0E0383EA0313DBB21A0982EA1E22A1
:10C2400042EA0322564582EAC30EEFD18549A4F89B
:10C250004CE001F10C0011F8013B83EA0E0383EA84
:10C260000313DBB21A0982EA1E2282EA032282EA5F
:10C27000C3031BB21FFA83FE8142A4F84CE0EAD14B
:10C2800083F0270383EA0313DBB21A0982EA1E2E26
:10C290008EEA032E8EEAC30EA2460FFA8EFE1FFA16
:10C2A0008EF65AF84E0FDFF8CCC1A4F84C604FEA76
:10C2B00016285FFA8EFE84F860E084F86180DAF870
:10C2C0000410DAF80820DAF80C30BAF810A0ACE85C
:10C2D0000F0004F25346ACF800A084F8538484F8AD
:10C2E00052E415F8011FD4F8FC0302F083FDAE42BE
:10C2F000F7D194F80E64002E40F0BE80B4F9AC2162
:10C30000B4F9AE319FED596AD9F80010069106EEE6
:10C31000902AB4F9B021534D84F851605B4207EE86
:10C32000102A07EE903AF8EEE66AF8EEE77AB8EEF1
:10C33000C77A67EE867A66EE866A27EE067A00226C
:10C34000CDED087ACDED076A8DED097A0A920B9250
:10C350000C920DF1180EBEE80F002E460FC69EE897
:10C36000070094F816C486E807004FF00508FE2081
:10C37000C8214FF01E0E1C230CF1010284F84E0060
:10C3800084F8521084F80E8484F853E084F84F3017
:10C39000291F84F850C04FF6FF7084F8162401E07E
:10C3A00011F8013B434083EA0313DBB21A0982EA26
:10C3B000102242EA03228D4282EAC300F0D1294DC5
:10C3C000A4F84C0005F11C0115F8013B434083EA39
:10C3D0000313DBB21A0982EA102282EA032282EAFC
:10C3E000C3031BB298B28D42A4F84C00ECD183F089
:10C3F000270383EA0313DBB21A0982EA102282EAD6
:10C40000032282EAC3031BB29AB24FEA122C5FFAEC
:10C4100083FEDFF86080A4F84C2084F871C084F8B3
:10C4200070E004F14E0604F16E0930687168B2687C
:10C43000F36845460FC510364E45A846F5D10C4D5C
:10C440003388A8F8003005F1240684F862E484F803
:10C4500063C415F8011FD4F8FC0302F0CBFCAE4214
:10C46000F7D10CE0E01D0020EF21002088C3E43A62
:10C47000CB210020CC210020731E84F80E3494F8C8
:10C480000F340193002B40F08481D24B1B680522AE
:10C490009D0684F80F2400F18382DFEDCF7AB0EEA1
:10C4A000677AB4F95A35B4F9B011CC4DCC48CDED1A
:10C4B000077AB3F5FA6FA8BF4FF4FA63B3F57A7F42
:10C4C000B8BF4FF47A73A3F57A72642303FB02F3C7
:10C4D00085FB032580FB0120DB17CA170026C3EB71
:10C4E000A51306A9C2EBA0028DED087AADF82A309B
:10C4F000ADF82820069609960D4600910FCDDFF87D
:10C50000E4E22E6894F816C484F850C075460FC54E
:10C510004A212E60AEF1040800250CF10100FE2234
:10C52000142384F85310C82184F85150464684F8E7
:10C53000160484F84E2084F84F3084F852104FF6D9
:10C54000FF7501E016F8013B6B4083EA0313DBB291
:10C550001A0982EA152242EA0322B64582EAC30595
:10C56000F0D1A049A4F84C5001F1140011F8013B9E
:10C570006B4083EA0313DBB21A0982EA152282EACE
:10C58000032282EAC3031BB29DB28142A4F84C503D
:10C59000ECD183F0140383EA0313DBB21A0982EAB5
:10C5A000152282EA032282EAC30325461BB21FFA40
:10C5B00083FC55F84E0FDFF838E2A4F84CC0DBB22C
:10C5C0004FEA1C2A84F869A084F8683069680293ED
:10C5D000AA68EB68AEE80F00286969692B8BAEE8A2
:10C5E000030004F23F45AEF800309DF8083084F8AF
:10C5F0005BA4A94684F85A3404F25B4A19F8011F77
:10C60000D4F8FC0302F0F6FBCA45F7D1764A94F859
:10C6100078351278013BDBB212F0010214BFC02161
:10C620004021172B9BBF71481B184FF0000E93F849
:10C630002CE0B4F89433980706BF0120019041F034
:10C64000100113F4027F019818BF022013F0100F9D
:10C6500018BF062013F0200F0CBF034610230193D0
:10C66000002A40F0B2840322019B069303234FF07B
:10C67000000C8DF82030009B8DF81CE08DF81E100A
:10C680008DF81F208DF81DC093E80700DFF854E1F6
:10C6900084F853C0AEE8030094F816148EF8002016
:10C6A00001F1010A4FF0FE090923C82084F851C0A6
:10C6B00084F8501084F816A484F84E9084F84F3013
:10C6C00084F852004FF6FF7E01E018F8013B83EA40
:10C6D0000E0383EA0313DBB21A0982EA1E2242EA3E
:10C6E0000322464582EAC30EEFD13E49A4F84CE04E
:10C6F00001F1090011F8013B83EA0E0383EA0313F9
:10C70000DBB21A0982EA1E2282EA032282EAC3030A
:10C710001BB21FFA83FE8142A4F84CE0EAD183F0F9
:10C72000320383EA0313DBB21A0982EA1E2282EA89
:10C73000032282EAC303A6461BB21FFA83FC5EF8FB
:10C740004E0F2B4EA4F84CC0DBB24FEA1C2884F8E5
:10C750005D3084F85E80DEF80410DEF8082007C63D
:10C76000BEF80C109EF80E203180B27004F58A6677
:10C7700084F8508484F84F3415F8011FD4F8FC0372
:10C7800002F038FBAE42F7D108E0013B84F80A34EE
:10C79000AFE5019B03F1FF3984F80F94C4F80074EE
:10C7A000FEF728BB2D2384F83332FEF7E3BF94F85D
:10C7B0001432D9F80020C4F81022013B012B3EF6B8
:10C7C00002AF1022022384F8E62184F8E831FEF754
:10C7D000FABE00BFBC8D002000000000D34D6210E7
:10C7E00067666666E01D00206F3D002054910308D7
:10C7F000CC210020DEF80000000600F1CC839CF87C
:10C800000C0000283FF440A894F89613032900F286
:10C81000B485DFE811F05F01550146012F01B4F83E
:10C82000E43300220133A4F8E43384F8DC23FEF778
:10C83000D0BA84F88F03FFF76DBA0A4608460D4652
:10C8400000918C4688468A460B46B4F8D013A64E13
:10C85000CDF818E0C1EB012186FB016E8E44C917AB
:10C86000C1EB6E21BDF80060ADF81E804FF0000EE8
:10C87000ADF820C0ADF82260ADF824508DF82CE062
:10C88000ADF81CA0ADF82600ADF82820ADF82A3090
:10C890008DF82D1006AD0FCD944E84F851E0B646BC
:10C8A000AEE80F0095E8030094F816C44EF8040BA8
:10C8B00023250CF10108FE201623C822AEF8001033
:10C8C00084F8535084F850C084F8168484F84E00DD
:10C8D00084F84F30311F84F852204FF6FF7501E085
:10C8E00011F8013B6B4083EA0313DBB21A0982EAB9
:10C8F000152242EA03228E4282EAC305F0D17B4927
:10C90000A4F84C5001F1160011F8013B6B4083EA8A
:10C910000313DBB21A0982EA152282EA032282EAB1
:10C92000C3031BB29DB28142A4F84C50ECD183F0FA
:10C93000F40383EA0313DBB24FEA131E8EEA152ECB
:10C940008EEA032E8EEAC30E25460FFA8EFE1FFADC
:10C950008EF855F84E0F664EA4F84C805FFA8EFEA6
:10C960004FEA182C84F86AE084F86BC06968AA68FA
:10C97000EB680FC628696969AA6904F23F4507C6D2
:10C9800004F25D4684F85DC484F85CE415F8011F88
:10C99000D4F8FC0302F02EFAAE42F7D1FFF782BAC8
:10C9A000B4F8D631DFED536A07EE903AB4F8D031DF
:10C9B000F8EEE77A07EE103A67EEA67AB8EE477A15
:10C9C0006FE5D4F8CC214C4982EAE273A3EBE27321
:10C9D00003EB5303A1FB0331C908002AACBF41F0AC
:10C9E000004141F04041FFF784B894F8C431042B72
:10C9F0008CBF03250225FEF744BC012338682B7049
:10CA000002F0ECF90546386802F0E8F96D067EF4AC
:10CA10005AAA8A2800F09F848E287EF454AA94F89B
:10CA20004832002B7EF481A9344BC4F850322D23B8
:10CA300084F85432FEF751BA94F8C431042B8CBFF9
:10CA400003260226FFF741BA2D4B94F8B9211B8823
:10CA500003EB830303EB83039D00ADB2002A40F098
:10CA6000B1844FF0FF330FFA83FA0FF087FA40B228
:10CA7000FEF7D8BCD4F89C2353799079D17903F18F
:10CA8000407303EB002303EB0141002384F896334A
:10CA90004FF4826027F08DF9002384F86132FEF7AD
:10CAA0007FB9D4F89823137A507992781B0403EB5A
:10CAB000002313444A1C84F8962303EB0161E7E743
:10CAC000D4F89823D379107952781B0403EB002310
:10CAD0001344EFE7D4F898239379D07812781B04A5
:10CAE00003EB00231344E5E703082080E01D00204A
:10CAF000CC2100200AD7233C1F85EB51701F00205A
:10CB00003C950020022027F0E5F9FF2026F0CEFF1B
:10CB10000378FF2B00F0D58390F90100C517EDB223
:10CB2000C0B227F0ADF9284627F0AAF9032027F074
:10CB3000D1F9FF2026F0BAFF0378FF2B00F05783CE
:10CB4000B0F90850E8B2C5F3072527F099F928464F
:10CB500027F096F994F8B831002B40F09382D24B2D
:10CB60001B68980640F1398294F8C231990700F1A8
:10CB70006D8300252F46012027F0ACF9384627F0B9
:10CB80007FF9284627F07CF9092027F0A3F9002037
:10CB900027F076F9002027F073F9B4F8DA2194F839
:10CBA000C451B2F5967F0AD994F8643103F00F03AB
:10CBB000072B04D842F20F75954228BF1546BB4F8C
:10CBC000052027F087F93B7A002B00F0BD83A5F103
:10CBD000200307EE903A9FEDB67AF8EEE77AF6EE8C
:10CBE000006A67EE877ABEEE007AF5EEC07AF1EE63
:10CBF00010FA58BFB0EE667A77EE877AFDEEE77AE4
:10CC0000CDED007ABDF90050E8B227F039F9C5F34F
:10CC1000072027F035F994F8C221002304930593E7
:10CC2000930700F1BD8294F8DC31012B00F0B8824B
:10CC3000B7F90030DFED9F6A07EE103AB7F902301E
:10CC400007EE903AB8EEC77AF8EEE77A27EE267A42
:10CC500067EEA67ABDEEC77AFDEEE77A06A88DEDFF
:10CC6000067ACDED077A27F047F95E21306802F0A9
:10CC7000C1F894F86431FEF717BA8F4B0793A3F10C
:10CC8000240600222121A3F1210703F8242CB170EE
:10CC90007270069725F028FA884B8949B4F89423D6
:10CCA000002814BF99468946530500F1B481D00786
:10CCB00000F19882910740F10683DFF828924FF047
:10CCC0000308424649467F4829F0E8FE07EB08037F
:10CCD0000EA87D4A013340F8203D9B1A002207F838
:10CCE0000820737027F05FF9FEF736BA724B774968
:10CCF00007930EAEA3F1210046F8200D0A2003F899
:10CD0000230C0027082003F8220C03F8247C30466B
:10CD10000988FCF742FE6E4B6E491B6881FB0321BC
:10CD2000DB17C3EBA101304689B2FCF736FE0FF0EA
:10CD300025F9069BB4F8BA21591C06911F70069B71
:10CD4000110A5F1C06971970069B591C06911A70F0
:10CD5000069B5A1C06921870304627F024F9FEF7FD
:10CD6000F8B9B4F9AE319FED5C8A534A079207EEE9
:10CD7000903AF8EEE77A0EAE67EE887AA2F12101DA
:10CD8000FDEEE77A46F8201DA2F124030020CDED48
:10CD9000007A02F8240C1E2208209A70BDF80010B8
:10CDA00058703046FCF7F9FDB4F9AC3107EE903A13
:10CDB000F8EEE77A304667EE887AFDEEE77ACDED59
:10CDC000007ABDF80010FCF7E8FDB4F9B03107EEC9
:10CDD000903AF8EEE77A304667EE887AFDEEE77A29
:10CDE000CDED007ABDF80010FCF7D7FD304627F0F6
:10CDF000DAF8FEF7ABB9C4F84CB22E70FEF763B8A0
:10CE000094F8EA03C0B10138C0B2344D013028446F
:10CE1000002215F8013B534083EA0313DBB2120AE8
:10CE2000D90042EA0322A84281EA131382EA0302EC
:10CE3000EFD1002A7EF4AAAA244B294D244AD4F823
:10CE4000F4031B881168EB619268036BE962EA6482
:10CE50000021B4F8E423EE66E963EA65002B00F0F4
:10CE60009D825B68816C8B423BBFC2685B1A5B1A18
:10CE70009B18002B7DF4A8AF036802219B6998479B
:10CE8000042394F8EB0385F874301AF0F9F80323BF
:10CE900084F8DC33FDF798BF0221386801F092FF77
:10CEA00094F85432FDF752BFBC8D00202C95002021
:10CEB000E4380E3F0050C347AC950020C4BA0308C5
:10CEC000BCBA03088B950020899500203C95002072
:10CED000409500206766666658A08B41742100204B
:10CEE0001C000020D4BA0308A3785E09012E40F08C
:10CEF000648103F00F0E13F0100300F07B81C64A2B
:10CF0000E3782779A4F88603D11887EA0300C4F8E8
:10CF10007C23134684F86662C4F88013073A84F8C9
:10CF20008C03A4F8847394F88C03BC4F0CE012F8C3
:10CF3000011BC4F87C63BA4280EA0100197007D271
:10CF4000D4F88013D4F87C33994203F10106EED172
:10CF5000BA4284F88C0300F03982127894F88C334A
:10CF60009A4200F0C781AE4BC4F868320133012207
:10CF7000B4F88413C4F86C3200204FF6F67384F8CA
:10CF80006602A4F8701284F8782284F87823A4F852
:10CF90007232FEF770BC102300250422184606A941
:10CFA0008DF818308DF819208DF81A508DF81B5017
:10CFB0008DF81C508DF81D5026F0E0FE84F861526B
:10CFC000FDF7EEBE3422FEF71FBF94F8AF33002BFF
:10CFD0000CBF04220522FFF747BB924B93E80300E6
:10CFE00006AB83E80300184626F086FF3DE61020D6
:10CFF00026F070FF284626F043FF284626F040FF23
:10D00000212026F067FF284626F03AFF284626F022
:10D0100037FFFEF723B84FF00308DFF8289250E6F9
:10D02000B4F97212D4F86C72501C02F00F0242F084
:10D0300010020029B8BF42F0200284F88E0394F851
:10D0400070028DF81820BA1B5040C0B28DF819201C
:10D0500084F88F030DF11A02FEF73FBE724B198858
:10D06000FEF7B7BD714B6420B3F900A0FEF7DAB943
:10D070001A4618461D4600939C46FFF7E6BB24223D
:10D08000FEF7C2BE6A4F97F80080B8F1000F3FF478
:10D0900066ADDFF894A1B4F8C051BAF800302D01A4
:10D0A0006422ADB202FB03834FEA4802B3FBF2F302
:10D0B00045EA0325ADB2C3F303231D43062026F042
:10D0C00009FFE8B226F0DCFE280A26F0D9FEB4F803
:10D0D000C0315849BAF8005001339BB293FBF8F2C3
:10D0E00008FB12334A7AA4F8C031012A00F0878184
:10D0F0006E23514A497B03FB05F382FB0302DB17D6
:10D10000C3EBA203002940F075814C4D9FB2A5FBF3
:10D1100007356D093A201FFA85F826F0DBFE5FFA25
:10D1200088F026F0ADFE4FEA182026F0A9FE3B203D
:10D1300026F0D0FE642303FB15739BB240480533F1
:10D1400080FB0320DB17C3EBA000C0B226F098FEE3
:10D15000002026F095FE354F394D282026F0BAFEE6
:10D160003B6885FB0325DB17C3EBA505E8B226F07A
:10D1700087FEC5F3072026F083FE042026F0AAFED2
:10D18000B4F8BA31002B40F01481BD6885F3100566
:10D19000E8B226F075FEC5F3072026F071FEDEE446
:10D1A0000121D4F8C821D4F8CC3184F8DC1104A8CA
:10D1B0000492059326F0A0FE57E5194B84F8660209
:10D1C0005E1C4FF6F6710122A4F8700284F8780212
:10D1D000C4F86832C4F86C62A4F8721284F8782338
:10D1E000FEF749BB4FF00408DFF85C9069E50025C5
:10D1F0002846AAE494F86622002A3EF43CAB94F850
:10D200008D23013202F00F02724500F0C18084F8D4
:10D210006632FEF730BB00BF981D0020941D002031
:10D2200004200020549103083C95002040950020E4
:10D23000639500202C950020310CC3301F85EB51E5
:10D2400067666666C8BA0308CCBA0308112026F0E0
:10D2500041FEB4F8D621784D4FF4F36707FB02F294
:10D2600085FB0235D217C2EB6535E8B226F008FE21
:10D27000C5F3072026F004FE192026F02BFEB4F893
:10D28000D6316E4A07FB03F382FB0301DB17C3EBC6
:10D29000611382FB0321DA17C2EB6112642101FBE7
:10D2A0001233D8B226F0ECFD002026F0E9FD94F808
:10D2B000C231B4F8D0519A077FF55BACEFB22D0ABA
:10D2C00059E428462DE4484628F000FD8046F8E45D
:10D2D0001022FEF799BD0099322026F04FFDFEF78F
:10D2E00029BD06AB00930DF11E05FEF713BD2022EC
:10D2F000FEF78ABD524BD4F87C23C4F88023002764
:10D3000003F55B7203F51B76C4F86C2203F5177105
:10D3100003F55C703A46C4F86862C4F87C3384F85C
:10D320006672A4F87072A4F8727201F0F9FE01300E
:10D3300058D0D4F86832C4F86C320123C4F868625B
:10D3400084F87833FEF797BAE8B226F099FD280AF8
:10D3500026F096FD5FE43B4B1B6898067DF5B3AD68
:10D3600094F84832002B7DF4E0AC374BC4F85032CF
:10D370002D2384F85432FDF7B0BD4B1CDBB2042BD7
:10D3800084F896334FEA01613FF47FABFFF780BB2F
:10D39000D4F88013D4F87C332C4AC4E5C269036AFC
:10D3A0009A423CBFC1685218D31A62E50822FEF7C0
:10D3B0002BBD0EF0E3FD26F063FD002026F060FD9E
:10D3C000FFF7CDBB224B1B68FFF74DBB84F88DE305
:10D3D000FEF751BA1A4618461D4600939C469846D9
:10D3E000FFF733BAD4F868320222591CC4F8681225
:10D3F0001A709EE79BB23A7893FBF2F385E63920E8
:10D4000026F068FDE8B226F03BFD280A26F038FD3C
:10D41000A1E61A46FFF719BA1A461846FFF715BAD9
:10D420001A4618461D46FFF710BA1A4618461D46FA
:10D430000093FFF70ABA00BF89B5F8141F85EB51B6
:10D44000981D0020BC8D0020A41F00208F1D0020EF
:10D4500040950020436A8269F0B4D154436A04695C
:10D46000426B0133A34228BF00234362FAB1116823
:10D4700011F0010101D0F0BC7047856A1768866918
:10D4800027F001072E449D421760D6600BD3641B22
:10D49000546081621368002143F0010380F84C104E
:10D4A000F0BC136070475D1B55608362F2E7826DCC
:10D4B000D36843F08003D360DDE700BF026B10B494
:10D4C00062B1836CC2684469D11A013B615C5DF84A
:10D4D000044B08BF13468364C8B27047016A4369AE
:10D4E000C4685B5C0131A14228BF114601625DF84E
:10D4F000044BD8B2704700BF436B13B190F84C0097
:10D500007047836A406A181AB0FA80F04009704781
:10D51000416A836A99420AD3CB1A416B026961B1AD
:10D520004968501E0B4483420AD2C01A70470269F0
:10D530001144CB1A416B0029F2D1501EC01A70471A
:10D5400000207047036B43B1826C5B6893422FBF2E
:10D55000981AC0689B1AC0187047C269036A9A4239
:10D560002FBFD01AC0688018C01A70470A4B30B558
:10D5700003F1100493F900205D78072AC8BF143A1C
:10D58000811804338D7213F8025C855413F8012C52
:10D590000A75A342EED130BDA891030803682DE9B6
:10D5A000F041DF691FB13B46BDE8F0411847002A52
:10D5B000164611DD04460D460E4400E023689B68C4
:10D5C000204698470028F9D0236815F8011B1B68EE
:10D5D00020469847AE42F1D1BDE8F08100232521D5
:10D5E0002622017042708370C3707047038A2DE950
:10D5F000F0478589ADB21D4029D00F4606464FF051
:10D6000000484FF00009B5FA85F328FA03F2D24337
:10D6100091B21B3B15403182042B16D8DFE803F092
:10D620003129211903007B6A002B32D003F1FF3A24
:10D630001FFA8AFAC7F824903C6A34B1236820465E
:10D64000514698476468002CF8D1002DDBD1BDE825
:10D65000F0873868716B036889B29847002DD2D182
:10D66000F5E77868B16B036889B29847002DCAD195
:10D67000EDE7B868F16B036889B29847002DC2D115
:10D68000E5E7F868316C036889B29847002DBAD194
:10D69000DDE7F36A1FFA83FACEE700BF30B5044630
:10D6A000806D61718389A26823F400531B041B0CF5
:10D6B000838185B0A379009213F0040230D04FF437
:10D6C000805213F00203ADF804205CD1ADF80630AF
:10D6D0004FF480630022ADF8083011F00103ADF87B
:10D6E0000C2028D1ADF80A3008238D07694648BFC1
:10D6F000ADF80A300FF0ECFFA279A36DD10724D466
:10D7000012F0080F9A8A1BD122F008021204120CA0
:10D710009A829A8992B242F400529A8105B030BD41
:10D7200013F00203ADF804202AD04FF4005513463D
:10D73000ADF80650CEE70423ADF80A300C23D4E749
:10D7400092B242F008029A82E3E710498B4215D068
:10D75000A1F548418B420FD001F580618B4209D081
:10D760000B498B42CCD105200121FDF7B9F8A279F4
:10D77000A36DC5E70320F7E70220F5E70020F3E7F4
:10D78000ADF80630A6E74FF400539FE700100140C4
:10D790000014014010B50446806DA160838923F414
:10D7A00000531B041B0C8381A37984B013F0040283
:10D7B000009135D04FF4805213F00203ADF80420ED
:10D7C0005CD1ADF806304FF480636279ADF8083073
:10D7D000D1074FF00003ADF80A30ADF80C3045BF6B
:10D7E0000423ADF80A3008230C236946920748BF8A
:10D7F000ADF80A300FF06CFFA279A36DD1071FD4EA
:10D8000012F0080F9A8A16D122F008021204120CA4
:10D810009A829A8992B242F400529A8104B010BD61
:10D8200013F00203ADF8042025D04FF40051134645
:10D83000ADF80610C9E792B242F008029A82E8E712
:10D8400010498B4215D0A1F548418B420FD001F50C
:10D8500080618B4209D00C498B42D1D10520012136
:10D86000FDF73EF8A279A36DCAE70320F7E702208F
:10D87000F5E70020F3E7ADF80630A6E74FF40053D4
:10D880009FE700BF0010014000140140F0B50C29D3
:10D8900034D8DFE801F0893333335E333333343344
:10D8A00033330700048C9689B2F802E01788734D71
:10D8B00024F480542404240C0484038C8488818BF5
:10D8C00023F4005321F4E6411B0409041B0C46EA2F
:10D8D0000E06090C43EA063341EA0721A8429BB22F
:10D8E000A4B289B200F09E8005F58065A84200F0E0
:10D8F000998092688480818302640384F0BD048CE3
:10D900009589B2F802C0B2F800E05C4F24F480744C
:10D910002404240C0484038C8688818B23F40073F4
:10D920001B0421F073011B0C45EA0C04090443EAB3
:10D930000423090CB8429BB2B6B241EA0E015CD096
:10D940004F4CA04259D0926886808183C263038481
:10D95000F0BD048C9589B2F802C0B2F800E0474EE1
:10D9600024F010042404240C0484038C8788018B85
:10D9700023F0200321F4E6411B0409041B0C45EAB3
:10D980000C04090C43EA041341EA0E21B0429BB295
:10D99000BFB289B25DD03A4CA0425AD0926887801B
:10D9A000018382630384F0BD048C9789B2F802E09E
:10D9B0001688324D24F001042404240C0484038CC2
:10D9C0008488018B23F002031B0421F073011B0CDC
:10D9D00047EA0E0709043B43090CA8429BB2A4B2D4
:10D9E00041EA060125D005F58065A84221D092685C
:10D9F0008480018342630384F0BDD589148A578AE9
:10DA000023F4006343EA05254FF6FF332B40958846
:10DA100026F440563C4343EA052346EA04169BB2EB
:10DA2000B6B290E7158A24F4804444EA8514A4B27F
:10DA30005FE7D689158A578A23F00803334324F415
:10DA4000407496883D4323F004032C433343A4B22F
:10DA5000CDE7D489158A568A23F0800343EA04135C
:10DA60004FF6BF741C40938827F44067354344EA5F
:10DA7000031347EA85079BB2BFB28FE7000001405E
:10DA8000000401402DE9F84F782200219148924C82
:10DA9000DFF86C92914D924E924FDFF868822BF036
:10DAA0007CFA91489149DFF860E2DFF860C2002219
:10DAB0001359834200F0F680B3F1804F00F0F480F8
:10DAC000AB4200F0F380B34200F0F280BB4200F0C2
:10DAD000F180734500F0F080634500F0EF8043452E
:10DAE00000F0EE80DFF828A2534500F0EB800AF545
:10DAF000806A534500F0E8800AF5806A534500F0DB
:10DB0000E580AAF5983A534500F0E2800AF5806A6C
:10DB1000534500F09A800AF5806A534508BF0D23EB
:10DB200000F094801832902AC2D1DFF8AC81704E98
:10DB300008F190074FF0030A4FF0020998F80430FB
:10DB40001C09013C032C03F00F0377D8694A32F813
:10DB5000140040FA03F2D20770D5012505FA03F349
:10DB6000013B184028F05CFD634B1B5D184416EB2D
:10DB7000C00263D056F83030604C98F8081003F1BA
:10DB80003F4000F57E00800A205C00F01F04400941
:10DB9000032805FA04F57FD0042877D0022804D1A1
:10DBA0005248406C054351484564B2F804E0BEFA5F
:10DBB0008EF2C2F11F0292B2D00803EB800002F095
:10DBC0000702046A92000F25954024EA05040462C6
:10DBD000046A01FA02F22243002502624FF0010CAE
:10DBE0002A4603E0102A05F1020527D00CFA02F0BC
:10DBF00030EA0E0102F10102F4D11C680AFA05F1C3
:10DC0000C9430C401C60D3F800B009FA05F444EA9B
:10DC10000B041C609C680C409C609C689C605C6869
:10DC200024EA0000586058685860D8680140D960FC
:10DC3000D968D960102A05F10205D7D108F1180872
:10DC400047457FF47BAFBDE8F88F0C2309EBC30396
:10DC50004FF0010A1B7D03F01F0B5B09032B0AFA2F
:10DC60000BFA0ED0042B07D0022B7FF45BAF4B6C6A
:10DC70004AEA03034B6455E70B6B4AEA03030B6361
:10DC800050E70B6C4AEA03030B644BE71748006B41
:10DC900005431648056388E71448006C054313489C
:10DCA000056482E70023D1E70123CFE70223CDE714
:10DCB0000323CBE70423C9E70523C7E70623C5E70A
:10DCC0000723C3E70823C1E70923BFE70A23BDE70A
:10DCD0000B23BBE72429002000A803080004004010
:10DCE00000080040000C00400000014000380240E5
:10DCF000A07B002094A8030890A80308D8A70308D5
:10DD0000A8910308000401400010004000140040E6
:10DD10000040014000286AD003682DE9F04F03F16C
:10DD20003F4404F57E045F4EA40A0125345D04F0EF
:10DD30001F066409032C05FA06F559D0042C00F0DF
:10DD4000AC80022C59D08588B5FA85F0C0F11F004F
:10DD500080B2C40803EB840400F00700266A800048
:10DD60000F27874026EA07062662276A01F0030686
:10DD70008240701E3A430128C1F3810CC1F30018A0
:10DD80002262C1F341113DD90024224601274FF000
:10DD9000030E03E0102A04F1020426D007FA02F071
:10DDA000A84302F10102F5D1D3F800C00EFA04F045
:10DDB000C04300EA0C0CC3F800C0D3F8008006FA98
:10DDC00004FC4CEA080CC3F800C0D3F80CC000EA0D
:10DDD0000C00D860D3F80CC001FA04F040EA0C0043
:10DDE000102AD86004F10204D8D1BDE8F08F704742
:10DDF0002D4C266C35432564A5E72B4C666C3543CA
:10DE00006564A0E7002002464FF0010E4FF00309C1
:10DE100004E00132102A00F102003CD00EFA02F7B1
:10DE200037EA0504F5D1D3F800A009FA00F4E44379
:10DE30000AEA040AC3F800A0D3F800B006FA00FA10
:10DE40004AEA0B0AC3F800A0D3F808A004EA0A0AB9
:10DE5000C3F808A0D3F808B00CFA00FA4AEA0B0A93
:10DE6000C3F808A0D3F804A02AEA07075F60D3F834
:10DE700004A008FA02F747EA0A075F60DF683C403F
:10DE8000DC60DF6801FA00F401323C43102ADC60F8
:10DE900000F10200C2D1BDE8F08F034C266B354380
:10DEA000256350E7D8A703080038024010B50409DD
:10DEB000013C032C17D80D4B33F8142000F00F0051
:10DEC00042FA00F313F001030DD0012303FA00F02E
:10DED0000138104028F0A4FB054A064B125D10449F
:10DEE00003EBC00010BD002010BD00BF94A80308C4
:10DEF00090A80308A07B002001490248FFF776BBE9
:10DF0000742900200008004001490248FFF76EBB59
:10DF10004C2900200004004002494FF08040FFF7E8
:10DF200065BB00BF24290020F0B50668B30AA3F53D
:10DF30008013022B50D8384CE55C022D4CD8437925
:10DF4000A8009F08002952D09C080223B6F80CE0D4
:10DF5000A340441907EB440743EA0E032F4C07F193
:10DF6000040E9BB244F8271044F82E20B381EFF33F
:10DF70001181502383F312884219D200A7183B69FC
:10DF80005BB33B620433421904EBC202576917B119
:10DF90001F6053690433421904EBC202976917B139
:10DFA0001F6093690433421904EBC202D76917B1A9
:10DFB0001F60D36904330022C9B21A6081F311884B
:10DFC000284404EBC004236A5BB9B38923F001033E
:10DFD0001B041B0CB381F0BDF0BD02F120032344F0
:10DFE000D1E7B3899BB243F00103B381F0BDB3899C
:10DFF0000A4C4FF0020E0EFA07FE9BB223EA0E0304
:10E0000000EB050E07EB4E07B3813B1D44F82710CC
:10E0100044F82320ABE700BF609B030824290020BD
:10E0200010B5036882480139834282B089B200F09A
:10E03000CA80A0F58060834200F0C58000F5804072
:10E04000834200F0B78000F58060834200F0B28028
:10E0500000F58060834200F0AD80764C188824681B
:10E060006408B4FBF2F4013CA4B282B2B3F1804F75
:10E070000AD07148834207D000F58060834203D004
:10E0800000F58060834202D122F0700292B26B48A8
:10E09000834200F0A18000F58060834200F0A680FA
:10E0A00022F4407200F56C4092B283421A80D96229
:10E0B0001C854FD05E4A93424CD001229A821A8826
:10E0C00092B242F001021A80B3F1804F00F09880C2
:10E0D000594A934200F0968002F58062934200F024
:10E0E000938002F58062934200F0908002F5806296
:10E0F000934200F08D8002F58062934200F08A80A6
:10E1000002F57042934200F0878002F5705293420C
:10E1100000F0848002F58062934200F0818002F575
:10E12000806293427ED0A2F5983293427CD002F571
:10E13000806293427AD002F58062934208BF0D223A
:10E1400015D002A84FF0012340F8043D1BF0F4FF66
:10E1500002B010BD0122002119869A821A8838481F
:10E1600092B242F0010283421A80ADD10A46354B89
:10E1700003EBC20301A85C7D8DF80440012300225B
:10E180008DF805308DF807308DF806201BF0D4FF90
:10E190001B2C08D02E2CDBD12B4B019301A81BF09C
:10E1A000CBFF02B010BD294B019301A81BF0C4FFA7
:10E1B00002B010BD1F4C18882468B4FBF2F4013C77
:10E1C000A4B282B252E71B4C18882468B4FBF2F464
:10E1D000013CA4B282B257E701201A80D9621C85A3
:10E1E00098821A8892B202431A8071E701201A803D
:10E1F000D9621C8598821A8892B202431A8063E71A
:10E200000122B4E70222B2E70322B0E70422AEE71C
:10E210000522ACE70622AAE70722A8E70822A6E71C
:10E220000922A4E70A22A2E70B22A0E70C229EE71C
:10E230000004014038940020000400400010004019
:10E2400000000140A89103082C0100011901000100
:10E250002B4B98423CD0B0F1804F3BD0A3F57C4390
:10E26000984239D003F58063984237D003F5806334
:10E27000984235D003F58063984233D003F580632C
:10E28000984231D003F5704398422FD003F5705374
:10E2900098422DD003F5806398422BD003F580631C
:10E2A000984229D0A3F59833984227D003F580638C
:10E2B000984207D003F58063984208BF0D2202D030
:10E2C000002070470C220F4B03EBC203187D7047F0
:10E2D0000022F8E70122F6E70222F4E70322F2E740
:10E2E0000422F0E70522EEE70622ECE70722EAE740
:10E2F0000822E8E70922E6E70A22E4E70B22E2E740
:10E3000000000140A89103082DE98048013085B044
:10E31000C3B203938A4D8B4F8B4C8C4E0A230293CE
:10E32000DFF82C9225F066FE4FF4FA7A4FF0100CCD
:10E330004FF47A70D9F80430C3F30803002B40F08F
:10E34000C180EFF31183002B40F0BC802968A268E4
:10E3500000BF2B689942F9D1D7F800E000FB0EF31B
:10E360009B1AB3FBFEF300FB01314FF0010E01914C
:10E37000D9F80430C3F30803002B40F08780EFF393
:10E380001183002B40F082802B68A16800BF2A68AF
:10E390009342F9D1D7F800B000FB0BF2521AB2FB4E
:10E3A000FBF200FB0323019A9B1AB3F57A7FDFD3BC
:10E3B000BAF1010ABED1039B002B40F0BD804FF49F
:10E3C0007A7ADFF88C9150464FF0100CD9F804306F
:10E3D000C3F30803002B40F09280EFF31183002B6E
:10E3E00040F08D802968A26800BF2B689942F9D15E
:10E3F000D7F800E000FB0EF39B1AB3FBFEF300FB23
:10E4000001314FF0010E0191D9F80430C3F3080334
:10E4100003BBEFF31183EBB92B68A16800BF2A6837
:10E420009342F9D1D7F800B000FB0BF2521AB2FBBD
:10E43000FBF200FB0323019A9B1AB3F57A7FE3D327
:10E44000BAF1010AC2D1029B013B02937FF468AF8B
:10E45000FCF73CFAEFF311888CF31288A16823686B
:10E46000DB0344BFC6F800E0A1682B6832685FFA9E
:10E4700088F888F31188D7F800801A4400FB08F365
:10E480005B1AB3FBF8F300FB0233D4E7EFF3118818
:10E490008CF31288A1682368DB0344BFC6F800E050
:10E4A000A1682B6832685FFA88F888F31188D7F87A
:10E4B00000801A4400FB08F35B1AB3FBF8F300FB7F
:10E4C000023370E7EFF311828CF31288D4F808E07E
:10E4D0002368D90303D501233360D4F808E02B68FF
:10E4E0003168D2B282F311883A68194400FB02F312
:10E4F000A3EB0E03B3FBF2F300FB013135E7EFF3BF
:10E5000011828CF31288D4F808E02368D90303D56C
:10E5100001233360D4F808E02B683168D2B282F36B
:10E5200011883A68194400FB02F3A3EB0E03B3FB16
:10E53000F2F300FB013164E718461CF0E3F83EE714
:10E54000EC7D0020F07D002010E000E0E87D002060
:10E5500000ED00E02DE9F04F013085B0C3B2039328
:10E560000B4602918B4C8C4E002B00F099808B4D0A
:10E570008B4FDFF8309225F03DFD4FF4FA7A4FF0E3
:10E58000100C4FF47A70D9F80430C3F30803002B51
:10E5900040F0DE80EFF31183002B40F0D980296832
:10E5A000A26800BF2B689942F9D1D7F800E000FBC0
:10E5B0000EF39B1AB3FBFEF300FB01314FF0010E8B
:10E5C0000191D9F80430C3F30803002B40F0878091
:10E5D000EFF31183002B40F082802B68A16800BF0D
:10E5E0002A689342F9D1D7F800B000FB0BF2521A17
:10E5F000B2FBFBF200FB0323019A9B1AB3F57A7F6F
:10E60000DFD3BAF1010ABED1039B002B40F0BD80DD
:10E610004FF47A7ADFF88C9150464FF0100CD9F80D
:10E620000430C3F30803002B75D1EFF31183002BE3
:10E6300071D12968A26800BF2B689942F9D1D7F837
:10E6400000E000FB0EF39B1AB3FBFEF300FB01316D
:10E650004FF0010E0191D9F80430C3F3080313BB46
:10E66000EFF31183FBB92B68A16800BF2A689342BE
:10E67000F9D1D7F800B000FB0BF2521AB2FBFBF253
:10E6800000FB0323019A9B1AB3F57A7FE3D3BAF117
:10E69000010AC4D1029B013B0293002B7FF467AFB8
:10E6A00005B0BDE8F08FEFF311888CF31288A168F4
:10E6B0002368DB0344BFC6F800E0A1682B6832681A
:10E6C0005FFA88F888F31188D7F800801A4400FBB5
:10E6D00008F35B1AB3FBF8F300FB0233D2E7EFF366
:10E6E00011888CF31288A1682368DB0344BFC6F845
:10E6F00000E0A1682B6832685FFA88F888F3118817
:10E70000D7F800801A4400FB08F35B1AB3FBF8F358
:10E7100000FB023370E7EFF311828CF31288D4F818
:10E7200008E02368D90303D501233360D4F808E057
:10E730002B683168D2B282F311883A68194400FB21
:10E7400002F3A3EB0E03B3FBF2F300FB01317FE70F
:10E75000EFF311828CF31288D4F808E02368D90310
:10E7600003D501233360D4F808E02B683168D2B2B6
:10E7700082F311883A68194400FB02F3A3EB0E03FD
:10E78000B3FBF2F300FB013118E718461BF0BAFFA8
:10E790003EE700BF10E000E0E87D0020EC7D0020B7
:10E7A000F07D002000ED00E0204B5B68C3F3080320
:10E7B00030B4BBB9EFF31183A3B91D4B1D4C1868DE
:10E7C000A16800BF1A689042F9D11B4B1C684FF436
:10E7D0007A7202FB04F3591AB1FBF4F130BC02FB6C
:10E7E00000107047EFF31182102383F31288114950
:10E7F0008C680B6813F4803F104B02D00120186026
:10E800008C680B49D2B20D68186882F311880A4BE4
:10E8100019684FF47A72284402FB01F31B1B30BCC9
:10E82000B3FBF1F302FB0030704700BF00ED00E0E6
:10E83000EC7D002010E000E0F07D0020E87D00206D
:10E840002DE9F84F8046FFF7AFFF254E2549DFF849
:10E85000A0E0254A254D844610274FF47A74012004
:10E86000DEF80430C3F30803D3B9EFF31183BBB967
:10E870000B68D2F808A000BFD1F800904B45F7D143
:10E88000D6F800B004FB0BF9A9EB0A09B9FBFBF9B8
:10E8900004FB0393A3EB0C034345E1D3BDE8F88FDE
:10E8A000EFF3118A87F31288D2F808B01368DB03FC
:10E8B00044BF2860D2F808B00B68D5F800905FFA22
:10E8C0008AFA8AF31188D6F800A0994404FB0AF367
:10E8D000A3EB0B03B3FBFAF304FB0933DAE700BF46
:10E8E000F07D0020EC7D002010E000E0E87D0020BD
:10E8F00000ED00E02DE9F04FDFF830C1474A48490C
:10E90000484E494D8046102718F1FF38C0F08480EA
:10E91000DCF80430C3F30803002B5CD1EFF3118360
:10E92000002B58D10B68946800BF08688342F9D166
:10E93000D6F800904FF47A7000FB09FEAEEB040E9F
:10E94000BEFBF9FE00FB03EEDCF80430C3F3080362
:10E950004FF47A740120FBB9EFF31183E3B90B682C
:10E96000D2F808A000BFD1F800904B45F7D1D6F8F7
:10E9700000B004FB0BF9A9EB0A09B9FBFBF904FB96
:10E980000393A3EB0E03B3F57A7FBDD2DCF804301A
:10E99000C3F30803002BDFD0EFF3118A87F312884B
:10E9A000D2F808B01368DB0344BF2860D2F808B07F
:10E9B0000B68D5F800905FFA8AFA8AF31188D6F8C6
:10E9C00000A0994404FB0AF3A3EB0B03B3FBFAF397
:10E9D00004FB0933D5E7EFF3118487F31288D2F8EB
:10E9E00008901368D80303D501232B60D2F8089050
:10E9F0000B682868E4B284F31188D6F800A04FF4BD
:10EA00007A7400EB030E04FB0AF3A3EB0903B3FBD8
:10EA1000FAF304FB0E3E97E7BDE8F08F10E000E04C
:10EA2000EC7D0020F07D0020E87D002000ED00E07E
:10EA300030B4EFF31183102282F312880649074C99
:10EA40000A680748013200250A602560DBB20268C7
:10EA500083F3118830BC7047EC7D0020E87D0020F6
:10EA600010E000E00F4B1B88014643B90E4B0F4AE4
:10EA70001B7810680BB981F00101FAF7B5B80C4B9F
:10EA80005A691AB118B91A68106058747047094A5F
:10EA900018681188084A92FBF1F20121026059744A
:10EAA000704700BFC47D0020C67D0020C87D0020C7
:10EAB000CC7D0020E47D002020A1070038B5254B47
:10EAC0005C69236B73B1A36D626BCAB1998A1A88B2
:10EAD000C90592B201D5D20700D438BD4FF6F772FE
:10EAE0001A8038BDA36D99891A88890692B2EBD530
:10EAF0009206E9D5E26ACAB1988880B29047E2E707
:10EB000099891A880D0692B2E0D51006DED5A26A60
:10EB1000616A8A4219D0A1692569885C98800132AE
:10EB2000B2FBF5F105FB1122A262CFE79B88E269F7
:10EB30006169DBB28B54E269E068A36D0132B2FB1C
:10EB4000F0F100FB1122E261BEE7DA6822F08002F8
:10EB5000DA60BBE7003C002038B5254BDC68236B4E
:10EB600073B1A36D626BCAB1998A1A88C90592B252
:10EB700001D5D20700D438BD4FF6F7721A8038BDE0
:10EB8000A36D99891A88890692B2EBD59206E9D5C8
:10EB9000E26ACAB1988880B29047E2E799891A88F8
:10EBA0000D0692B2E0D51006DED5A26A616A8A42ED
:10EBB00019D0A1692569885C98800132B2FBF5F112
:10EBC00005FB1122A262CFE79B88E2696169DBB293
:10EBD0008B54E269E068A36D0132B2FBF0F100FBF7
:10EBE0001122E261BEE7DA6822F08002DA60BBE758
:10EBF000003C002038B5254B9C68236B73B1A36D96
:10EC0000626BCAB1998A1A88C90592B201D5D20736
:10EC100000D438BD4FF6F7721A8038BDA36D9989BC
:10EC20001A88890692B2EBD59206E9D5E26ACAB192
:10EC3000988880B29047E2E799891A880D0692B2C7
:10EC4000E0D51006DED5A26A616A8A4219D0A169B0
:10EC50002569885C98800132B2FBF5F105FB112231
:10EC6000A262CFE79B88E2696169DBB28B54E269FB
:10EC7000E068A36D0132B2FBF0F100FB1122E2610A
:10EC8000BEE7DA6822F08002DA60BBE7003C0020D1
:10EC900038B5254B1C68236B73B1A36D626BCAB189
:10ECA000998A1A88C90592B201D5D20700D438BD15
:10ECB0004FF6F7721A8038BDA36D99891A888906B4
:10ECC00092B2EBD59206E9D5E26ACAB1988880B2D1
:10ECD0009047E2E799891A880D0692B2E0D51006AE
:10ECE000DED5A26A616A8A4219D0A1692569885C69
:10ECF00098800132B2FBF5F105FB1122A262CFE749
:10ED00009B88E2696169DBB28B54E269E068A36DBC
:10ED10000132B2FBF0F100FB1122E261BEE7DA68DA
:10ED200022F08002DA60BBE7003C0020436B826A7D
:10ED3000816930B41C68456A24F001041144AA4278
:10ED40001C60D9600DD3016900248A1A5A6084625C
:10ED50001A68002142F0010280F84C1030BC1A60A1
:10ED60007047AA1A5A608562F2E700BF03685B6ABF
:10ED700003B11847704700BF03681B6A03B1184707
:10ED8000704700BF03682DE9F041DF691FB13B46C2
:10ED9000BDE8F0411847002A164611DD04460D462D
:10EDA0000E4400E023689B68204698470028F9D06D
:10EDB000236815F8011B1B6820469847AE42F1D125
:10EDC000BDE8F08103689B69184700BF03685B6971
:10EDD000184700BF03681B69184700BF0368DB685A
:10EDE000184700BF03689B68184700BF03685B684B
:10EDF000184700BF03681B68184700BF38B50C46AA
:10EE0000097849B1054601342B6828461B689847A4
:10EE100014F8011B0029F7D138BD00BF10B40B4B0B
:10EE20000B4A1C7801238340234052F8200031B95B
:10EE3000B3FA83F149095DF8044BF9F7D5BE191C03
:10EE400018BF01215DF8044BF9F7CEBEB67D002056
:10EE5000B87D0020064B53F820302BB11A689B88F0
:10EE600051690B4201D1138370475383704700BF30
:10EE7000B87D0020026802F13F4303F57E032DE9CF
:10EE8000F04F9B0A544DEB5C03F01F055B09012416
:10EE9000032B04FA05F400F09980042B00F0918014
:10EEA000022B3ED001F00306731E012BC1F3810C2F
:10EEB000C1F300188588C1F3411137D900242346D6
:10EEC00001274FF0030E03E0102B04F1020426D0BB
:10EED00007FA03F0A84303F10103F5D1D2F800C00B
:10EEE0000EFA04F0C04300EA0C0CC2F800C0D2F8DD
:10EEF000008006FA04FC4CEA080CC2F800C0D2F804
:10EF00000CC000EA0C00D060D2F80CC001FA04F08A
:10EF100040EA0C00102BD06004F10204D8D1BDE807
:10EF2000F08F2E4B5D6C2C435C64BBE700200346E6
:10EF30004FF0010E4FF0030904E00133102B00F1F4
:10EF400002003CD00EFA03F737EA0504F5D1D2F8F7
:10EF500000A009FA00F4E4430AEA040AC2F800A097
:10EF6000D2F800B006FA00FA4AEA0B0AC2F800A08A
:10EF7000D2F808A004EA0A0AC2F808A0D2F808B039
:10EF80000CFA00FA4AEA0B0AC2F808A0D2F804A068
:10EF90002AEA07075760D2F804A008FA03F747EAFD
:10EFA0000A075760D7683C40D460D76801FA00F47C
:10EFB00001333C43102BD46000F10200C2D1BDE804
:10EFC000F08F064B1D6B2C431C636BE7034B1D6CD2
:10EFD0002C431C6466E700BFD8A703080038024032
:10EFE0002DE9F04F4A484B494B4B4C4C4FF0010A2E
:10EFF0004FF002094FF004084FF0080C4FF0100ECC
:10F0000020274026802530F8022B12F0010F03D074
:10F010001960A3F804A0083312F0020F03D019609E
:10F02000A3F80490083312F0040F03D01960A3F87A
:10F030000480083312F0080F03D01960A3F804C04D
:10F04000083312F0100F03D01960A3F804E008335E
:10F0500012F0200F02D019609F80083312F0400F89
:10F0600002D019609E80083312F0800F02D0196020
:10F070009D80083312F4807F05D04FF4807B1960A7
:10F08000A3F804B0083312F4007F05D04FF4007BDE
:10F090001960A3F804B0083312F4806F05D04FF460
:10F0A000806B1960A3F804B0083312F4006F05D028
:10F0B0004FF4006B1960A3F804B0083312F4805FBA
:10F0C00005D04FF4805B1960A3F804B0083312F444
:10F0D000005F05D04FF4005B1960A3F804B008335B
:10F0E00012F4804F05D04FF4804B1960A3F804B0A0
:10F0F0000833D20B04D04FF4004219609A800833D1
:10F1000001F58061A1427FF47EAFBDE8F08F00BFC2
:10F1100094A8030800000240A07B002000100240D9
:10F120002DE9F04FB0F908502DED048B0D81EDB2B3
:10F13000382D87B00C4600F0A782804691462ED924
:10F14000802D00F0E68078D8522D00F0968040F2B5
:10F150007582542D00F0DF826E2D40F02181824BAC
:10F160000A681B88814DFF2BA8BFFF23511C21601B
:10F170001370A96881F3100189B22046FAF731FCB7
:10F180007B4B20461988FAF72CFC296801F30F0104
:10F1900089B220460125FAF724FC2B4646E0042DCF
:10F1A00062D040F20282202D00F0978040F231823E
:10F1B000242D00F0A882282D40F0F2800B68DFF8A3
:10F1C000D4816C4E591C022221601A7023680627D4
:10F1D0005A1C22601F7023680A22591C21601A7071
:10F1E000236801255A1922601D70B8F800102046C6
:10F1F000FAF7F7FBB8F802102046FAF7F2FB23689B
:10F200005A1922601F7023685022591921601A7000
:10F2100023680022591921601A7031882046FAF7B4
:10F22000E0FB71882046FAF7DCFB2B462846638119
:10F2300007B0BDEC048BBDE8F08F822D25D0C0F067
:10F240008282A02D00F07382FE2D40F0A9804A4DED
:10F2500005F1080635F8021B2046FAF7C2FBB54255
:10F26000F8D101252B46E1E72A4644492046FAF722
:10F2700073FB00212046FAF7B4FB22680021531CDF
:10F28000012523602B461170D0E70B683C4A374DAF
:10F2900011783C4A581C20601970D1882046FAF732
:10F2A000A0FB314B22681B88FF2B02F10101A8BF94
:10F2B000FF2321601370A96881F3100189B22046F1
:10F2C000FAF78FFB296801F30F0189B22046FAF79C
:10F2D00088FB2D4B22681978D1E70B68294D591C02
:10F2E0006A7821601A7023682A78591C21601A7084
:10F2F0002368AA78591C21601A70E9882046FAF719
:10F3000070FB23682A79591C21601A702268697978
:10F31000B5E7DFF884801D4F1D4EDFF880A008F1AF
:10F320000D090A2516E0322D00F05781A5F13C00A9
:10F33000C0B2132840F2578100232268511C21607B
:10F3400015702268C14502F101012160137088D057
:10F3500018F8015B0A2DE6D1BAF80030FF2BA8BFE0
:10F36000FF23DBB2E9E700BF3C9500204095002079
:10F370005C210020E42900209894002040BB030871
:10F3800063950020401F0020A01F0020676666666E
:10F39000FC290020208D0020699203082C2A0020DF
:10F3A000A5F10A03E72B00F2EA80DFE813F08F05EE
:10F3B000E800E800E800E800E800E800E800E8000D
:10F3C000E800E800E800E800E800E800E800E800FD
:10F3D000E800E800E800E800E800E800E8003F0591
:10F3E000E800E800E8002E05E800E800E80029054C
:10F3F000E800E804E800CF04E800C304E800BE0425
:10F40000E8008D02E8005602E800E800E800470244
:10F410004E02E800B404E800E800AB04E800E800AD
:10F42000E800E800E8008D04E800E800E800E800F3
:10F430007104E800DB07E8003602C307E800E800D3
:10F44000E800E800E800E800E8007F07E80054076B
:10F45000E8002507E800A306E8009206E800E800B7
:10F46000E800E8006C06390630060806F605D00507
:10F47000BA05A1051904E800DF03A003E800E800CD
:10F48000E800E8009403E800E8003604E800E8003B
:10F49000E8002504580483034403E800E800E8007A
:10F4A00033032003E800E800E800E800E800E80093
:10F4B000E800E800E800E800E800E800E800E8000C
:10F4C000E800E800E8006C06E800E800E800E80072
:10F4D000E800E800E800E800E800E800E800E800EC
:10F4E000E800E802E800E800E800E800E800E800DA
:10F4F000E800E800E800E800E800E800E800E800CC
:10F50000E800E800E800E800E800E800E800E800BB
:10F51000E800E800E800E800E800E800E800E800AB
:10F52000E800E800E800E800E800E800E800E8009B
:10F53000E800E800E800E800E800E800E800E8008B
:10F54000E800E800E800E800E800E800E800E8007B
:10F55000E800E800E800E800E800E800E800E8006B
:10F56000E800E800E800E800E800E800E800E8005B
:10F57000E800E800E800E800E800DC02B202742DD0
:10F5800000F03881772D64D1D8F80030D8F8042005
:10F590009A421EBF5A1CC8F800201978B84A08BF02
:10F5A0000021204606F06AFC5BE6022D00F0A380F5
:10F5B00000F29080012D7FF4F3AE0B680022591CFD
:10F5C00021601A7023685A1C22601D702268242151
:10F5D000531C23602B46117028E63388FF2BA8BFED
:10F5E000FF23DBB2A9E624F061FA00283FF4A4AEC1
:10F5F00003780A2B00F20F81B0F9023087FB031267
:10F60000DB17C3EBA2039BB2FF2BA8BFFF23DBB228
:10F6100093E6052D7FF4C4AE0B229A492046FAF7F3
:10F620009BF9082298492046FAF796F90125072206
:10F6300096492046FAF790F92B46F7E5442D7FF4DA
:10F64000AFAE002A3FF40DAE914B136001252B465F
:10F65000ECE5F52D01F02B80762D00F0A586472DE9
:10F6600000F04487292DD8F8003000F01387392D99
:10F6700000F0E186212D00F0EA862846414606F09A
:10F680008FFE054603B2D1E50A68824B0125511C65
:10F6900021601570226805215019206011702268C0
:10F6A0000A21501920601170226800215019206031
:10F6B00011702268197850192060117022685978E9
:10F6C00050192060117022689978531923602B46D5
:10F6D0001170ABE50B680222591C21601A70236877
:10F6E00001255A1922601D702268002153192360D8
:10F6F0002B4611709AE50422674920460125FAF746
:10F700002BF92B4692E5654B196820460125FAF73F
:10F7100051F92B468AE50B6800215A1C22601970AA
:10F7200022680125531923602B4611707EE55C4B3E
:10F7300008461968FAF73EF95A4B20461968FAF755
:10F7400039F9594BE0E7DFF87C91584F09F10E0683
:10F750004FF00A081DE0B8F1500F32D0B8F1320F67
:10F7600031D0A8F13C00C0B213282FD9002529467A
:10F7700023685A1C2260204683F80080FAF731F98A
:10F7800029462046FAF72DF9B1453FF46AAD19F83C
:10F79000018BB8F10A0FDED1454B9D68196805EB66
:10F7A00085054FF6FF736D009D42A8BF1D46994227
:10F7B000A8BF194625EAE57521EAE171ADB289B223
:10F7C000D6E73C4BE9E797E82200E8E724F06EF93A
:10F7D0000028CBD003780A2BC8D8B0F90430B0F990
:10F7E000061003EB830383F3500521EAE171ADB208
:10F7F00089B2BDE7D8F80030D8F804209A421EBF7D
:10F800005A1CC8F8002019782B4A08BF002120464E
:10F8100006F034FB25E50023F9E6236800255A1C91
:10F8200022601D7023685A1C22601D7023685A1CB8
:10F83000226029461D702046FAF7BCF800212046B8
:10F840000125FAF7B7F82B46F0E422680121531896
:10F8500023600D460B461170E8E4184D184E05F173
:10F86000280795F902100023F2568A4200F0C58558
:10F870000C333C2BF8D10835AF42F2D1F1E400BF94
:10F880002D5B010848BB030854BB030860BB030899
:10F89000215C01086752002038BB0308C8530020D0
:10F8A000107AFF1F147AFF1F187AFF1FF429002017
:10F8B000A8290020E8290020F95B0108E09B00202E
:10F8C0005845002059920308974B03F15A052268C6
:10F8D0005979501C2060117022681978501C2060E2
:10F8E000117022685978501C206011702268997834
:10F8F000501C206011702268D978501C2060117053
:10F90000226819790633501C9D4220601170DED1A7
:10F91000A7E4864B03F1700522681978501C20601B
:10F92000117022685978501C2060117022689978F3
:10F93000501C206011702268D978501C2060117012
:10F9400022681979501C2060117022685979501C66
:10F9500020601170226899790733501CAB422060F7
:10F960001170D9D17DE4724D2046A989FAF739F892
:10F97000698920460125FAF734F82B4656E42368B6
:10F98000DFF8E0C1591C9CF8002021601A709CF837
:10F990000030002B3FF465AC664E674D6748684900
:10F9A0000023226816F8017F02F1010EC4F800E07E
:10F9B0001770226815F8017F02F1010EC4F800E00B
:10F9C0001770226810F8017F02F1010EC4F800E000
:10F9D0001770226811F8017F02F1010EC4F800E0EF
:10F9E00017709CF8002001339342DADB39E4226877
:10F9F000544B501C19782060117022685978501CA3
:10FA00002060117022689978501C20601170226863
:10FA1000D97834E44C4D2046A98AF9F7E2FFE98A07
:10FA20002046F9F7DEFF298B20460125F9F7D9FF9B
:10FA30002B46FFF7FBBBDFF830E10027FEB2714633
:10FA400000232268501C206016702268501C206021
:10FA50001370226811F8010F0133551C062B256025
:10FA60001070EED10137062F0EF1060EE6D13749A0
:10FA700000232268501C206017702268501C2060F0
:10FA80001370226811F8010F0133551C0B2B2560F0
:10FA90001070EED123682E49581C072220601A707E
:10FAA00023680022581C20601A70226891F8F01018
:10FAB000FFF7E5BB2368274A274910781C4A5D1CDD
:10FAC0002560187023689278581C20601A7022688C
:10FAD0008978FFF7D4BB214952232268501C20604B
:10FAE000137011F8013F002BF7D1FFF7BABB1C4888
:10FAF00000232268056803EB4301561C6D5C2660F9
:10FB00001570026825680A446E1C527826602A70B7
:10FB1000026825680A4401339278691C0A2B216027
:10FB20002A70E6D1FFF79DBBC82700207C75002016
:10FB3000308D00209F3D0020AF3D0020CF3D0020B4
:10FB4000BF3D0020843D0020C4400020C389002028
:10FB5000E08800200C9C0020488D0020289203089B
:10FB6000242100209D3D00209F890020B44D236862
:10FB70002A68591C127821601A702B6822689978BB
:10FB8000531C2360002311702A6821681A44013332
:10FB90005279481C032B20600A70F5D123682A682B
:10FBA000591C127A21601A7023682A68591CD2786D
:10FBB00021601A7023682A68591C127921601A7012
:10FBC0002B6820465989F9F70CFF23682A68591CCD
:10FBD000527A21601A702B6822685978FFF74FBB60
:10FBE00000212046F9F7E6FE012500212046F9F71D
:10FBF000F8FE2B46FFF71ABB924D20462988F9F7ED
:10FC0000F0FE69882046F9F7ECFEA9882046012518
:10FC1000F9F7E7FE2B46FFF709BB8B4D05F16006B0
:10FC2000A9882046F9F7DDFEE9882046F9F7D9FED4
:10FC300029892046F9F7D5FE2368AA7A591C216044
:10FC40001A702368EA7A591C21601A7055F80C1B47
:10FC50002046F9F7AFFEB542E2D1FFF702BB2268BA
:10FC60007A4B78491878551C2560107022685878AE
:10FC7000551C2560107022689B78501C2060137002
:10FC8000C98820460125F9F7ACFE2B46FFF7CEBA0E
:10FC900023686F4D591C2A7821601A7023686A788E
:10FCA000591C21601A7069882046F9F79AFE23686A
:10FCB0002A79591C21601A70E9882046F9F791FECB
:10FCC0002268297AFFF7DBBAFAF7D8FA2368614D80
:10FCD000002803F101010CBF0222032221601A70E7
:10FCE00029882046F9F766FEE9682046F9F762FEA2
:10FCF000FAF714FA012501462046F9F75BFE2B4678
:10FD0000FFF794BA0822544920460125F9F724FE4A
:10FD10002B46FFF78BBA2268504B501C9978206015
:10FD2000117022685978FFF7AABA4B4B2268597DA7
:10FD3000FFF7A5BA4A4D05F1800655F8041F204685
:10FD4000F9F738FEAE42F8D1FFF78BBA454D05F111
:10FD50004006B5F880102046F9F743FE236895F871
:10FD60008220591C21601A70236895F8832004357D
:10FD7000591CAE4221601A70EBD1FFF772BA364DB2
:10FD800023682A7A591C21601A70A98B2046F9F73A
:10FD900028FE298B2046F9F724FE698B2046F9F7C7
:10FDA00020FE2368EA7C591C21601A70E98C2046E9
:10FDB000F9F717FE298D2046F9F713FE2368AA7F6D
:10FDC000591C21601A70236895F82020591C216065
:10FDD0001A70A98C2046F9F704FE2368EA7A591CA8
:10FDE00021601A70E9682046F9F7E4FD23682A7C4F
:10FDF000591C21601A70226895F82110FFF73FBA4C
:10FE0000194B22681978FFF73ABA184D204629880D
:10FE1000F9F7E7FDA9882046F9F7E3FD298920468F
:10FE20000125F9F7DEFD2B46FFF700BA104D114F03
:10FE300005F15006002128780F4A0B4626E000BF46
:10FE4000282100209488002088740020288D00201C
:10FE5000A88800203C08002098450020548D0020F0
:10FE6000DC880020E088002004230020243C0020BF
:10FE70006C81002028920308909203080133242B00
:10FE800002F10C0200F0B68212F80C1C8842F5D187
:10FE900003EB4303226807EB8303511C93F86430A0
:10FEA0002160137023686A78591C21601A702368D6
:10FEB000AA78591C21601A702368EA780435591C05
:10FEC000AE4221601A70B5D1FFF7CBB9AE4825F02C
:10FED000FDFE00287FF7C5A9AB4B1D18226813F85B
:10FEE000011B501C9D4220601170F7D1FFF7B9B97A
:10FEF000A64D20462988F9F774FD69882046F9F750
:10FF000070FDB5F90430A249DA1781FB0313C2EB87
:10FF1000A30399B220460125F9F763FD2B46FFF7AD
:10FF200085B99C4B20461988F9F75BFD9A4B204612
:10FF30001988F9F756FD994B21681A7801254B1C51
:10FF400002F0010223602B460A70FFF76FB9944B51
:10FF500022681B78934D511C03F00203216013703B
:10FF600023682A78591C21601A7069682046F9F7BD
:10FF700021FDA9682046F9F71DFDA9892046F9F75A
:10FF800030FD698A2046F9F72CFDA98A2046012513
:10FF9000F9F727FD2B46FFF749B9834E3378002B3D
:10FFA0003FF45FA9814F002537F8021F2046F9F77B
:10FFB00018FD337801359D42F6DBFFF752B97C4DD1
:10FFC0007C4EDFF82482DFF82492DFED7B8ADFEDC0
:10FFD0007B9A9FED7B9A05F1200708E020460435C7
:10FFE000F9F7FFFCAF4206F118063FF43AA9717C1D
:10FFF0000029F3D095ED008AB0EE480A26F0C2FE43
:020000040801F1
:1000000098F80030002B40F0C48381B2E6E710225C
:100010006C4920460125F9F79FFC2B46FFF706B9EE
:10002000694E338AB3F5007F06F1340594BF01278A
:100030000427403655F8041B91FBF7F1204689B29E
:10004000F9F7CFFCAE42F5D1604D614F05F10C06DA
:10005000B5EC010AD7ED087A80EE270A26F092FE69
:1000600081B22046F9F7BDFCAE42F1D1594D05F100
:100070000C0655F8041B204689B2F9F7B2FCAE42D3
:10008000F7D1FFF7EEB80023DFF86491DFF864B131
:100090000393029304930593984601214FF6FF7A48
:1000A00007E008F10108B8F10B0F00F0678219F9B9
:1000B000011F4E1CF5D04AFA08F3D807F1D5BBF85A
:1000C000003043FA08F3DA07EBD504A8FAF70AF888
:1000D000E7E72368404A4149D078414A5D1C2560E2
:1000E000187023681278581C20601A702268C9782A
:1000F000FFF7C5B800212046F9F773FC0021204620
:10010000F9F76FFC00212046F9F76BFC2268354DAA
:100110000023511C2160137022682968501C91F83B
:100120002F102060117022682968501C91F83A1035
:100130002060117022682968501C91F83B102060E3
:1001400011702268511C216013702268511C2160BB
:1001500013702268511C216013702B682046D98FC0
:10016000F9F73FFC2B682046998FF9F73AFC236892
:100170002A68591C92F8312021601A702B68226875
:1001800093F83210FFF77BB8CF790020381F00209A
:1001900067666666D01F0020D21F0020923F0020B5
:1001A0004E1F0020501F0020D4220020DE220020FD
:1001B00030810020489200200000404200407444FA
:1001C00000E0824420810020F41E002048A400208A
:1001D000209C0020C8880020308D0020488D002001
:1001E000408D002024210020EC400020C845002044
:1001F0007892030820210020B24D23686A79B24E1C
:10020000591C21601A7033682046198CF9F7E9FBF4
:1002100033682046598CF9F7E4FB69892046F9F7E1
:10022000E0FBA9892046F9F7DCFB33682046998C6E
:10023000F9F7D7FB33682046D98CF9F7D2FBE98967
:100240002046F9F7CEFB298A20460125F9F7C9FB9C
:100250002B46FEF7EBBF9B4EF378002B00F0858218
:1002600023680822591C21601A70236801229918FA
:1002700021601A702368954D591C2A7921601A70E3
:100280002368AA78591C21601A7029882046F9F73A
:10029000A8FB698A2046F9F7A4FB2368F279591C68
:1002A00021601A702268E978FEF7E9BF12F0BEF803
:1002B000FF28064600F0958206A9002501F8125D88
:1002C0000DF105008DF8055012F090F806A800F821
:1002D000115D12F07FF806A800F8105D0EF06EFFB9
:1002E00006A820F8085D0EF05DFF23685A1C226006
:1002F0001E7023689DF80520591C21601A70236820
:100300009DF80620591C21601A7023689DF807206B
:10031000591C21601A7023689DF80820591C21601F
:100320001A70BDF8101020460125F9F75AFB2B462C
:10033000FEF77CBF2268664B0125511C21601570B9
:100340002268997850192060117022681978501924
:100350002060117022685978531923602B46117060
:10036000FEF764BF5B4E3378002B3EF47AAF5A4FF2
:100370000025B846236817F81520591C21601A700B
:1003800098F8011001EB810101EB810101F2EE21EE
:1003900089B22046F9F725FB337801359D4208F1F3
:1003A0000208E7DBFEF75DBFD8F800305A1CC8F83A
:1003B00000201B78002B00F04F82102B07BF474A0C
:1003C00092E82200002529462268501C2060137004
:1003D0002046F9F7EFFA29462046F9F7EBFA404BA9
:1003E0002046D968F9F7E6FA00212046F9F7F9FA2C
:1003F000FEF73FBF00231B7AFFDE23685A1C2260F2
:10040000197029882046F9F7ECFA2368EA78591C14
:1004100021601A7023682A79591C21601A70236898
:10042000AA79591C21601A7023686A79591C2160C5
:100430001A70FFF720BA5A1CC8F800201A780A2A46
:1004400000F080824FF0FF352B46FEF7EFBE1A46D4
:10045000591CC8F80010234D12F8021B6970C8F827
:1004600000205A782A70DA1CC8F800209B78AB70FC
:100470004046F9F766FAD8F80030E880591C1A4669
:10048000C8F8001012F8021B2971C8F800205B7828
:100490006B71D7E75A1CC8F800201B780A2B00F0B4
:1004A000A881502BCED14046F9F74BFA0E4E308042
:1004B0004046F9F746FA4FF0FF3570802B46FEF7BD
:1004C000B5BE00BF0C9C002024210020C4400020A9
:1004D000F2790020D4220020107900208C26002000
:1004E00070230020401F0020E4290020D8F80430A9
:1004F000D8F8005040465D1BF9F70CFA052D06466A
:1005000000F23F8180252F464FF0010894E80C004F
:100510009B1A103BDFF82494AB42B8BF9FB2D9F8C6
:100520000C309B1B9F423146204688BF9FB2F9F793
:1005300041FAB8F1000F00F06181D9F80C30D4F81D
:100540000080F2199A4200F20E82F9F78FFF4146BD
:100550003A463046FAF70AF82368A8420344236073
:10056000B8BF002102DBFEF77CBE236801305A1CB5
:10057000A84222601970F8D1FEF773BEDFF8C0A35D
:100580004FF000084FF0080908F10108B8F1240FF6
:100590001BD0C8F1200209FA02F22AFA08F6A8F1E3
:1005A0002003164329FA03F31E4306F00102002339
:1005B0001343E9D05FFA88F021F0A4FD0028E3D0CE
:1005C000414604A8F9F78EFDDEE7CB4B1B78DB072D
:1005D00000F132810026C94FB04602E00136242ED8
:1005E0000ED031463846F9F78CFD0028F6D031465A
:1005F00004A8F9F786FD002854D108F10108EDE7B9
:10060000BF4BC04EB3F850102046F9F7EAF900216D
:100610002046F9F7E6F9BC4B1A68530103F02001B4
:10062000C2F340030B43C2F3800143EA4103C2F328
:10063000C00143EA8103C2F3401143EAC10102F061
:10064000100211432046F9F7CCF902A904222046F2
:10065000F9F782F923683178AC4A581C2060197088
:1006600011886429A8BF64212046F9F7BAF9962DAC
:1006700000F0E78000212046F9F7B3F92168B8F1CE
:10068000190348BFA8F11203A3F3C4034A1C226054
:1006900020460B701A4603A90125F9F75DF92B4690
:1006A000FEF7C4BD414602A8F9F71CFDA5E7D8F83E
:1006B0000030D8F804209A4240F0F3808F4BFF229C
:1006C0001A724FF00008924D0BF070F8414630223C
:1006D000904885F8008028F060FC8DF810809DF827
:1006E00010300B2B00F245818B4F8A4E42469DF80D
:1006F000103003EB430307EBC3035B7CE3B19DF8CE
:10070000103003EB430307EBC3035B69A3B19DF810
:10071000103003EB430307EBC3032021586946F86D
:100720002200F8F78CF92B7856F82300F8F743FAF3
:100730002A780132D2B22A709DF810300133DBB230
:100740008DF810309DF810300B2BD0D92368591C30
:1007500021601A70B9F1000F3EF483AD6F4BC9F8F8
:10076000003001252B46FEF761BD2368B1786C4A45
:10077000581C2060197023681278591C21601A7067
:1007800078E54046F9F7DDF84FF0000807460546E2
:10079000BCE6D9F8003013F48053B4EEE88A5FD099
:1007A000F1EE10FA11DBB4EEC98AF1EE10FA5BD863
:1007B000DFED5C7A9FED5C7A77EEC87AB4EEC78A9B
:1007C000F1EE10FAB0EE678A4ED94FF47A71B5EEB9
:1007D000408AF1EE10FA40F2DC5308BF1946FFF7E9
:1007E000FDBB22680125531923602B461070FEF7CC
:1007F0001DBD4046F9F7A5F84C4E58E6394620464F
:10080000F9F7EFF823685A1C226083F80080D9F8C2
:100810000C50D4F80080F219954280F0AC80AD1BEA
:10082000F9F724FE2A4641463046F9F79FFE236831
:1008300003442360FEF715BD049B43F001030493BA
:10084000C8E623680322591C21601A702368727855
:10085000591C21601A7011E7354A92E82200B3E56D
:10086000F1EE10FAC0F28180F7EE007A78EE677A46
:10087000B6EE007AF0EE696AE7EE876A40F2E93296
:10088000FDEEE67A17EE901AB1F5FA6FA8BF4FF4B5
:10089000FA619142B8BF114689B2002B3FF49EAB7A
:1008A00095E75A1C1946C8F80020144811F8022B85
:1008B0000272C8F800105B784372042A03D9FF2A39
:1008C0007EF4DBACFDE61B490978994205D8022A83
:1008D0007EF4D3ACFF2B7EF4D0AC236801255A19EB
:1008E00022601D70B9F1000F3EF4BBAC124BC9F889
:1008F00000302B46FEF79ABC6F3D0020702300208D
:10090000DC170020CA790020BC8D0020AE26002014
:10091000237300203C780020489200200940020800
:10092000248D002000C0884400C08244208D002017
:1009300060210020859400202D5C01083C080020E7
:1009400090E33FF49A1CC8F80020124A59781170BD
:10095000D91CC8F8001099785170191DC8F80010FA
:10096000DB7893706EE59F1BEFE54FF47A71FFF72C
:1009700035BB4246EAE6F9F779FD3A46414630464C
:10098000F9F7F4FD23680125034423602B46FEF7A5
:100990004DBC00BF675200202DE9F04FDFF80CB1CD
:1009A0002DED0C8B9BF800309DB0012B099002F0CF
:1009B0007383394C94F80021002A41F06B83072B94
:1009C000364D02F0E982002306936B68334898475E
:1009D00000286DD0B5F8A870002285F84920002FB6
:1009E00040F09B82B5F92460E96AB5F926002A6BCC
:1009F000B5F92830711AA96329490591821A686BE3
:100A0000EA630E461B1A95F84A1026482B641CF020
:100A10001BFC336813F0005302F0E282D5ED0F5A4D
:100A2000D5ED0E7A204A94ED676AD4ED686A94EDAC
:100A3000697AD4F8A8311268B8EEE58AD5ED105A73
:100A4000F8EEE77AF8EEE58A013377EE867A38EE4B
:100A5000268A78EE878A9342C4ED677A84ED688AA5
:100A6000C4ED698AC4F8A83101F066869BF800706D
:100A7000142F03F07982D4F8B0614FF0000A062EEB
:100A800002F28483DFE816F07618F2192113071AB0
:100A90003A1904187D1700BF80230020209C0020F5
:100AA000C8450020589C0020C08D0020959400204F
:100AB0009BF80090B9F1070F00F0E88294F8C0317C
:100AC000002B40F0F082D44B5B79002B40F0208269
:100AD00001239BF8002084F8C031072A02F0138418
:100AE00000230D93CD4B94ED72AA93ED007ACC4A7E
:100AF000DFF8A8A31268CB4BDFF8A4830692F7EEC9
:100B0000007A77EECA8AC84A0A9368EE878A079203
:100B1000F4EEE78AC54A059300255346F1EE10FA34
:100B200094ED719ADFF87C939FEDC1BADFEDC19A25
:100B3000DFEDC1BADFEDC1CADFEDC1AA9FEDC1CAC9
:100B4000C14F0892C24688BFF0EE678A2E4698468B
:100B5000BE4B2B44D3ED007ABD4BF5EE407A2B44CF
:100B6000F1EE10FA93ED008A17D0BA4B2B4493EDB7
:100B7000007A78EE476AB0EEE66AF4EEC67AF1EEF5
:100B800010FA08D5F5EEC06AF1EE10FACCBF37EED8
:100B9000878A37EE678A83ED008A079BB3F800E007
:100BA0001EF0030F00F08782022E04F0868706995C
:100BB000A94B91F8322006EE902A33F916202B44E7
:100BC00007EE102A13ED096A91F83130B8EEC77AB2
:100BD000F8EEE66A5A4207EE902AA6EE867A71008F
:100BE000F8EEE77AB4EEE77AF1EE10FA0AD407EEFF
:100BF000903AF8EE677AF4EEC77AF1EE10FA88BF11
:100C0000F0EE477A954B0B93954A0B44515EB3F93E
:100C10000A30C81A07EE100AB8EEC77A1EF0010FA4
:100C2000E7EE697A00F09782DFF87CE29EED008AB9
:100C300027EE888A94F8D8E1BEF1000F1FD0DFF8C4
:100C400068E2D4F8DC01DEED007ADFF860E25B1ADE
:100C500007EE103A099BDEF8001067EEA97AB8EEAD
:100C6000C78A1B1A8B4228EE278A01F3E681F7EE2A
:100C7000007AB4EEE7AAF1EE10FA01F1A981794BFE
:100C80002B44D3ED007A059BD3ED01DA69EE277A88
:100C900038EE6DDA67EE8D7AC8ED007A089BD9EDF3
:100CA000007A93ED007A704BD7ED006A67EE277AF1
:100CB0002B4427EEA87AD3ED007A67EE277AB0EEC0
:100CC000667AADEE277AF0EE477A94ED726AB7EE67
:100CD000007AB4EEC76AF1EE10FAACBF012300232C
:100CE00043B1F0EEE66AB0EEE77AB4EEE67AF1EE02
:100CF00010FA01D5C7ED007A022E04F0B9865B4ADE
:100D00005B4B52F826001B68B0EE6D0A9847594AB3
:100D1000594B52F826001B689847069B93F83A30C7
:100D2000632B04D8079B1B88002B01F09881B0EE41
:100D30006C8A524BD9ED007A38EE400A2B4493ED81
:100D4000008A83ED000A069B30EE480A93F848209B
:100D500080EE278ADAB1F7EE007AB4EEE7AAF1EE78
:100D600010FA14DB464BD3ED007AB0EEC87AB4EE3D
:100D7000E77AF1EE10FA0ADD424BD3ED007AB0EEDD
:100D8000CDDAB4EEE7DAF1EE10FA01F380823E4BF1
:100D900094F8E8212B44D3ED007A69EE277A27EE08
:100DA000888A8AED008A2AB9C8ED00CAC7ED00CA50
:100DB000CAED00CA059B043504330C2D06F101066B
:100DC0000AF1040A08F1040807F1040705937FF407
:100DD000BFAE9BF80030072B02F0EE81012B02F032
:100DE000978200230593294A0D4B11681B6893F8DD
:100DF0002F0011F48053069300F05A82DFF8B0E020
:100E0000234D9EF80030234EED8896ED037A13F0C3
:100E1000010F214B1A8B4DE00C9C002044760020E2
:100E20002421002044A40020202100209400002040
:100E300000009642CDCCCC3DAE47813F0000000083
:100E40000000C842610BB63B0881002038760020C4
:100E5000842400204C25002010250020308D002007
:100E6000381F0020F475002000760020BC8200208E
:100E7000B8820020208300201C83002060250020F1
:100E800058760020547600200C760020C8450020BB
:100E9000948800206495002098450020FC80002064
:100EA00014810020F0750020207600204876002074
:100EB0006F3D002008BFA4F8F021561B07EE906A92
:100EC000F8EEE77AB4EEE77AF1EE10FA42F29481A6
:100ED000571906EE907AF8EEE66AB4EEE67AF1EE8D
:100EE00010FA81F2FD83B4F8F021964283F28186F4
:100EF000DB4ADC4DD2ED004AD5ED003ADA4AC4EDCA
:100F00007D3AC4ED7E4AD2ED006ADFEDD87AE9E1A0
:100F1000D74B1B78013BDBB2DBE5D64BD6490A93B6
:100F200091F801A01B68DFF874839BF80090B8F972
:100F300006004FF47A71B1FBF3F3C3EB431603EBF6
:100F40008603DE00B6B2B74203F09480E96FB5F9CC
:100F500024E02B6E4A1C07EE90EA7344012AEA67EC
:100F60002B66F8EEE77A03F08F80D5ED1B5AD5EDAE
:100F70001D6A07EE102A37EEE56AB8EEC75A012F50
:100F800086EE057A37EE257A77EEC77A85ED1C7AFC
:100F9000E7EE866A85ED1B7AF0EE667AC5ED1E6A8D
:100FA000C5ED1D6A03F08386D5F89010B5F926E0EB
:100FB0006B6E4A1C07EE90EA7344012AC5F8902034
:100FC0006B66F8EEE77A03F07780D5ED205AD5ED21
:100FD000226A07EE102A37EEE56AB8EEC75A012FEB
:100FE00086EE057A37EE257A77EEC77A85ED217A97
:100FF000E6EE276A85ED207AF0EE667AC5ED236A83
:10100000C5ED226A03F08986D5F8A410B5F928E069
:10101000AB6E4A1C07EE90EA7344012AC5F8A4207F
:10102000AB66F8EEE77A03F06080D5ED255AD5ED92
:10103000276A07EE102A37EEE56AB8EEC75A012F85
:1010400086EE057A37EE257A77EEC77A85ED267A31
:10105000E6EE276A85ED257AF0EE667AC5ED286A18
:10106000C5ED276A03F04C86A8F80600B5F8A8304D
:101070009BF80090013BA5F8A8300A990023B9F12C
:10108000070F4B608B60CB607FF418ADFDF78CFBD6
:10109000069BDFF80882C01A94F8C031A8F8000057
:1010A000002B3FF410AD013B84F8C0311DB0BDEC06
:1010B0000C8BBDE8F08F94F8D83163B1022E04F0A8
:1010C000FF846E4B0B936E4A03EB460332F9161006
:1010D000B3F90A30B3E56B4B2B4493ED000A059B43
:1010E000D3ED01DA29EE000A38EE6DDA022E20EE99
:1010F0000D0A88ED000A7FF4D1AD634A634B106896
:101100001B689847089BD9ED007A93ED007A604BF5
:10111000D7ED006A1A785F4B83ED020A5E4B67EEEB
:10112000277A2B4467EEA87A93ED006A67EE867AF9
:10113000B0EE667AADEE277A012AF0EE477A02D059
:10114000192A7FF4C2ADB4EECBDAF1EE10FACCBFBF
:1011500001230023C4E5B2F900C0D4ED5E6A94ED2A
:101160005F7AB2F902000C908CEAEC70B4EEE67A89
:10117000A0EBEC70F1EE10FA0E900C984BBFB7EEAE
:10118000007AF7EE006A77EE665A76EEC75A0028C4
:10119000B8BF40420F900E9886460F98864541F39F
:1011A0003480BCF1000FD6BFCCF1000007EE10CAAE
:1011B00007EE100ADFF8E8E0B8EEC77A9EF800E024
:1011C00027EE297ABEF1000F01F03180DFF8D4E07C
:1011D0009EED005AB5EEC05AF1EE10FA41F3718758
:1011E000DFF8C4E0DEED004AF5EEC04AF1EE10FA99
:1011F00041F3678734EEC77AB7EE006AC7EE246A18
:1012000075EEC65AF4EEC66A65EEAA5AF1EE10FA09
:1012100085EE857A88BFF0EE466AF5EEC06AF1EE9B
:1012200010FA37EE067AB8BFF0EE6C6A66EE876A9F
:10123000F4EEC66AF1EE10FA88BFF0EE466AF5EEFB
:10124000C06AF1EE10FAB8BFF0EE6C6ADFF85CE04D
:101250009EED007A67EE877AA7EEA68AEAE400BFE1
:101260008C880020148D0020A4880020000000003D
:10127000248D002044A400200C9C0020308D0020F0
:10128000381F0020F47500208087002094870020FC
:1012900084740020FC8000200076002098940020B8
:1012A0002C7600202876002030760020247600203E
:1012B000E14BE24A5D8B92ED037AE14ADFF8B4E359
:1012C000D2ED003ADF4AC4ED7D3A07EE905ADE4D8A
:1012D000D2ED006AD5ED004AF8EEE77AC4ED7E4A19
:1012E00077EE677AC7EEA65AD84DD94A95ED005ADF
:1012F000D84D9FEDD97A95ED003AD84D9FEDD86A3B
:1013000095ED004AD2ED006AF7EE007AF4EEE75A66
:1013100035EE035AF1EE10FA88BFF0EE675A35EE5B
:10132000045AF4EEC75AF1EE10FA25EE065AB8BF89
:10133000F0EE475AB1EE667A33EEE43AB4EEC75AAD
:10134000F1EE10FAC4ED7F5A84ED813A00F1738416
:10135000B4EEE65AF1EE10FA88BFB0EE665ABB4A18
:101360009FEDBF6AD2ED017ABA4AD2ED012ABB4A9B
:1013700077EEA27A92ED014A77EE847A67EE867A6A
:10138000B4EEE77AF1EE10FA08DCF4EEE76AF1EE7B
:1013900010FA8CBFB0EE677AB0EE667AAB4A9FED7A
:1013A000B06AD2ED027AAB4A92ED024AAD4A77EECC
:1013B000847AD2ED006A67EE867AB1EE664AF4EE80
:1013C000C47AF1EE10FA08D4F4EEE67AF1EE10FAEF
:1013D0008CBFB0EE664AB0EE674A002841F0398211
:1013E000B7EE002AA04AA14E527894F80802002ACB
:1013F000FFEE002AB7EE006A327814BFF0EE467AAC
:10140000F0EE627A002814BFF0EE626AF0EE466AEF
:10141000002A02F0FB86B4EEC62AF1EE10FA24EEA2
:10142000274A934841F35E8290ED026A90ED011ADB
:10143000D0ED037ADFED881A27EE066A62EE262ADF
:10144000A5EE016AA7EE846A26EE226AB4EEE16A8E
:10145000F1EE10FAB4BFF0EE617AF0EE467A8DED5F
:10146000106A88BFB0EE616A012A00F0BD81D0ED3C
:10147000066AD0ED051A90ED072A67EE266AE5EEBA
:10148000216AE2EE046A66EEA26AF4EEC66AF1EE42
:1014900010FAF4EEE76A8CBFB0EE462AB0EE662A88
:1014A000F1EE10FA98BFB0EE426AA8BFF0EE667A8D
:1014B000022ACDED116A00F09781D0ED0A6AD0EDD5
:1014C000091A90ED0B2A67EE266AE5EE216AE2EE34
:1014D000046A66EEA26AF4EEC66AF1EE10FAF4EE61
:1014E000E76A8CBFB0EE462AB0EE662AF1EE10FA3B
:1014F00098BFB0EE426AA8BFF0EE667A032ACDED3F
:10150000126A00F07181D0ED0E6AD0ED0D1A90EDE7
:101510000F2A67EE266AE5EE216AE2EE046A66EEBD
:10152000A26AF4EEC66AF1EE10FAF4EEE76A8CBF36
:10153000B0EE462AB0EE662AF1EE10FA98BFB0EE91
:10154000426AA8BFF0EE667A042ACDED136A00F075
:101550004B81D0ED126AD0ED111A90ED132A67EE8F
:10156000266AE5EE216AE2EE046A66EEA26AF4EE0D
:10157000C66AF1EE10FAF4EEE76A8CBFB0EE462AC6
:10158000B0EE662AF1EE10FA98BFB0EE426AA8BF3C
:10159000F0EE667A052ACDED146A00F02581D0EDD3
:1015A000166AD0ED151A90ED172A67EE266AE5EE59
:1015B000216AE2EE046A66EEA26AF4EEC66AF1EE11
:1015C00010FAF4EEE76A8CBFB0EE462AB0EE662A57
:1015D000F1EE10FA98BFB0EE426AA8BFF0EE667A5C
:1015E000062ACDED156A00F0FF80D0ED1A6AD0ED25
:1015F000191A90ED1B2A67EE266AE5EE216AE2EEE3
:10160000046A66EEA26AF4EEC66AF1EE10FAF4EE2F
:10161000E76A8CBFB0EE462AB0EE662AF1EE10FA09
:1016200098BFB0EE426AA8BFF0EE667A072ACDED09
:10163000166A00F0D9801FE09845002064950020CC
:10164000148D00209C880020848B0020FC800020CA
:101650005C7600200881002000000000148100203A
:101660006F12833A607600200423002085940020C6
:10167000CC8700206F3D0020D0ED1E6AD0ED1D1AF2
:1016800090ED1F2A67EE266AE5EE216AE2EE046A13
:1016900066EEA26AF4EEC66AF1EE10FAF4EEE76ABC
:1016A0008CBFB0EE462AB0EE662AF1EE10FA98BF73
:1016B000B0EE426AA8BFF0EE667A082ACDED176A4E
:1016C00000F09280D0ED226AD0ED211A90ED232A0D
:1016D00067EE266AE5EE216AE2EE046A66EEA26A29
:1016E000F4EEC66AF1EE10FAF4EEE76A8CBFB0EEE3
:1016F000462AB0EE662AF1EE10FA98BFB0EE426AC2
:10170000A8BFF0EE667A092ACDED186A6CD0D0ED4C
:10171000266AD0ED251A90ED272A67EE266AE5EEB7
:10172000216AE2EE046A66EEA26AF4EEC66AF1EE9F
:1017300010FAF4EEE76A8CBFB0EE462AB0EE662AE5
:10174000F1EE10FA98BFB0EE426AA8BFF0EE667AEA
:101750000A2ACDED196A47D0D0ED2A6AD0ED291AB0
:1017600090ED2B2A67EE266AE5EE216AE2EE046A26
:1017700066EEA26AF4EEC66AF1EE10FAF4EEE76ADB
:101780008CBFB0EE462AB0EE662AF1EE10FA98BF92
:10179000B0EE426AA8BFF0EE667A0B2ACDED1A6A67
:1017A00022D0D0ED2E1A90ED2D2AD0ED2F6A27EE03
:1017B000217AA2EE057AA6EE847A27EE227AB4EE9A
:1017C000C67AF1EE10FAB4EEE77A8CBFF0EE466A14
:1017D000F0EE476AF1EE10FA8DED1B7AD8BFB0EE4D
:1017E000666AA8BFF0EE477A77EEC67AF7EE006A2F
:1017F000F4EEE67AF1EE10FAC4ED727A43F3E28188
:1018000086EEA77A012ADDED107A67EE877ACDEDB4
:10181000107A55D0DDED117A67EE877A022ACDED88
:10182000117A4DD0DDED127A67EE877A032ACDED7D
:10183000127A45D0DDED137A67EE877A042ACDED72
:10184000137A3DD0DDED147A67EE877A052ACDED67
:10185000147A35D0DDED157A67EE877A062ACDED5C
:10186000157A2DD0DDED167A67EE877A072ACDED51
:10187000167A25D0DDED177A67EE877A082ACDED46
:10188000177A1DD0DDED187A67EE877A092ACDED3B
:10189000187A15D0DDED197A67EE877A0A2ACDED30
:1018A000197A0DD0DDED1A7A67EE877A0B2ACDED25
:1018B0001A7A05D0DDED1B7A27EE877A8DED1B7A3B
:1018C000DF48006810F0805000F09A84F6EE005A6D
:1018D000C4ED7F5A002A02F0B4849EF80050DFF86D
:1018E0007493DFF87483DFF874A3DFF874E394F87B
:1018F00000C25B8B0793FDEEE37AD9ED006A9AF89C
:1019000003A0B8F906909EF800E005F0010301F08D
:10191000100817EE905A01F48001BCF1000F40F05E
:10192000A181B8F1000F00F06E85002B43F0F98023
:10193000BAF1000F43F08481C248DDED107A90EDDA
:10194000007AC149E7EE257ABDEEE47A17EE103A47
:10195000B0EE647AA3EE277AFDEEC77A17EE90EA2E
:1019600017EE907AAE45A8BF2F467345C8BF1F46F5
:1019700007EE907AF8EEE77A012AC1ED007A00F0DE
:101980004D8190ED047ADDED117AE7EE257AB0EE27
:10199000647AA3EE277AFDEEC77A17EE90EA17EE87
:1019A000907AAE45A8BF2F469E45B8BF1F4607EEAA
:1019B000907AF8EEE77A022AC1ED017A00F02E81E2
:1019C00090ED087ADDED127AE7EE257AB0EE647AD2
:1019D000A3EE277AFDEEC77A17EE90EA17EE907A1B
:1019E000AE45A8BF2F469E45B8BF1F4607EE907A6A
:1019F000F8EEE77A032AC1ED027A00F00F8190ED4C
:101A00000C7ADDED137AE7EE257AB0EE647AA3EE78
:101A1000277AFDEEC77A17EE90EA17EE907AAE4578
:101A2000A8BF2F469E45B8BF1F4607EE907AF8EE36
:101A3000E77A042AC1ED037A00F0F08090ED107A85
:101A4000DDED147AE7EE257AB0EE647AA3EE277A1C
:101A5000FDEEC77A17EE90EA17EE907AAE45A8BF72
:101A60002F469E45B8BF1F4607EE907AF8EEE77AFC
:101A7000052AC1ED047A00F0D18090ED147ADDEDF5
:101A8000157AE7EE257AB0EE647AA3EE277AFDEEBA
:101A9000C77A17EE90EA17EE907AAE45A8BF2F46A8
:101AA0009E45B8BF1F4607EE907AF8EEE77A062A01
:101AB000C1ED057A00F0B28090ED187ADDED167A6E
:101AC000E7EE257AB0EE647AA3EE277AFDEEC77AC8
:101AD00017EE90EA17EE907AAE45A8BF2F469E45C6
:101AE000B8BF1F4607EE907AF8EEE77A072AC1EDF5
:101AF000067A00F0938090ED1C7ADDED177AE7EE20
:101B0000257AB0EE647AA3EE277AFDEEC77A17EE57
:101B100090EA17EE907AAE45A8BF2F469E45B8BF13
:101B20001F4607EE907AF8EEE77A082AC1ED077AA9
:101B300074D090ED207ADDED187AE7EE257AB0EEDC
:101B4000647AA3EE277AFDEEC77A17EE90EA17EED5
:101B5000907AAE45A8BF2F469E45B8BF1F4607EEF8
:101B6000907AF8EEE77A092AC1ED087A56D090ED1E
:101B7000247ADDED197AE7EE257AB0EE647AA3EEE9
:101B8000277AFDEEC77A17EE90EA17EE907AAE4507
:101B9000A8BF2F469E45B8BF1F4607EE907AF8EEC5
:101BA000E77A0A2AC1ED097A38D090ED287ADDED7E
:101BB0001A7AE7EE257AB0EE647AA3EE277AFDEE84
:101BC000C77A17EE90EA17EE907AAE45A8BF2F4677
:101BD0009E45B8BF1F4607EE907AF8EEE77A0B2ACB
:101BE000C1ED0A7A1AD090ED2C7ADDED1B7AE7EE82
:101BF000257AE3EE274AFDEEE47A17EE900A854255
:101C0000A8BF05468342D8BF2B4607EE903AF8EEB0
:101C1000E77AC1ED0B7A002A00F0A68192000B4909
:101C2000094824F03BFF0A4B1B68002B00F0A18100
:101C300012F02CFD9DE1B0EE475AFFF790BB00BFBC
:101C4000F48C0020CC870020308100209C8700206D
:101C5000EC75002098870020E02200203821002029
:101C6000EC400020B8F1000F40F07283D248DDED67
:101C7000107A90ED007AD149E7EE257AB1EE433A39
:101C8000B0EE637AA3EE277AF0EE477ABEF1000F4A
:101C900041F07E83BAF1000F43F0CD82BDEEE47ACD
:101CA000FDEEE77A17EE107A17EE90CA17EE90EA7B
:101CB000AC45A8BFAE466745C8BFBE4607EE90EA32
:101CC000F8EEE77A012AC1ED007A00F04A8190ED42
:101CD000047ADDED117AE7EE257AB0EE637AA3EEB1
:101CE000277AFDEEC77A17EE90CA17EE90EAAC4558
:101CF000A8BFAE46BC45B8BFBE4607EE90EAF8EEB8
:101D0000E77A022AC1ED017A00F02B8190ED087A82
:101D1000DDED127AE7EE257AB0EE637AA3EE277A4C
:101D2000FDEEC77A17EE90CA17EE90EAAC45A8BF51
:101D3000AE46BC45B8BFBE4607EE90EAF8EEE77A7D
:101D4000032AC1ED027A00F00C8190ED0C7ADDEDF2
:101D5000137AE7EE257AB0EE637AA3EE277AFDEEEA
:101D6000C77A17EE90CA17EE90EAAC45A8BFAE4608
:101D7000BC45B8BFBE4607EE90EAF8EEE77A042A03
:101D8000C1ED037A00F0ED8090ED107ADDED147A6C
:101D9000E7EE257AB0EE637AA3EE277AFDEEC77AF6
:101DA00017EE90CA17EE90EAAC45A8BFAE46BC4508
:101DB000B8BFBE4607EE90EAF8EEE77A052AC1ED15
:101DC000047A00F0CE8090ED147ADDED157AE7EE1E
:101DD000257AB0EE637AA3EE277AFDEEC77A17EE86
:101DE00090CA17EE90EAAC45A8BFAE46BC45B8BF56
:101DF000BE4607EE90EAF8EEE77A062AC1ED057ACC
:101E000000F0AF8090ED187ADDED167AE7EE257AD6
:101E1000B0EE637AA3EE277AFDEEC77A17EE90CA8A
:101E200017EE90EAAC45A8BFAE46BC45B8BFBE466B
:101E300007EE90EAF8EEE77A072AC1ED067A00F09D
:101E4000908090ED1C7ADDED177AE7EE257AB0EE02
:101E5000637AA3EE277AFDEEC77A17EE90CA17EEE3
:101E600090EAAC45A8BFAE46BC45B8BFBE4607EE3B
:101E700090EAF8EEE77A082AC1ED077A71D090ED82
:101E8000207ADDED187AE7EE257AB0EE637AA3EEDC
:101E9000277AFDEEC77A17EE90CA17EE90EAAC45A6
:101EA000A8BFAE46BC45B8BFBE4607EE90EAF8EE06
:101EB000E77A092AC1ED087A53D090ED247ADDED56
:101EC000197AE7EE257AB0EE637AA3EE277AFDEE73
:101ED000C77A17EE90CA17EE90EAAC45A8BFAE4697
:101EE000BC45B8BFBE4607EE90EAF8EEE77A0A2A8C
:101EF000C1ED097A35D090ED287ADDED1A7AE7EE5A
:101F0000257AB0EE637AA3EE277AFDEEC77A17EE54
:101F100090CA17EE90EAAC45A8BFAE46BC45B8BF24
:101F2000BE4607EE90EAF8EEE77A0B2AC1ED0A7A90
:101F300017D090ED2C7ADDED1B7AE7EE257AE3EEF3
:101F4000273AFDEEE37A17EE900A8542A8BF0546D0
:101F50008742D8BF2F4607EE907AF8EEE77AC1EDB8
:101F60000B7A002B3FF457AE154B1B68002B7FF408
:101F70005FAE144B1B7893B1307868B10F4FDFF828
:101F80004C800025E8B2D8F80030B7EC010A984739
:101F9000307801358542F5DB0B4B1B6898479BF881
:101FA0000030072B01F01D81012384F800311DB0A2
:101FB000BDEC0C8BBDE8F08FCC8700203081002079
:101FC000EC75002054450020E8400020E04000204F
:101FD0000B9BB2F900E0B3F90A30C749AEEB03003E
:101FE000096880EAE073A3EBE0738B42BEF647AE6C
:101FF000B2F902300B9AB2F90C209A1A82EAE27313
:10200000A3EBE27399427EF73AAE0A99BB4BD1ED4E
:10201000017A93ED007AF0EEE77AF4EEC77AF1EE0A
:1020200010FA7EF52CAED1ED027AF0EEE77AB4EE3E
:10203000E77AF1EE10FA7EF722AEB14B1A88002350
:1020400084F8D831002A40F06D83AE4AAE4B117847
:10205000186881F00101F6F7C7FDFEF710BEAB4B23
:10206000AB4A2B4493ED007AD2ED007AA94B67EE90
:10207000277AF7EE006AF4EEE67AF1EE10FA93EDC5
:10208000007A88BFF0EE667A67EE877A27EE888A54
:10209000FEF74FBE072B02F0908500279E4B05935D
:1020A0001B689E4D590501F1C4809D4B1B78002B88
:1020B00040F003819B4B94F8126126B19A4A128832
:1020C000920742F0C48094F81811DA7F002941F099
:1020D000BA809E7F002E00F0C785022E02F070802D
:1020E000032E01F03C84914840880232D2B200298C
:1020F00002F05980002802F056808D4E3668B0FB01
:10210000F6F006B2A4F84861002A03F01C8207EE3C
:10211000906AF8EEE77AF7EE006A86EEA77ADFF8C3
:102120002092012AD4ED576AD9ED007A77EEE67A4B
:1021300067EE877AC4ED537A21D0D9ED017AD4EDD8
:10214000586A77EEE67A022A67EE877AC4ED547A07
:1021500015D0D9ED027AD4ED596A77EEE67A032AE2
:1021600067EE877AC4ED557A09D0D9ED037AD4EDBC
:102170005A6A77EEE67A67EE877AC4ED567A9BF86C
:102180000000092803F0B882002E40F3748592B352
:10219000D4ED577A94ED537A77EE877A012AC4ED1D
:1021A000577AC9ED007A21D0D4ED587A94ED547A5B
:1021B00077EE877A022AC4ED587AC9ED017A15D0F4
:1021C000D4ED597A94ED557A77EE877A032AC4EDE7
:1021D000597AC9ED027A09D0D4ED5A7A94ED567A3B
:1021E00077EE877AC4ED5A7AC9ED037A013A022A6A
:1021F000B8BF0222D2B2002918BF022200F03CBDB3
:102200004F023FF563ABFFF765BB0C98DFF834E195
:102210000028D8BF404207EE100A9EF800E0B8EE52
:10222000C77A27EE297ABEF1000F7EF4CFAFDFF830
:1022300018E19EED006AB4EEEB6AF1EE10FA40F19F
:10224000F287B7EE005A35EE465ADFED3A6ADFF80C
:10225000FCE036EEC77A25EE0C5ADEED006AA5EEFC
:10226000076A26EE267AB5EEC07AF1EE10FA40F251
:102270002887CAEE876AB7EE006A35EEC67AF0EEB6
:10228000465AE7EE265AF0EE656AFEF7D1BF012303
:102290000999C4F8DC11022A84F8D8317EF477ADAC
:1022A000174A1288002A43F05681164A164B1178B5
:1022B0001868F6F799FCFEF76ABD1F4A194BB2F988
:1022C00006105A8B91423FF7F6AE1C4A1278012A4B
:1022D00001F05487192A01F051870E2A3FF4EBAE22
:1022E000082A3FF4E8AEDFF858900022C9F8082029
:1022F000C4F80C21DFE600BF4C76002050760020A9
:10230000C47D0020C67D0020C87D0020F824002068
:102310001C76002018760020C8450020209C002054
:10232000841B00209845002020210020D42200207A
:102330006481002000003443E022002004230020B8
:10234000649500202C76002034760020287600202A
:10235000002B42F0FD81BEF1000F41F09782FDEEAF
:10236000E47A0DF1400C17EE90EAFDEEE67A0CEB04
:1023700082030693D848DFF8649308944FFA8AF3EF
:1023800017EE907AB1EE433A8AF0010807921C46A4
:10239000034693ED007AFCEC017AE7EE257A1030E3
:1023A000B0EE637AA3EE277AFDEEC77A17EE903A85
:1023B00017EE902AAB42A8BF2A469F42CCBF00210D
:1023C0000AF00101002914BF114639469E45CCBFD1
:1023D000002308F0010307EE901A002B14BF1346E8
:1023E0007346B8EEE77A07EE903A069BF8EEE77A86
:1023F000002C18BFF0EE477A6345E9EC017AC7D1AB
:10240000079A089C07E4B448DDED107A90ED007A55
:10241000B249E7EE257ABAF1000F42F00F82BDEE25
:10242000E47A17EE107AB0EE647AA3EE277AFDEE26
:10243000C77A17EE90CA17EE90EAAC45A8BFAE4631
:102440006745C8BFBE4607EE90EAF8EEE77A012A74
:10245000C1ED007A3FF485AD90ED047ADDED117A9F
:10246000E7EE257AB0EE647AA3EE277AFDEEC77A1E
:1024700017EE90CA17EE90EAAC45A8BFAE46674586
:10248000C8BFBE4607EE90EAF8EEE77A022AC1ED31
:10249000017A3FF466AD90ED087ADDED127AE7EE51
:1024A000257AAE46B0EE647AA3EE277AFDEEC77ABF
:1024B00017EE90CA6545A8BFE6466745C8BFBE4649
:1024C00007EE90EAF8EEE77A032AC1ED027A3FF4CC
:1024D00048AD90ED0C7ADDED137AE7EE257AB0EE9B
:1024E000647AA3EE277AFDEEC77A17EE90CA17EE4C
:1024F00090EAAC45A8BFAE46BC45B8BFBE4607EEA5
:1025000090EAF8EEE77A042AC1ED037A3FF429ADA8
:1025100090ED107ADDED147AE7EE257AB0EE647A6C
:10252000A3EE277AFDEEC77A17EE90CA17EE90EA6F
:10253000AC45A8BFAE46BC45B8BFBE4607EE90EA64
:10254000F8EEE77A052AC1ED047A3FF40AAD90ED82
:10255000147ADDED157AE7EE257AB0EE647AA3EE13
:10256000277AFDEEC77A17EE90CA17EE90EAAC45CF
:10257000A8BFAE46BC45B8BFBE4607EE90EAF8EE2F
:10258000E77A062AC1ED057A3FF4EBAC90ED187AB4
:10259000DDED167AE7EE257AB0EE647AA3EE277ABF
:1025A000FDEEC77A17EE90CA17EE90EAAC45A8BFC9
:1025B000AE46BC45B8BFBE4607EE90EAF8EEE77AF5
:1025C000072AC1ED067A3FF4CCAC90ED1C7ADDED24
:1025D000177AE7EE257AB0EE647AA3EE277AFDEE5D
:1025E000C77A17EE90CA17EE90EAAC45A8BFAE4680
:1025F000BC45B8BFBE4607EE90EAF8EEE77A082A77
:10260000C1ED077A3FF4ADAC90ED207ADDED187A9C
:10261000E7EE257AB0EE647AA3EE277AFDEEC77A6C
:1026200017EE90CA17EE90EAAC45A8BFAE46BC457F
:10263000B8BFBE4607EE90EAF8EEE77A092AC1ED88
:10264000087A3FF48EAC90ED247ADDED197AE7EE4E
:10265000257AB0EE647AA3EE277AFDEEC77A17EEFC
:1026600090CA17EE90EAAC45A8BFAE46BC45B8BFCD
:10267000BE4607EE90EAF8EEE77A0A2AC1ED097A3B
:102680003FF46FAC90ED287ADDED1A7AE7EE257A0B
:10269000B0EE647AA3EE277AFDEEC77A17EE90CA01
:1026A00017EE90EAAC45A8BFAE46BC45B8BFBE46E3
:1026B00007EE90EAF8EEE77A0B2AC1ED0A7A3FF4CA
:1026C00050AC90ED2C7ADDED1B7AE7EE257AE3EE47
:1026D000274AFDEEE47A36E4CC87002030810020E2
:1026E00007EE902AF8EEE77A724EDFF8ECC1D6EDED
:1026F000004ADCED003A704EC4ED7D3A77EE677A21
:1027000006EE905ABCEEC77AF8EEE66A17EE102A8B
:1027100077EEE67AC4ED7E4AA4F8F021D6ED006AA1
:10272000FEF7E0BD65494A69002A3EF4A8AA0A6896
:1027300013604B74FEF7A3BA07EE103A9BF8003013
:10274000DFF89881C4F8A871B8EEC77AF7EE006A8E
:10275000132B86EE879AB8F90400B4F8AC6195EDB6
:10276000080A01F01284564B564A93ED001A93ED75
:10277000093A93ED162A93ED1F6AD3ED0B1A93EDE8
:10278000144AD3ED015AD3ED0A3A93ED0C7A93ED46
:10279000155AD3ED172AD3ED206AD3ED044AD3EDB1
:1027A000030A67EE897A69EE288A29EE088AA1EE83
:1027B000273A02EB86070021A2EE286AC4F89C1192
:1027C000C4F8A011A1EE884AE5EEA73AA7EE085A90
:1027D00093ED1A7AD3ED0F5A93ED021AD3ED0E1A38
:1027E00087ED003AE2EEA86A64EEC34A27EE467A25
:1027F00093ED0D2AD3ED192A87ED204AE0EEC33A76
:1028000065EEC45A93ED183AC3ED093AE1EE274A52
:10281000F0EE477AA1EEC45AE2EE085AE2EEC66A3A
:10282000E3EE287AC3ED0A4A83ED145AC3ED155A34
:1028300087ED406AC3ED1F6AC3ED207AC4F8A41186
:10284000731C03F01F03A4F8AC31A8F80400FEF7D2
:102850000DB91D4A107900283EF4C2AD1B4800781E
:1028600000283EF4BDAD1278DFED192A07EE902A5C
:10287000184AF8EE676A128807EE900A06EE102AE8
:10288000F8EEE77AB8EE466A66EEA77AF7EE006AE7
:1028900087EE862AB4EEE22AF1EE10FA88BFB0EE97
:1028A000622AB4EEE62AF1EE10FAB8BFB0EE662A5C
:1028B000FEF798BD8C880020A4880020CC7D0020E5
:1028C00080900020E48D0020401F002063950020B0
:1028D000713DAA3F3C950020148D00209894002063
:1028E0000000000090ED026A90ED012AD0ED037A1D
:1028F0005FED052A27EE066AA5EE026AA7EE846A56
:1029000026EE266AB4EEE26AF1EE10FAB4BFF0EEFB
:10291000627AF0EE467A8DED106A88BFB0EE626A98
:10292000012A3EF461AFD0ED062AD0ED051A90EDF4
:10293000072A67EE222AE5EE212AE2EE042A62EE59
:10294000A62AF4EEC62AF1EE10FAF4EEE72A8CBFBE
:10295000B0EE462AB0EE622AF1EE10FA98BFB0EE61
:10296000426AA8BFF0EE627A022ACDED112A3EF447
:102970003BAFD0ED0A2AD0ED091A90ED0B2A67EE95
:10298000222AE5EE212AE2EE042A62EEA62AF4EEDD
:10299000C62AF1EE10FAF4EEE72A8CBFB0EE462A12
:1029A000B0EE622AF1EE10FA98BFB0EE426AA8BF0C
:1029B000F0EE627A032ACDED122A3EF415AFD0ED87
:1029C0000E2AD0ED0D1A90ED0F2A67EE222AE5EEC1
:1029D000212AE2EE042A62EEA62AF4EEC62AF1EEDD
:1029E00010FAF4EEE72A8CBFB0EE462AB0EE622A67
:1029F000F1EE10FA98BFB0EE426AA8BFF0EE627A2C
:102A0000042ACDED132A3EF4EFAED0ED122AD0ED1C
:102A1000111A90ED132A67EE222AE5EE212AE2EE42
:102A2000042A62EEA62AF4EEC62AF1EE10FAF4EEBB
:102A3000E72A8CBFB0EE462AB0EE622AF1EE10FA19
:102A400098BFB0EE426AA8BFF0EE627A052ACDEDDB
:102A5000142A3EF4C9AED0ED162AD0ED151A90ED29
:102A6000172A67EE222AE5EE212AE2EE042A62EE18
:102A7000A62AF4EEC62AF1EE10FAF4EEE72A8CBF8D
:102A8000B0EE462AB0EE622AF1EE10FA98BFB0EE30
:102A9000426AA8BFF0EE627A062ACDED152A3EF40E
:102AA000A3AED0ED1A2AD0ED191A90ED1B2A67EECD
:102AB000222AE5EE212AE2EE042A62EEA62AF4EEAC
:102AC000C62AF1EE10FAF4EEE72A8CBFB0EE462AE1
:102AD000B0EE622AF1EE10FA98BFB0EE426AA8BFDB
:102AE000F0EE627A072ACDED162A3EF47DAED0EDE7
:102AF0001E2AD0ED1D1A90ED1F2A67EE222AE5EE60
:102B0000212AE2EE042A62EEA62AF4EEC62AF1EEAB
:102B100010FAF4EEE72A8CBFB0EE462AB0EE622A35
:102B2000F1EE10FA98BFB0EE426AA8BFF0EE627AFA
:102B3000082ACDED172A3EF457AED0ED222AD0ED6B
:102B4000211A90ED232A67EE222AE5EE212AE2EEF1
:102B5000042A62EEA62AF4EEC62AF1EE10FAF4EE8A
:102B6000E72A8CBFB0EE462AB0EE622AF1EE10FAE8
:102B700098BFB0EE426AA8BFF0EE627A092ACDEDA6
:102B8000182A3EF431AED0ED262AD0ED251A90ED6C
:102B9000272A67EE222AE5EE212AE2EE042A62EED7
:102BA000A62AF4EEC62AF1EE10FAF4EEE72A8CBF5C
:102BB000B0EE462AB0EE622AF1EE10FACDED192AF7
:102BC00098BFB0EE426AB8BFF0EE672A0A2A02F058
:102BD0008B84D0ED2A7AD0ED291A90ED2B2A67EE5E
:102BE000277AE5EE217AE2EE047A67EEA67AF4EE31
:102BF000C67AF1EE10FAF4EEE27A8CBFB0EE462A15
:102C0000B0EE672AF1EE10FACDED1A7A98BFB0EE69
:102C1000426AB8BFF0EE627A0B2A3EF4E5ADD0ED21
:102C20002E2AD0ED2D1A90ED2F2A67EE222AE5EEFE
:102C3000212AE4EE022A62EEA62AB4EEE26AF1EE5E
:102C400010FAF4EEE27A8CBFB0EE627AB0EE467A19
:102C5000F1EE10FACDED1B2A58BFB0EE476AB8BFAF
:102C6000F0EE627AFEF7C0BDA4F84861002900F0DA
:102C70007281DFF868930222CA49DFEDCB6A0868E7
:102C80009BF800C0017890F802E007EE901AF8EE89
:102C9000E77AB0EE007A67EEA67AF4EEC77AF1EE44
:102CA00010FA40F3A68237EEC77ADFEDC06AB0EEC5
:102CB000676AA7EE266AB0EE467A9FEDBD6AD9ED47
:102CC000006A66EE866AB0EEE66AC4ED5B6A84ED81
:102CD0005E6ABEF1000F13D005EE90EAB8EEE55A39
:102CE000DFEDB15A66EEA64A25EE255AF7EE005AF8
:102CF00075EEC55A64EE864AE5EE245A66EEA56A7C
:102D0000DFEDAC5A417927EE257A27EE267AC9B154
:102D1000DFEDA56ADFEDA85A26EE266A06EE901AC8
:102D2000F8EEE66A66EE866AF4EEE56AF1EE10FA0F
:102D300000F3A885F7EE005A75EEE66A85EEA66AFE
:102D400027EE067ABCF10C0F9FED9C8ADFED9C6AA2
:102D500000F05885B4EEC87AF1EE10FA98BFB0EEE4
:102D6000478AB4EEE68AF1EE10FAB8BFB0EE668A92
:102D700084ED418A002A00F0E280B0EE007AF4EEA1
:102D8000C77AF1EE10FA05DD37EEC77ADFED876A14
:102D9000E7EE267A99ED017ADFED856A27EE267A4D
:102DA000B0EEC76A84ED5C7A84ED5F6ABEF1000F15
:102DB00013D006EE90EADFED7C5AF8EEE66A27EED5
:102DC000075A66EEA56AF7EE005A75EEE65A25EE4A
:102DD000065AE6EE855A27EE257ADFED766A817986
:102DE00067EEA67A67EE877AA9B107EE101AB8EEF9
:102DF000C77ADFED6D5ADFED706A27EE067A27EEAF
:102E0000257AB4EEE67AF1EE10FA40F32D85DFED87
:102E10006D6A67EEA67ABCF10C0F00F0D284DFED8C
:102E2000676A9FED677AF4EEE67AF1EE10FA88BFF2
:102E3000F0EE667AF4EEC77AF1EE10FAB8BFF0EE73
:102E4000477A012AC4ED427A79DD4278DFED566A8D
:102E500007EE902AF8EEE77AB0EE007A67EEA67AEF
:102E6000427AF4EEC77AF1EE10FA05DD37EEC77A52
:102E7000DFED4E6AE7EE267A99ED027ADFED4C6AD5
:102E800027EE267AB0EEC76A84ED5D7A84ED606A3B
:102E90009AB106EE902ADFED445AF8EEE66A27EE84
:102EA000075A66EEA56AF7EE005A75EEE65A25EE69
:102EB000065AE6EE855A27EE257ADFED3E6AC2799C
:102EC00067EEA67A67EE877A0AB307EE102AB8EEA5
:102ED000C77ADFED355ADFED386A27EE067A27EE3E
:102EE000257AB4EEE67AF1EE10FA0CDCB5EEC07A93
:102EF000F1EE10FA01F14981B7EE006A36EE477A39
:102F0000C6EE076A01E0DFED2F6A67EEA67ABCF134
:102F10000C0F00F09484DFED296A9FED297AF4EE1E
:102F2000E67AF1EE10FA88BFF0EE667AF4EEC77A30
:102F3000F1EE10FAB8BFF0EE477AC4ED437ABCF177
:102F4000090F00F0328493F82160002E40F0E583F1
:102F5000002384F818311C4B1B689E0609D51B4BB7
:102F60001B8803F0300323B1194B1B78D80701F1FC
:102F7000FD86184B1B7823B9174EB378002B41F010
:102F8000A8819BF80030072B00F063840022072BF8
:102F900084F800217DF417ADFBF706FC0690FDF7E1
:102FA00014BD00BF282100200AD7233CD7A36841C5
:102FB0006F12033B00004843A4707D3F00C0F944FA
:102FC00000C0F9C40000C842BC8D002020210020B0
:102FD0004E1F00208B3F0020F279002064950020D6
:102FE000D54A0A9292460026D44FDFF86C83B14648
:102FF000B7EC018AD5ED087AB8EEC88A28EE278AA0
:10300000B9F1000F02F023857BBB9BF80010082963
:103010003BD006F5D260B0EE480A2844D5F88C368D
:10302000984706F5E360D5F81437284498479BF88D
:103030000030032BB0EE408A22D0D5F8AC30D7F860
:103040004406B0EE480A98470AEB890309F10109E2
:10305000B9F1030F06F12C0683ED010A3DF428AD0A
:10306000059B1B6803F00053C2E706F5F460B0EE61
:10307000480A2844D5F89C379847B0EE408AC4E700
:1030800023F080FE28F81900D7E7B0EE480A23F0B5
:1030900079FE28F81900BCE7A94BAA4C1A68AA4B7C
:1030A000DFF8B48294F80001D2691B88A8F80020E8
:1030B000A8F8023000287EF4F0AF0690A34DFDF78B
:1030C00084BCDFEDA36AFEF7C1B8DFF8B492D4ED9B
:1030D000017A94ED006AB9F80000D9F8143077EE5F
:1030E000A77AF0EE006AB0EE677AA6EE267A01388B
:1030F00004EBC002D6EE267A083A1033F6EE003A18
:1031000027EE237A67EEA37A84ED207AC4ED217A44
:103110008C4CA64604F1800192ED027A92ED036A8E
:10312000DEED036ADEED027A53ED014A13ED025A39
:1031300037EE674A76EEC65A77EE277AE4EE845A7F
:103140000138A2F10802E5EE047A0EF1080E03F14F
:10315000080336EE267A01F10801E4EE877AE5EEFF
:10316000475A67EEA37A25EEA37AC1ED007A81ED86
:10317000017AD1D1142F09D1FBF716FBDFF8D881E2
:10318000A0EB0A00A8F80200D4F8B0616A4B0A93D9
:10319000704A059BDDF828A01B68013682FB0612E9
:1031A0009119F217C2EBA102C2EBC202B61AC4F81F
:1031B000B06103F0005316E7FBF7F6FA9BF8003016
:1031C0000D9ADFF89481801A012BA8F8020000F014
:1031D000A180072B7DF405AEFBF7E6FA0590FDF71D
:1031E00002BEFBF7E1FA059A5B4B801AD880FEF726
:1031F000DBBEB0EE677A60E5584D594E594AD5EDC1
:10320000004AD6ED003A584D1278C4ED7D3AC4ED2F
:103210007E4AD5ED006A12B1012284F80022D4ED75
:103220007F7AFEF75FB8DFF85CE19EED007AFFF78A
:103230001AB8AB68002B3EF438AF05F144012846BC
:103240009847FEF732BF4948494ED0F8EC0036683F
:1032500044F6206E7045A8BF7046B0F57A7FB8BFBF
:103260004FF47A7016F0100F059E80B2A4F81A0180
:10327000366801F0B884F60400F17B833D4ED6F841
:1032800000C0BCF936E0DFF80091DFF80081D4F827
:103290001C61D9ED037AA8FB00084FEA9818642056
:1032A00090FBF8F01428BDEEE77A04EB4609A8BFBE
:1032B000142001368642C4F81C6117EE10AAA4BF80
:1032C0000026C4F81C6104EB4606A9F820A1B6F953
:1032D000200107EE100AB8EEC77A77EEC77AFDEE46
:1032E000E77ACDED067ABDF9186086EAE670A0EBC4
:1032F000E670704502F318811F4806464FF07E5075
:103300003060FEF7E6BEFBF74FFA0D90FDF7EABB23
:10331000DFF84480FBF748FA184AD4F8EC31126819
:103320000590C31A9A1AC4F8EC01A8F80430A8F85A
:103330000620FDF758BD00BF44A40020589C002083
:10334000648B002080230020AE260020209C0020DB
:10335000000000009324499298940020848B002060
:1033600090880020EC400020A0880020DC1700207E
:10337000F48C00202421002094000020648100208F
:10338000CC8D00202876002064950020D34D62105B
:10339000BAF1000F3EF482ACF4EEE47AF1EE10FAEA
:1033A000B8BFF0EE667AFDEEE77ABDEEE67A17EE8C
:1033B00090EA17EE90CAAE4517EE107AA8BFAC4659
:1033C0007745C8BFBC4607EE90CAF8EEE77A012AF7
:1033D000C1ED007A3EF4C5AD90ED047ADDED117AD1
:1033E000E7EE257AB0EE637AA3EE277AB4EEE47ABC
:1033F000F1EE10FAF0EE477AB8BFF0EE667AFDEE25
:10340000E77A17EE90EA17EE90CAAE45A8BFAC4631
:10341000BE45B8BFBC4607EE90CAF8EEE77A022A6E
:10342000C1ED017A3EF49DAD90ED087ADDED127AA2
:10343000E7EE257AB0EE637AA3EE277AB4EEE47A6B
:10344000F1EE10FAF0EE477AB8BFF0EE667AFDEED4
:10345000E77A17EE90EA17EE90CAAE45A8BFAC46E1
:10346000BE45B8BFBC4607EE90CAF8EEE77A032A1D
:10347000C1ED027A3EF475AD90ED0C7ADDED137A74
:10348000E7EE257AB0EE637AA3EE277AB4EEE47A1B
:10349000F1EE10FAF0EE477AB8BFF0EE667AFDEE84
:1034A000E77A17EE90EA17EE90CAAE45A8BFAC4691
:1034B000BE45B8BFBC4607EE90CAF8EEE77A042ACC
:1034C000C1ED037A3EF44DAD90ED107ADDED147A46
:1034D000E7EE257AB0EE637AA3EE277AB4EEE47ACB
:1034E000F1EE10FAF0EE477AB8BFF0EE667AFDEE34
:1034F000E77A17EE90EA17EE90CAAE45A8BFAC4641
:10350000BE45B8BFBC4607EE90CAF8EEE77A052A7A
:10351000C1ED047A3EF425AD90ED147ADDED157A17
:10352000E7EE257AB0EE637AA3EE277AB4EEE47A7A
:10353000F1EE10FAF0EE477AB8BFF0EE667AFDEEE3
:10354000E77A17EE90EA17EE90CAAE45A8BFAC46F0
:10355000BE45B8BFBC4607EE90CAF8EEE77A062A29
:10356000C1ED057A3EF4FDAC90ED187ADDED167AEA
:10357000E7EE257AB0EE637AA3EE277AB4EEE47A2A
:10358000F1EE10FAF0EE477AB8BFF0EE667AFDEE93
:10359000E77A17EE90EA17EE90CAAE45A8BFAC46A0
:1035A000BE45B8BFBC4607EE90CAF8EEE77A072AD8
:1035B000C1ED067A3EF4D5AC90ED1C7ADDED177ABC
:1035C000E7EE257AB0EE637AA3EE277AB4EEE47ADA
:1035D000F1EE10FAF0EE477AB8BFF0EE667AFDEE43
:1035E000E77A17EE90EA17EE90CAAE45A8BFAC4650
:1035F000BE45B8BFBC4607EE90CAF8EEE77A082A87
:10360000C1ED077A3EF4ADAC90ED207ADDED187A8D
:10361000E7EE257AB0EE637AA3EE277AB4EEE47A89
:10362000F1EE10FAF0EE477AB8BFF0EE667AFDEEF2
:10363000E77A17EE90EA17EE90CAAE45A8BFAC46FF
:10364000BE45B8BFBC4607EE90CAF8EEE77A092A35
:10365000C1ED087A3EF485AC90ED247ADDED197A5F
:10366000E7EE257AB0EE637AA3EE277AB4EEE47A39
:10367000F1EE10FAF0EE477AB8BFF0EE667AFDEEA2
:10368000E77A17EE90EA17EE90CAAE45A8BFAC46AF
:10369000BE45B8BFBC4607EE90CAF8EEE77A0A2AE4
:1036A000C1ED097A3EF45DAC90ED287ADDED1A7A31
:1036B000E7EE257AB0EE637AA3EE277AB4EEE47AE9
:1036C000F1EE10FAF0EE477AB8BFF0EE667AFDEE52
:1036D000E77A17EE90EA17EE90CAAE45A8BFAC465F
:1036E000BE45B8BFBC4607EE90CAF8EEE77A0B2A93
:1036F000C1ED0A7A3EF435AC90ED2C7ADDED1B7A03
:10370000E7EE257AE3EE273AF4EEE34AF1EE10FA1B
:10371000C8BFF0EE663AFEF714BC1E21CD48F6F79E
:10372000F0FC00283FF414ACCB4B1B885B063FF544
:103730000FAC94F88431B34241F06A87C74BD4EDA3
:10374000627A93ED017A94ED435ADFEDC55A9FED0D
:10375000C56A67EEC56A68EE277AE8EE076AE5EEA5
:10376000077AF4EEE56AF1EE10FA8CBFB0EE657AF6
:10377000B0EE667AB4EEC67AF1EE10FAF4EEE57ABF
:10378000B8BFB0EE467AF1EE10FA88BFF0EE657A77
:10379000F4EEC67AF1EE10FAB8BFF0EE467A84ED98
:1037A000417AC4ED437AFFF7D3BBFDEEC87ADFF868
:1037B000D48217EE902AA8F80460A8F80620FFF734
:1037C000C2BB9FEDA77ADFEDA76ADFF8B882F4EEFF
:1037D000C77AF1EE10FA98BFB0EE677AFDEEE77A9D
:1037E000B4EEE67AF1EE10FA17EE901AB8BFB0EE2A
:1037F000667A012A84ED427AA8F802103FF725ABD9
:10380000FFF7A1BBB4EEC87AF1EE10FA98BFB0EEA4
:10381000478ABDEEC77AB4EEE68ADFF86882F1EE39
:1038200010FA17EE101AB8BFB0EE668A84ED418A1E
:10383000A8F80010002A7FF4A0AAFFF784BBBDEE11
:10384000E77ADFF8408217EE102AA8F80420FFF785
:1038500062BBFAF7A9FFDFF82C829BF80030C01B8F
:10386000A8F80400FFF792BBB5EEC07AF1EE10FAAB
:1038700000F18F84B7EE006A36EE477AC6EE076A2B
:10388000FFF7C7BA9FED786AFFF75ABAFDEEE47A00
:1038900010A817EE90EAFDEEE67A00EB820306939D
:1038A000DFF8E491DFF8E4C108944FFA8AF317EEE9
:1038B000907AB1EE433A8AF0010807921C464B46D3
:1038C00093ED007AF0EC017AE7EE257A0AF0010335
:1038D00009F11009B0EE637AA3EE277AF4EEC74A35
:1038E000F1EE10FAD8BF0023002BF0EE477A18BF94
:1038F000B0EE667ABDEEC77AFDEEE77A17EE102AD3
:1039000017EE901AAA4217EE103AA8BF2B4697421C
:10391000CCBF00220AF00102002A08BF3B46A942A0
:1039200017EE902A07EE103AA8BF2A468E45CCBF64
:10393000002308F00103002B08BF724607EE902A0F
:10394000B8EEC77AF8EEE77A069B002C18BFF0EEC7
:10395000477A9842ECEC017AB1D1FEF751BD93F869
:103960002000C0EB401600EB8600C00080B2FEF7DE
:10397000BCBB3E4ED6F800C0BCF836E04FEA5E0E47
:1039800081E43B4BD4F8B4810A93B4F8AC91C9F10B
:103990002003D8B2374B09EB481E03EB8E0E830889
:1039A00001F0A58601331B013349344A07930EEB1E
:1039B000030C0EF1100313ED024A13ED035A13ED3D
:1039C000016A13ED047A51ED024A51ED035A51EDAB
:1039D000016A51ED047A64EE244A65EE255A66EEDA
:1039E000266A67EE277A1033634542ED024A42EDBC
:1039F000035A42ED016A42ED047A01F1100102F12D
:103A00001002D8D1079B1E49A3F11002964401EB86
:103A1000020C224410F0030309D0BEEC017AFCEC46
:103A2000017A67EE277A013BE2EC017AF5D1B9F130
:103A3000000F41F02084142F7FF4AAABFAF7B4FEF4
:103A4000DFF84080D4F8B061A0EB0A00A8F80200CB
:103A5000FFF79EBBF48C0020202100209400002062
:103A600000C0F94400C0F9C40000C842242100206D
:103A700044A40020E48D0020748F002090230020B7
:103A8000648F002098940020CC8700203081002093
:103A9000D4F8B491E74AE84B0A9203EBC9031268E1
:103AA00007929DED077A9B88DFEDE47AE44AF8EE11
:103AB000478A09EE103A643BC82BA8BFC82368EEBA
:103AC000A78AF8EE497A782BB8BF782368EEA78AE0
:103AD00007EE903A4FF02C08B0EE680A08FB092870
:103AE000B8EEE78A23F09AF9B8EEC99AF0EE409A58
:103AF000B0EE680A23F0F4F838EE097A79EE487AE5
:103B000028EE098A67EE877AB7EE006A88EE277A90
:103B1000142FF8EE007A77EE076A60EE277A89EEC6
:103B2000A67A77EE065A36EE477AC6EE256A67EE33
:103B3000A67A27EE267AC8ED006A88ED047AC8EDE9
:103B4000026AC8ED017AC8ED037A01F0FB85BD4B2E
:103B50009BF8007009F1010983FB0938A8EBE978AB
:103B600008EB48080136A9EB0808C4F8B061C4F8AE
:103B7000B4810AE7DFF8EC92B9F80070D9F804E0F4
:103B80004FEA570C4FEA8C0204EB8708FF0804EB5E
:103B9000020300F09F8010320137AB4803EB071798
:103BA000424410330EF1100608F1100151ED032AC2
:103BB00051ED043A10ED043A10ED032A51ED026A7A
:103BC00011ED016A10ED020A10ED018A12ED044AAE
:103BD00012ED035A53ED044A53ED035A13ED027AE2
:103BE00053ED017A52ED020A12ED011A73EE238AA7
:103BF00072EE221A40ED048A40ED031A70EE268A16
:103C000078EE061A40ED028A40ED011A74EE848ABD
:103C100075EE851A43ED048A43ED031A77EE208A88
:103C200077EE811A43ED028A43ED011A73EE633A8F
:103C300075EE655A16ED035A32EE623A74EE644A36
:103C400065EE631A16ED044A23EE052A64EE652A32
:103C5000E3EE041A1033BB4224EE843AA3EE842A26
:103C600000F1100006F11006A5EE853A01F11001F1
:103C700002F11002E4EE852A41ED071A01ED082A4F
:103C800002ED073A42ED082A56ED055A16ED065A9E
:103C900070EE666A38EE466A30EEC77A71EE677A81
:103CA00026EE253A65EEE63A25EE674A67EE054AC6
:103CB000E6EE053AA6EE853AA7EE254AE7EEA54AD6
:103CC00001ED063A41ED053A02ED064A42ED054A9C
:103CD0007FF46CAF1FFA8CF6724631465B4820F0D9
:103CE0001DFB3146D9F80420404620F017FB9BF815
:103CF0000030142B7FF448AAFFF73EBA544B1A78D1
:103D0000D4F8B4E14C489FED537A4FEACE0C00EB67
:103D10000C0383ED007A002A7CD04C49B0EE476A50
:103D2000F0EE476A0023F1EC017A013367EEA77ADF
:103D300005EE903AB4EEE77AF1EE10FAF8EEE55AB5
:103D4000B8BFB0EE677A934276EEA76AA7EEA56A8F
:103D5000E9D1F5EEC06A00EB0C03F1EE10FA83ED49
:103D6000007A57DDC6EE265A3B4B3C4A1288F7EEE6
:103D7000007A75EEE75AD3ED007A65EEA77AFDEE8C
:103D8000E77A17EE903A812B41F370809342A8BFF7
:103D9000134607EE903AF8EEE77A314B2C2101FBFF
:103DA0000E3393ED097AD3ED003A93ED0A6A93ED61
:103DB000014AD3ED046AD3ED034A93ED025AA3EE10
:103DC000A77AA4EE276A66EEC76AA7EE646ABDEE1C
:103DD000C77AE5EE276A17EE101A812983ED096A82
:103DE000C3ED0A6A41F33F808A42A8BF0A4607EE44
:103DF000902AF8EEE77AFCEEE77ACDED077ABDF887
:103E00001C3000EB0C029380BEF1000F02D1132F87
:103E100001F0BE83152F7FF4ADA96044DFF8488020
:103E2000838828F81E30034BD4F8B0610A93FFF75B
:103E3000AFB900BF44A40020E48F002027D4D236BD
:103E4000C0A3002056555555902300208023002004
:103E5000C68D002000000000C88D0020C48D002009
:103E6000FC8F0020CC8D002098940020DFF88493F4
:103E7000D748D9F80820B9F80C1021F0C7FE9BF8F4
:103E80000070142F01F08784D4F8B0610136C4F8B3
:103E9000B061FFF71CB9DFF8609399F800205FEA82
:103EA000920801F0E084DFF854C308F101004001FA
:103EB0000CEB000E0CF12003ACF1700113ED076A5E
:103EC00053ED056A13ED037A53ED017A53ED025A6F
:103ED00013ED084A53ED064A13ED045A26EE066A1E
:103EE00066EEA66A27EE077A67EEA77AA4EE046A62
:103EF00020337345E4EEA46A01F11001A5EE057AC2
:103F0000E5EEA57AF1EEC65AB1EEE66AF1EEC76AC1
:103F1000B1EEE77A41ED085A01ED076A41ED066A14
:103F200001ED057ACAD12038844404EB081112F05F
:103F3000030318BF0CF1080C0FD05CED017A1CEDE7
:103F4000027A67EEA77A013BE7EE077A0CF1080CDC
:103F5000B1EEE77AA1EC017AEFD1142F01F02784BA
:103F60000136C4F8B061CBE6FAF71EFC9BF800708E
:103F7000142F05BFDFF88882D4F8B061D4F8B0619F
:103F8000A8F800608246FCF77ABD924FDFF8749281
:103F900097ED004A97ED097AD7ED014A97ED0A6A45
:103FA000D7ED046A97ED035AD7ED025A67EE897A86
:103FB00009EB8603A4EE277AA4EEA76A66EEC76A29
:103FC000A5EE476AE5EEA76A27EE000A87ED096AC3
:103FD000C7ED0A6A83ED007A29EE088A22F0D2FE44
:103FE00069EE288AD7ED145AD7ED1F6A97ED0B1AA0
:103FF000D7ED161A97ED155A97ED207A97ED0C2A02
:10400000D7ED172A97ED0F6AD7ED1A7A97ED0E3A8A
:10401000D7ED0D3A97ED194AD7ED184AE1EE085A57
:10402000002209EB8603E8EEA16A00B2C4F89C21E5
:10403000A2EE085AC4F8A021C4F8A421A8EEA27ADE
:1040400026EE656A67EEE67AA3EE655AA3EE886A05
:10405000A6EEC47AE8EEA47A87ED145AC3ED205A8E
:1040600087ED156AC3ED406A87ED1F7AC7ED207AA8
:10407000FEF7E6BBB5F92430EA6207EE903A01227A
:10408000F8EEE77A2B66EA670023012FC5ED1C7A6C
:10409000C5ED1B7A6B6701F06D82B7427CF484AF8B
:1040A000B5F926306B6607EE903A00220123F8EE50
:1040B000E77A2A63C5F890300023012FC5ED217AF5
:1040C000C5ED207AC5F8883001F04182B7427CF412
:1040D0009BAFB5F92830AB6607EE903A002201237A
:1040E000F8EEE77A6A63C5F8A4300023012FC5ED26
:1040F000267AC5ED257AC5F89C307CF4B5AF9FEDE6
:10410000368AB9F1030F48D0BAF1000F09D007EE93
:1041100090AAF8EEE77AF4EEC87AF1EE10FA01F11F
:10412000C4832E4AAB6E126894F8B811A8F8060042
:1041300003EB560393FBF6F600236E63936213635F
:10414000D36221B1264B1B88002B7CF48FAF254B0B
:104150001B6813F4003304D0234B1B79002B41F070
:10416000368322491A46C85C012803F10C0301F08A
:1041700066800132152AF6D1FCF778BF1C4A927B83
:10418000002A3EF4B0A8FDF796BFF7EE006AFEF7EE
:10419000BCBEF7EE006AFEF73CBEB0EE480A22F065
:1041A000F1FD00B2B0E7B4F84861013E36B2002E2E
:1041B000A4F848617EF75AADDFF84C90FDF7E7BFF1
:1041C000B4F81A0100F57A7080B2FDF78EBF00BF17
:1041D000802300208090002000000000648B0020DD
:1041E0001E210020C0270020401F002048990308FE
:1041F00068930020CC8D0020C68D00200024002074
:1042000098940020E48D002064950020C448DFEDE0
:10421000C57A0068C4ED727A10F0805000F0028513
:10422000B7EE007A77EE677AF4EEE57AF1EE10FAFF
:1042300088BFF0EE657AF0EE675AC4ED7F7AFDF73D
:1042400049BB9EF8003003F00103FDF78ABEB64A71
:10425000DFEDB67A92ED080AB4EEE70AF1EE10FA55
:1042600041F20580069322F023FED4ED457A20EE3C
:10427000270A22F087FDB0F5617F069B01F3678076
:1042800007EE900AF8EEE76ADFEDA97A66EEA76A14
:1042900007EE906AB8EEE77AFDEEE67A17EE902A1E
:1042A0002032402A41F29B829FEDA20A069322F01F
:1042B00069FD00B207EE900A069BB8EEE77ADFF8D8
:1042C0009492D9ED037A77EE877AC9ED037AFDF7F8
:1042D000FABEDFF8848298F80020013A0D2A18D837
:1042E000DFE812F0EA012A02FB01C701AD017A0101
:1042F000630198013E010701E600DA00CF000E00DD
:104300001F2006931DF0FEFE069B10B9012288F8BF
:104310000020012B01F00580F278002A3EF431AE36
:10432000059A1268D20441F1B482834A928807EE5A
:10433000902AF8EEE77A814991ED012AD1ED022A1F
:1043400091ED033AD1ED043A91ED054AD1ED064ADB
:1043500091ED075AD1ED085A91ED096AD1ED0A6A3B
:1043600091ED0B7AB4EE672AF1EE10FAF4EE672ABB
:1043700014BF01220022F1EE10FAB4EE673A18BF22
:1043800042F00102F1EE10FAF4EE673A18BF42F083
:104390000102F1EE10FAB4EE674A18BF42F00102D2
:1043A000F1EE10FAF4EE674A18BF42F00102F1EEA6
:1043B00010FAB4EE675A18BF42F00102F1EE10FA9B
:1043C000F4EE675A18BF42F00102F1EE10FAB4EEB3
:1043D000676A18BF42F00102F1EE10FAF4EE676A64
:1043E00018BF42F00102F1EE10FAB4EE677A18BF7E
:1043F00042F00102F1EE10FA18BF42F00102002A69
:1044000041F0AE8191ED007AB4EE677AF1EE10FAE8
:1044100041F0A6814A4ED4F898113268914201F2D7
:10442000A68198F80030012B3EF4ABAD94F89421AE
:10443000002A3EF4A6AD0B2B18D801229A4040F674
:10444000030112EA010917D112F4C06F0ED0093B23
:10445000012B0BD8452015F0C9FCFF2015F0C6FC38
:10446000384815F039FC484615F0C0FC364B326828
:104470005A600B2388F80030002384F89431FEF74B
:1044800080BD012B01F017820E23132088F8003025
:1044900014F04EFBB3783CE7012B01D1F6F748F856
:1044A0000D23132088F8003014F042FBB37830E776
:1044B000254A234952680968C8328A4205D322F046
:1044C0005FF9B37800283FF424AF032B7FF41EAFCD
:1044D000DFF88890D9F8000013F0CEFB1B4B1B7857
:1044E0000022022BC9F8002001D114F049FAB37858
:1044F0000CE7174B1B78002B01F0BA811A201DF036
:1045000001FE002841F0B48194F89431002B41F071
:10451000AF81092388F800301CF0D4FBB378F8E6AB
:10452000F48C002000000080548200208FC2753C73
:10453000D06D393A00000000948800209C8700204C
:10454000EC7D002004BD0308188D00206081002050
:10455000BC81002064950020F1790020A07A002021
:104560001A201DF0CFFD0028D6D0A64B1B88002BAB
:10457000D2D1A54B4520D3F8009015F037FC0E2082
:1045800015F034FC48461CF073F8DDF824904846DA
:104590001CF06EF89D4A4FF480510A234846118062
:1045A00088F800301CF08AF8B6E715F071FB984BDC
:1045B000002105208DE80300A3F108020291532099
:1045C0001DF04EF800287FF465AF924AB378106072
:1045D000082288F800209CE615F05AFB8E4A0292C9
:1045E000A2F10C034FF007090193CDF80090A2F15E
:1045F00008030021143A47201DF032F800287FF408
:1046000049AF844B88F800904FF0FF3283E80500F3
:10461000B3787EE615F03CFB1CF06EFB00283FF4FF
:1046200039AF22F0ADF800283FF434AF774AB378C1
:104630004FF4805111800A2288F8002069E615F0B5
:1046400027FB764B002102208DE80300A3F108022E
:10465000029148201DF004F800287FF41BAF6D4A3A
:10466000B37810604FF0FF315160062288F80020C7
:104670004FE615F00DFB6A4A0292A2F10C032521C8
:1046800001930091A2F10A035021163A49201CF02F
:10469000E7FF00287FF4FEAE059B1B6813F0800245
:1046A00001F0C0815B4AB37810604FF0FF31516078
:1046B000052288F800202CE6DFF87CE19EF8003027
:1046C000D90701F1BA811F201DF01CFD00283FF41D
:1046D000E1AE0C2388F80030DCE6DFF8389115F005
:1046E000D7FA504AD9F80430126864339342BFF4C1
:1046F000D1AE402015F0A4FA00287FF4CBAED9F853
:10470000003049494FF0400A0FE0069115F06EFB6A
:104710000699D9F800300A680133013ABAF1010A62
:104720000A60C9F8003001F03281404AD35C184673
:10473000002BEAD101F030B93A4A364912684A6092
:10474000394800220A600321026088F80010E0E581
:10475000069B002B00F01586FDEEE47A10A901EB14
:10476000820217EE90CAFDEEE67A91462346524643
:1047700074462F482F4F17EE908AB1EE433A9E466B
:10478000CA4613E0FDEEC77A17EE903A634503DBA5
:10479000AB42A8BF2B46994607EE909AF8EEE77A0F
:1047A0005145E7EC017A00F1100027D090ED007A36
:1047B000F1EC017AE7EE257AE146B0EE637AA3EEFA
:1047C000277AF0EE477A002ADCD0434634B1B4EEC3
:1047D000647AF1EE10FA48BFF0EE667AFDEEE77A01
:1047E00017EE909AC14504DBA94517EE903AA8BF91
:1047F0002B4607EE903AF8EEE77AD1E77446FDF7DC
:10480000B3BB00BF688B0020788B0020128D002086
:10481000BC960308188D0020749603085896030868
:10482000AA940308EC7D00209C7A002034940308AD
:10483000CC870020308100206F3D0020BDEEE67A5D
:1048400017EE107AB0EE647AA3EE277AF0EE477A8C
:10485000BEF1000F40F02C83FDEEC77A17EE90CA30
:1048600017EE90EAAC45A8BFAE466745C8BFBE4646
:1048700007EE90EAF8EEE77A012AC1ED007A3DF4FE
:1048800070AB90ED047ADDED117AE7EE257AB0EEAB
:10489000647AA3EE277AFDEEC77A17EE90CA17EE78
:1048A00090EAAC45A8BFAE46BC45B8BFBE4607EED1
:1048B00090EAF8EEE77A022AC1ED017A3DF451ABB5
:1048C00090ED087ADDED127AE7EE257AB0EE647AA3
:1048D000A3EE277AFDEEC77A17EE90CA17EE90EA9C
:1048E000AC45A8BFAE46BC45B8BFBE4607EE90EA91
:1048F000F8EEE77A032AC1ED027A3DF432AB90ED8F
:104900000C7ADDED137AE7EE257AB0EE647AA3EE49
:10491000277AFDEEC77A17EE90CA17EE90EAAC45FB
:10492000A8BFAE46BC45B8BFBE4607EE90EAF8EE5B
:10493000E77A042AC1ED037A3DF413AB90ED107AC7
:10494000DDED147AE7EE257AB0EE647AA3EE277AED
:10495000FDEEC77A17EE90CA17EE90EAAC45A8BFF5
:10496000AE46BC45B8BFBE4607EE90EAF8EEE77A21
:10497000052AC1ED047A3DF4F4AA90ED147ADDED38
:10498000157AE7EE257AB0EE647AA3EE277AFDEE8B
:10499000C77A17EE90CA17EE90EAAC45A8BFAE46AC
:1049A000BC45B8BFBE4607EE90EAF8EEE77A062AA5
:1049B000C1ED057A3DF4D5AA90ED187ADDED167AB1
:1049C000E7EE257AB0EE647AA3EE277AFDEEC77A99
:1049D00017EE90CA17EE90EAAC45A8BFAE46BC45AC
:1049E000B8BFBE4607EE90EAF8EEE77A072AC1EDB7
:1049F000067A3DF4B6AA90ED1C7ADDED177AE7EE63
:104A0000257AB0EE647AA3EE277AFDEEC77A17EE28
:104A100090CA17EE90EAAC45A8BFAE46BC45B8BFF9
:104A2000BE4607EE90EAF8EEE77A082AC1ED077A6B
:104A30003DF497AA90ED207ADDED187AE7EE257A1D
:104A4000B0EE647AA3EE277AFDEEC77A17EE90CA2D
:104A500017EE90EAAC45A8BFAE46BC45B8BFBE460F
:104A600007EE90EAF8EEE77A092AC1ED087A3DF4FC
:104A700078AA90ED247ADDED197AE7EE257AB0EE8A
:104A8000647AA3EE277AFDEEC77A17EE90CA17EE86
:104A900090EAAC45A8BFAE46BC45B8BFBE4607EEDF
:104AA00090EAF8EEE77A0A2AC1ED097A3DF459AAAC
:104AB00090ED287ADDED1A7AE7EE257AB0EE647A89
:104AC000A3EE277AFDEEC77A17EE90CA17EE90EAAA
:104AD000AC45A8BFAE46BC45B8BFBE4607EE90EA9F
:104AE000F8EEE77A0B2AC1ED0A7A3DF43AAA90ED86
:104AF0002C7ADDED1B7AE7EE257AE3EE274AFDEE10
:104B0000E47A17EE900A8542A8BF0546B842A8BFCE
:104B10002F4607EE907AF8EEE77AC1ED0B7AFDF7B3
:104B200020BA069B002B00F08784FDEEE67A10A9E0
:104B300001EB820217EE908AFDEEE47A914623465D
:104B400052467446CB48CC4F17EE90CA9E46CA4692
:104B500014E0FDEEC77A17EE909ACC4503DCA94528
:104B60004B46A8BF2B4607EE903AF8EEE77A514540
:104B7000E7EC017A00F110003FF440AE90ED007ACE
:104B8000F1EC017AE7EE257A6346B0EE647AA7EE9F
:104B9000837AF0EE477A002ADBD034B1F4EE474A4C
:104BA000F1EE10FAC8BFF0EE667AFDEEE77A434602
:104BB00017EE909AC845D2DDD5E7F9F7F5FD07461F
:104BC000FDF76CBAAD48006810F080502AD0B6EE00
:104BD000007A67EE877AF4EEE75AF1EE10FA3FF5C5
:104BE0002AABFFF71DBB16F0805F7EF444ABFDF7E8
:104BF00070BAA34DA34EA44AD5ED004AD6ED003AB3
:104C0000A24D1278C4ED7F7AC4ED7D3AC4ED7E4AA0
:104C1000D5ED006A002A3CF465AB012284F800223D
:104C2000FCF760BB11F4800001D00020CFE7B6EEA6
:104C3000007AF4EEC75AF1EE10FAC8DCFCF74ABE6F
:104C4000FDEEE67A284610AB8A49DFF82CC217EE53
:104C5000907A754603EB82088646D1ED007AB3EC74
:104C6000017AA7EEA57A1031B0EE646AA3EE076A66
:104C700007EE907AB0EE467A35B1F4EE464AF1EEA0
:104C800010FAC8BFB0EE667ABDEEC77A17EE100A0A
:104C9000874204DC7045A8BF704607EE900AF8EE24
:104CA000E77A4345ECEC017AD7D1FCF7B4BF012A8F
:104CB00040F3608407EE101AB8EEC77AC7EE876A31
:104CC000B1EEE68AB9F1030F14D0BAF1000F09D0A2
:104CD00007EE90AAF8EEE77AF4EEC87AF1EE10FA51
:104CE00000F1E3852B6E03EB560393FBF6F3EB62C7
:104CF000FFF7D3B9B0EE480A22F044F800B2E4E777
:104D0000012A7FF7FCA907EE101AB8EEC77AC7EEA2
:104D1000876AB1EEE68AFFF7F4B9012A40F31784F7
:104D200007EE101AB8EEC77AC7EE876AB1EEE68AC8
:104D3000B9F1030F14D0BAF1000F09D007EE90AA11
:104D4000F8EEE77AB4EEE78AF1EE10FA00F3AD85FB
:104D50006B6E03EB560393FBF6F32B63FFF7B6B9C9
:104D6000B0EE480A22F00EF800B2E4E7484B494A98
:104D7000B3F90430DFED487A82FB0312DB17C3EB93
:104D8000A2031BB208EE103AB8EEC88A28EE278AB2
:104D9000B0EE480AF5F7DEF8F0EE408AB0EE480AC9
:104DA000F5F75EF83D4BD878002800F0A1833C4A27
:104DB000B4F98E11B2F9023044F250665B1AB34274
:104DC00000F3E283374EB342BCBF03F50C43A0337C
:104DD00046429E4200F3D6838342A8BF0346B2F9FF
:104DE0000020B4F98CE10B4419B2A2EB0E0344F29B
:104DF00050629342A4F88E1100F3C083294A934273
:104E0000BCBF03F50C43A0339E4203DC9842A8BF0D
:104E1000184606460EEB06031BB207EE903A07EE65
:104E2000101AF8EEE77AF8EEC76A27EEE87A60EE35
:104E3000277AA0EE267AA4F88C31E8EEA67ADFED88
:104E40001A6A27EE267A67EEA67ABDEEC77AFDEEDD
:104E5000E77A17EE102A17EE903AA4F89021A4F8FA
:104E60009231FEF786B88223FEF7CBBFDFED0F7AD3
:104E7000FEF793BFCC87002030810020F48C002007
:104E8000848B002090880020EC400020A088002027
:104E9000381F00206766666635FA8E3C2440002085
:104EA00080400020B0B9FFFFCDCCCC3D00000243D4
:104EB000B4EEE47AF1EE10FAB8BFF0EE667AFDEEE9
:104EC000E77A17EE90EA17EE90CAAE45A8BFAC4657
:104ED0007745C8BFBC4607EE90CAF8EEE77A012ACC
:104EE000C1ED007A3DF43DA890ED047ADDED117A34
:104EF000E7EE257AB0EE647AA3EE277AB4EEE47A90
:104F0000F1EE10FAF0EE477AB8BFF0EE667AFDEEF9
:104F1000E77A17EE90EA17EE90CAAE45A8BFAC4606
:104F2000BE45B8BFBC4607EE90CAF8EEE77A022A43
:104F3000C1ED017A3DF415A890ED087ADDED127A05
:104F4000E7EE257AB0EE647AA3EE277AB4EEE47A3F
:104F5000F1EE10FAF0EE477AB8BFF0EE667AFDEEA9
:104F6000E77A17EE90EA17EE90CAAE45A8BFAC46B6
:104F7000BE45B8BFBC4607EE90CAF8EEE77A032AF2
:104F8000C1ED027A3CF4EDAF90ED0C7ADDED137AD1
:104F9000E7EE257AB0EE647AA3EE277AB4EEE47AEF
:104FA000F1EE10FAF0EE477AB8BFF0EE667AFDEE59
:104FB000E77A17EE90EA17EE90CAAE45A8BFAC4666
:104FC000BE45B8BFBC4607EE90CAF8EEE77A042AA1
:104FD000C1ED037A3CF4C5AF90ED107ADDED147AA3
:104FE000E7EE257AB0EE647AA3EE277AB4EEE47A9F
:104FF000F1EE10FAF0EE477AB8BFF0EE667AFDEE09
:10500000E77A17EE90EA17EE90CAAE45A8BFAC4615
:10501000BE45B8BFBC4607EE90CAF8EEE77A052A4F
:10502000C1ED047A3CF49DAF90ED147ADDED157A74
:10503000E7EE257AB0EE647AA3EE277AB4EEE47A4E
:10504000F1EE10FAF0EE477AB8BFF0EE667AFDEEB8
:10505000E77A17EE90EA17EE90CAAE45A8BFAC46C5
:10506000BE45B8BFBC4607EE90CAF8EEE77A062AFE
:10507000C1ED057A3CF475AF90ED187ADDED167A46
:10508000E7EE257AB0EE647AA3EE277AB4EEE47AFE
:10509000F1EE10FAF0EE477AB8BFF0EE667AFDEE68
:1050A000E77A17EE90EA17EE90CAAE45A8BFAC4675
:1050B000BE45B8BFBC4607EE90CAF8EEE77A072AAD
:1050C000C1ED067A3CF44DAF90ED1C7ADDED177A18
:1050D000E7EE257AB0EE647AA3EE277AB4EEE47AAE
:1050E000F1EE10FAF0EE477AB8BFF0EE667AFDEE18
:1050F000E77A17EE90EA17EE90CAAE45A8BFAC4625
:10510000BE45B8BFBC4607EE90CAF8EEE77A082A5B
:10511000C1ED077A3CF425AF90ED207ADDED187AE9
:10512000E7EE257AB0EE647AA3EE277AB4EEE47A5D
:10513000F1EE10FAF0EE477AB8BFF0EE667AFDEEC7
:10514000E77A17EE90EA17EE90CAAE45A8BFAC46D4
:10515000BE45B8BFBC4607EE90CAF8EEE77A092A0A
:10516000C1ED087A3CF4FDAE90ED247ADDED197ABC
:10517000E7EE257AB0EE647AA3EE277AB4EEE47A0D
:10518000F1EE10FAF0EE477AB8BFF0EE667AFDEE77
:10519000E77A17EE90EA17EE90CAAE45A8BFAC4684
:1051A000BE45B8BFBC4607EE90CAF8EEE77A0A2AB9
:1051B000C1ED097A3CF4D5AE90ED287ADDED1A7A8E
:1051C000E7EE257AB0EE647AA3EE277AB4EEE47ABD
:1051D000F1EE10FAF0EE477AB8BFF0EE667AFDEE27
:1051E000E77A17EE90EA17EE90CAAE45A8BFAC4634
:1051F000BE45B8BFBC4607EE90CAF8EEE77A0B2A68
:10520000C1ED0A7A3CF4ADAE90ED2C7ADDED1B7A5F
:10521000E7EE257AB0EE647AA3EE277AF4EEC74A79
:10522000F0EE477AF1EE10FAC8BFF0EE667AFDEEC6
:10523000E77AFCF788BEBDEEE67AFCF731BDD4F81C
:10524000BC6153003EB1981801EB8000767840783D
:10525000B042BBF40BAF134401EB83010023C4F84D
:10526000BC11A4F80A32C4F80C32FBF7FFBE9FED64
:10527000D07AFFF724B8830001EB030E04EB030C94
:10528000CC4B03EBC8185FEA990300F07C83013331
:105290001B01079308EB03000EF1100108F1100346
:1052A0000CF1100213ED024A13ED035A13ED016ADB
:1052B00013ED047A51ED024A51ED035A51ED016AA2
:1052C00051ED047A64EE244A65EE255A66EE266AAC
:1052D00067EE277A1033834242ED024A42ED035AC9
:1052E00042ED016A42ED047A01F1100102F110026F
:1052F000D8D1079B103B08EB03020EEB030163447C
:1053000019F003093EF497ABB2EC017AF1EC017AA3
:1053100067EE277AB9F10109E3EC017AF4D1FEF7DF
:105320008ABBA549A54AC968126891423EF6F4AF06
:1053300098F800200C3A022A7DF623AE94F89421C6
:1053400088F80030002A3DF41CAEFFF795B807EE50
:10535000906ADFED9B6AB8EEE77A66EEA65A9FED9B
:10536000995A9FED996ADFED997AA5EE856A26EE46
:10537000A55AE5EE867AE5EE276A26EE870AFEF75D
:1053800095BFFDEEE67A10ABCDED087AFDEEE47A3E
:105390000B948F4FDFF86082CDF82490544617EEBF
:1053A00090CADDF820A00A91B1EE433A03EB8202E5
:1053B000CDF818E097ED007AF3EC017AE7EE257A64
:1053C000B0EE637AA3EE277AF0EE477ADCB9FDEE11
:1053D000C77AE64617EE909ACC4504DCA94517EE4D
:1053E00090EAA8BFAE4607EE90EAF8EEE77A00280A
:1053F00000F043829342E8EC017A07F11007D9D11B
:105400000B9CFCF7B1BD069931B1F4EE474AF1EEC1
:1054100010FAC8BFF0EE667AFDEEE77A17EE90EA72
:10542000F24507EE90AA04DCAE45A8BFAE4607EEF3
:1054300090EAF8EEE77ADAE7FDEEE47A10AB17EEE1
:1054400090CAFDEEE67A0B94614FDFF8AC81CDEDAA
:10545000087A544603EB8202CDF824900A91CDF8E5
:1054600018E017EE90AA05E09A42E8EC017A07F1FD
:105470001007C5D097ED007AF3EC017AE7EE257AB4
:10548000B0EE647AA3EE277AF0EE477ADCB9FDEE4F
:10549000C77AE64617EE909ACC4503DCA945CE467E
:1054A000A8BFAE4607EE90EAF8EEE77A0028DBD117
:1054B0000A990029D8D109998E4607998E45B8BF17
:1054C000F0EE667AD0E7069931B1F4EE474AF1EE94
:1054D00010FAC8BFF0EE667AFDEEE77AD64617EE10
:1054E000909ACA45DEDCD9E7F0EE627AFCF77CB927
:1054F000384B9FED396AB3F90020B3F9023007EE5B
:10550000902A06EE903AF8EEE77AF8EEE66A27EE91
:10551000E87A60EE277AA0EE267AE8EEA67A27EE01
:10552000067A67EE867A90E4BCF838009FED2B7A15
:1055300007EE900AF8EEE77A294867EE877AC0ED21
:10554000007AFCF7C6BDDFF8B490FCF718BE9FEDFB
:10555000188AFFF7EDBB234A516900293BF417ACC9
:1055600021490888214991FBF0F1106801605374CA
:10557000FBF70DBC9FED0E8AFFF7A4BBA3F50C4310
:10558000A03B41E433462AE4A3F50C43A03B1FE4CF
:105590009FED170A174B0A9325EE800A21F0F2FBC4
:1055A000DFF85C80D4F8B061A8F80600FDF7F0BD24
:1055B00000000000E48D00203C08002068810020ED
:1055C00084F9223F92E741B99730083C15A82ABEDA
:1055D000CC87002080400020CDCCCC3D6F12833A98
:1055E00094000020CC7D0020E47D002020A1070055
:1055F0000000C84244A400203081002064950020AF
:105600009894002035FA8E3CDB0FC93F0000000063
:1056100007EE906AB8EEE76A5FED067A1FED067A4C
:1056200084F8846126EE276A76EE077AFDEEE76A53
:1056300016EE903A2033402B40F247811FED0D7A51
:10564000DC4BFDEEC67A83ED017A17EE903A2033FB
:10565000402B00F23781DFEDD87AB4EEE76AF1EE45
:1056600010FA40F32082DFEDD55ADFEDD57A01E064
:10567000B0EE666AB4EEE76AF1EE10FA76EE656AAD
:10568000F6DCDFEDE17AF4EEE76AF1EE10FA40F1D4
:105690000782DFEDCA5A9FEDCB6A01E0F0EE676A40
:1056A000F4EEC66AF1EE10FA76EEA57AF6D4DFEDE6
:1056B000C66AF4EEE67AF1EE10FA40F35081DFEDBF
:1056C000BE6A76EEE77A67EEA75A9FEDC05A9FED65
:1056D000C06ADFEDC06AA5EE856A27EEA55AE5EE41
:1056E000866AE5EE267AC4ED627AFEF72CB8BA49EE
:1056F000BA4A8C46FEF78EB999ED000A08930791D5
:10570000069221F03FFBDFF8F0E2DFF8F082DEF8EE
:10571000ECE0DFF8ECC2A8F800008CFB0E3C4FEA8E
:10572000EE70C0EBAC1007EE900AF8EEE77A069A3E
:105730000799089BFDEEE77A17EE900AA8F8020099
:10574000FCF722BDF9F730F8DFF8B082D4F8B49155
:10575000D4F8B061A0EB0A00A8F80200FEF7F7B990
:105760009F4A126802F59C520832C4F8982198F8B2
:105770000020012A7DF405AC94F89421002A7DF4E0
:1057800000AC032B00F0928121F00CF8012384F887
:105790009431FDF7F6BBF9F707F8DFF860829BF864
:1057A0000070A0EB0A00A8F80200FEF76DBBF8F746
:1057B000FBFFDFF8488299F80020D4F8B0619BF82D
:1057C0000070A0EB0A00A8F80400FEF7C9BB854BE7
:1057D0001B78002B00F0CF800023FEF7C2BCDFED6A
:1057E000767AF4EEE76AF1EE10FA40F35681DFEDD7
:1057F000735A9FED736A01E0F0EE676AF4EEC66AD1
:10580000F1EE10FA76EEE57AF6DCDFED7F6AF4EE83
:10581000E67AF1EE10FA40F13D81DFED685A9FED36
:10582000696A01E0F0EE667AF4EEC67AF1EE10FAFB
:1058300077EEA56AF6D4DFED647AF4EEE76AF1EE6E
:1058400010FA04DDDFED5C7A77EEE66A85E5DFEDE0
:105850006D7AF4EEE76AF1EE10FA44BFDFED6A7A92
:1058600077EEE66A79E55D4901F1800CFEF75FBBF2
:1058700009981AF023FFFEF74FBE0A9900297FF41A
:10588000B9AD09998E4607998E45B8BFF0EE667A94
:10589000B0E5554A1278002A71D1544A128B07EEAE
:1058A000902AF8EEE77AFEF746BDA8F80600A5F8BC
:1058B000A860FBF7E2BBF4F7E1FC00283EF4EAAD98
:1058C000FEF7E2BDDFED4A7A0DE7B4EEC76AF1EE0E
:1058D00010FA0FDDB0EE677ADFED385ADFED386A87
:1058E00001E0B0EE677AB4EEE67AF1EE10FA77EE08
:1058F000E57AF6DC9FED447AF4EEC77AF1EE10FA21
:105900000FD5B0EE677ADFED2D5ADFED2E6A01E09C
:10591000B0EE677AB4EEE67AF1EE10FA77EEA57A99
:10592000F6D49FED297AF4EEC77AF1EE10FA6DDD28
:105930009FED217A77EE677A67EEA75A9FED235A9B
:10594000DFED236A9FED237AE5EE856A27EEA55AFF
:10595000A5EEA67AE5EE077AB0EE677A70E6DFED9F
:10596000296AF4EEE67AF1EE10FA44BFDFED266A1A
:1059700076EEE77AA7E613F0BFF8FBF777BBDFED2B
:105980001C7AFEF7D8BC634671464246B8E4194A11
:10599000D35C002B7EF47EAD00234FF0FF32C9F8BC
:1059A0000030042388F80030C9F80420B378FEF7EB
:1059B000B0BC00BF94000020DB0F4940DB0FC940A2
:1059C000E4CB1641E4CB16C1DB0FC93F92E741B9E6
:1059D0009730083C15A82ABE648F00208023002041
:1059E000EC7D002063950020EC400020C4400020A6
:1059F0000000000034940308DC1700209894002075
:105A0000D34D6210DB0FC9BFDB0F49C01FED037A16
:105A1000F4EEC77AF1EE10FA44BF1FED057A77EE87
:105A2000677A89E73E49B3780A604FF0FF324A60EF
:105A3000072288F80020FEF76CBC80200CF046F8A6
:105A400008B112F03FF920F0ADFEFEF73CBE9BF826
:105A50000010132913D0002B43D113297DF4D7AAAA
:105A6000B0EE480A21F08EF9A8F80200FDF7D1BA8D
:105A700094F8E831002B7BF4ACA9FBF795B9B0EEB4
:105A8000480A0893079121F07DF90799A8F80000CA
:105A9000089BE0E7F0EE676ACDE6F0EE667AB4E6E2
:105AA000F0EE667A03E6F0EE466AEAE580200CF056
:105AB0000DF800287DF465AA66E694F8D831EBB1BC
:105AC0000A9BD3ED03DA174B93ED020A164B38EE1F
:105AD0006DDA29EE000A20EE0D0A83ED020AFBF7CB
:105AE0000CBB06F5F460B0EE480A2844D5F89C37A4
:105AF00098479BF80010B0EE408AAEE7094B2B4464
:105B000093ED000A059BD3ED01DA29EE000A38EE89
:105B10006DDA20EE0D0A88ED000AFBF7EEBA00BF41
:105B2000188D0020F4750020FC80002003680A7A9C
:105B3000591C01601A70704738B50B4C23688BB143
:105B40005A68821A002A054604DA0CE05A68AA1A32
:105B5000002A07DB9A68226018461A689047236873
:105B6000002BF3D138BD38BDBC8000200B4B002288
:105B700010B4027203F178040421890742BF197935
:105B8000815401329C4203F1180303D0072A01DC3F
:105B90009979F2E75DF8044B704700BF00A803084D
:105BA00010B4104C0423214613F001034FF00002FF
:105BB00001F1180108D10132062A0ED08B7913F0B9
:105BC000010301F11801F6D002EB420204EBC2021C
:105BD0005DF8044B13790370704703705DF8044B54
:105BE000704700BF00A80308012332213122417011
:105BF000427103700371704770B54E6805463046B8
:105C000020F064F8314604460246286820F046FF3A
:105C10002A68131901333B212B60115570BD00BF59
:105C200008B518F0DBFBF4F751FE00BF024A034B46
:105C3000127819780CF006BC782300207923002014
:105C400038B5384B5A899989914224BF00225A812C
:105C5000198ADA89914224BF0022DA81DA788AB17E
:105C6000072A0FD0304C3148A27801210025062A9E
:105C700001709970DD714CD92379DFED2D6A002B0D
:105C800036D138BDDA799B78284807EE103A002AD9
:105C900044D0DFED276A0178234CB8EEC77A07EECF
:105CA000901AA278F8EEE77A27EE267A062A67EEAF
:105CB000877A2BD81F4B03EB8203D3ED006AF4EEF7
:105CC000E76AF1EE10FA10DDC6EE877AFDEEE77AAC
:105CD00017EE903A102BA8BF1023012BB8BF012359
:105CE000DBB28B4228BF0B4603702379002BC8D050
:105CF000013A032AC5D8B7EE000A80EE260A21F041
:105D000041F82388984238BF208038BDDFED086A0B
:105D1000D5E7DFED097AB0EE677ACBE7DFED076A0A
:105D2000B9E700BF0C9C0020C4400020248D002057
:105D30006F120338DC9603086F12833A6F1203392F
:105D4000F0B5474B1A6883B00123500200935CBF43
:105D500003F180530093D100424909685CBF43F0CE
:105D6000100300938F0748BF43F0C6033E4948BF66
:105D70000093160648BF43F44063097848BF009378
:105D8000D40548BF43F0006301F0EF0048BF009323
:105D900008286D465BD00E2959D0D0033348009BAC
:105DA00000784CBF43F4204343F40053D7044CBF66
:105DB00043F0644343F0444300280CBF07200F2006
:105DC000960648BF43F48073540748BF43F400333A
:105DD00043F400245205009403D5254A1279002A81
:105DE00039D1182908BF009B019004BF43F06073AC
:105DF00000930027012639462846FCB2F4F781F9C2
:105E000060B11C4B002203F5D87103E08B420FD028
:105E100013F80C2C944203F10C03F7D10137242F13
:105E2000E9D195E80300144B83E8030003B0F0BD0B
:105E30007A0904F01F0455F8223006FA04F40137F9
:105E400023EA0404242F45F82240D4D1E9E743F49F
:105E500080530093A1E743F4C0130093C1E700BF50
:105E6000C8450020BC8D002004230020EC40002009
:105E70002C95002090920308702300202DE9F84F04
:105E80004E014FF0000B174D8146904606F120075A
:105E90005C46594628465FFA8BFAF4F732F9C0B1EE
:105EA000A64215D8A74213D900200F4A014604E0A4
:105EB0000131242914D012F80C0C504502F10C02C7
:105EC000F6D10A4B01EB410103EB81014846C04783
:105ED00001340BF1010BBBF1240FDAD1BDE8F88FCF
:105EE0000021F3E7702300209092030884920308B6
:105EF00000210A4A0B4604E00133242B0BD012F890
:105F00000C1C884202F10C02F6D1054803EB430356
:105F100000EB830070470020704700BF9892030891
:105F20008492030800210A4A0B4604E00133242B23
:105F30000BD012F80C1C884202F10C02F6D1054875
:105F400003EB430300EB830070470020704700BF62
:105F5000909203088492030808B501210220F8F703
:105F60005DFF094B1B7803F00503052B08D00021CA
:105F70000120F8F753FF00210846F8F74FFFFEE72E
:105F800018F0DCFAF3E700BFFC3B0020022828BF32
:105F9000022010B4084C094B207000EBC00200EB4B
:105FA000820207495DF8044B013003EB4203C0B2A3
:105FB0000B6012F0D1BE00BFCA79002078520020D9
:105FC0002421002008B517F081FAF3F7ABFABDE8F9
:105FD000084017F063BA00BF2DE9F047A84FA94E5B
:105FE00017F074FABE421ED2DFF82483DFF8249340
:105FF0004446258862197DB14A450DD2052D0BD93D
:1060000033886188C3F30B03994200F0D8801446AB
:1060100025886219002DEFD1716830461436F3F7E8
:1060200005FABE42E4D3984A5378022B40F2EC8042
:1060300000239649537013789548022B016000F2B3
:10604000DF8003EBC301934A03EB810302EB4303BD
:10605000914C184623600EF08DFF904A1378A3F1FF
:10606000170102290FD98E4911F83300002840F09A
:10607000D180D8000144497829B18A4911F83330D8
:10608000002B00F0F580884B9A78042A00F0E78016
:1060900032B91A88B2F5F07F84BF4FF4F0721A80DB
:1060A000824D834A2B681A40002A00F0E480DE0704
:1060B00000F1D080580400F1C880190700F1C080B9
:1060C0009A0100F1B7809B0400F1AD8023689A8C9F
:1060D000D98C914224BF00229A84FFF7B1FD0AF0C7
:1060E0005DFE10B9734811F0F7FB1CF083F8002136
:1060F0003022714822F051FF704B256803F15001A6
:1061000002E00433994279D01A78002AF9D19C78B8
:10611000D8788442F5D26A496A4B0A7028461D60D5
:1061200008F0DEFF684B694A1E78694969486A4B86
:106130001160C825642212FB0652684C006B31F8CE
:10614000041C5A60002221809A60DA601A615A6148
:106150009A61DA6183F8202083F8212008B117F0D2
:10616000F1F85F4B9FED5F5A1B885F4A9FED5F6AB6
:1061700055795F4C5F496048086006EE903AF8EE4A
:10618000E66A1388C5EE265A07EE103A538812794C
:10619000C4ED005A07EE903AB8EEC77A574BF8EEC6
:1061A000E77A1D725A7227EE067A67EE867ABDE8A4
:1061B000F04783ED017AC3ED007A17F06FB9637988
:1061C0009B077FF424AF716894F804A03046F3F77E
:1061D0002DF93388BAEB133F0BD173887068AA1F6F
:1061E000C3F30B039A4204F10601A8BF1A4620F03C
:1061F00055FC1436BE42FFF4FBAE14E701228AE7D9
:1062000000231370234B23E7204903EB430301EBE7
:10621000830110E7D8000D186D68002D7FF42AAFB8
:106220001725157026E73648F3F736F94020F3F7BF
:1062300033F94BE746F20900F3F72EF92B6842E7F2
:106240003048F3F729F92B683AE72F48F3F724F998
:106250002B6832E72D48F3F71FF92B682AE71A8BD2
:10626000B2F57A7FBFF41CAF4FF47A721A8317E746
:106270001823137007E743F008032B6017E700BFEC
:106280009805000888010008CA7900209C79002040
:1062900028210020785200202421002004230020FF
:1062A000489F0308CCA50308C4400020C853002021
:1062B00009600002E09B0020542600206C81002031
:1062C000841B002088260020A8880020E8A4002045
:1062D000348D0020F41E0020382100201C80002076
:1062E00090240020C0C9FB489425002017B7D1385E
:1062F00094240020A08200203661023D7C82002090
:10630000094000020160000209200002086000024A
:10631000074000080080000808B517F0D7F8F3F729
:1063200001F917F0BBF8FFF757FE0120BDE8084060
:1063300012F012BD38B50D4C0D4DAC4206D261685D
:1063400020461434F3F772F8AC42F8D3094B0A4CE8
:106350000A481860002525700EF00CFE084B094A0B
:1063600065701A60BDE8384007F0C4BF88010008B6
:106370009805000824210020CA79002078520020C6
:10638000282100209C79002008B5FFF7D3FF17F0E3
:106390009DF8F3F7C7F8BDE8084017F07FB800BFD5
:1063A0002DE9F0470B684A680B388AB00C46D51ABD
:1063B000EF2800F27881DFE810F07C0176017601A9
:1063C0007601760176017601760176017601760115
:1063D0007601760176017601760176017601760105
:1063E00076017601760176017601EA0176018A026C
:1063F00076017B027601760176017402760126022F
:106400007601D2017601C1017601BA0176019401CB
:106410007601520176017601760176014D01760111
:106420007705760176016A057601760176017601B7
:1064300076017601650576017601760146057601DD
:10644000C105760176018405760176017601760133
:10645000760176017601F0007601D0047601E80538
:10646000760106057601340576017601760176011E
:106470007601760176017601760176017601760164
:106480007601760176017601760176017601760154
:106490007601760176017601760176017601760144
:1064A0007601760176017601760176017601760134
:1064B0007601760176017601760176017601760124
:1064C0007601760176017601760176017601760114
:1064D0007601760176017601760176017601760104
:1064E00076017601760176017601760176017601F4
:1064F00076017601760176017601760176017601E4
:1065000076017601760176017601760176017601D3
:1065100076017601760176017601760176017601C3
:1065200076017601760176017601760176017601B3
:1065300076017601A4047D04640476012704F30344
:10654000E7037601DC03AE039C0397036D0376013A
:106550005A03760176014B0336032E031C030C030A
:10656000FD02E90276017601760176017601760177
:106570007601760176017601760176017601760163
:106580007601DE0276017601B302760176017601AC
:1065900076017601760176011B020846F3F7D1F900
:1065A00005460BF043FFFF2854D0B5F57A7F80F005
:1065B00034850AAE002306F8243DEF0831460DF17C
:1065C00003008DF8033001370BF010FF9DF8033006
:1065D000FFB205F00705BB4205F1010503D19DF8A7
:1065E0000430AB4203D0294638460BF00BFF94E849
:1065F0000C009B1A012B2DDD531C0AA823600023DD
:10660000157800F8253D0BF0E5FE9DF80330AB4210
:106610000AD0B44B1B683BB19A79AA4204D31B68D9
:106620001B690BB12846984723685A1C22603046E4
:1066300000221C788DF8042008F0C0FD9DF804307D
:10664000A34207D0A74B1B6823B11B685B690BB142
:1066500020469847012318460AB0BDE8F087A249B2
:10666000A1FB05216A1A01EB52018908C1EBC102A5
:10667000B5EB020917D1C9B24F1EFFB20029E9D00C
:10668000DFF868A201375A1C226093F90060974B2B
:10669000002593F90210B14203F1080300F093843E
:1066A0000135052DF5D14FF0FF3318460AB0BDE88E
:1066B000F0878F49102D4FF0000328BF10250B6085
:1066C0004B608B60CB600B74002DC3D023685A19CC
:1066D0000133236013F8010C01F8010B9A42F7D142
:1066E000B8E75A1C0A601A780E2ADCD8991C216077
:1066F00058780328D7D87F4D02EB42025200A918E0
:10670000DE1C487126609878A8541A1D2260DA7839
:106710004A705A1D22601A798A709A1D22605A792D
:10672000CA70DA1D22609B790B71012393E75A1C12
:106730000A60714A1B78537501238CE75A1C0A6062
:106740001E781F2EAFD8052DADD10846F3F7E2F81D
:106750006A4B43F8260007F0CDFD01237BE7674D28
:1067600005F140062046F3F7ECF82368A5F8800011
:10677000591C1A46216012F8021B85F8821022600B
:106780005B7885F883300435AE42EBD162E75A1C62
:106790000A601E78132E86D89A1C0A6000205D7845
:1067A0005749024605E00132242A3FF47CAF11F834
:1067B0000C0C854201F10C01F5D15248524902EB13
:1067C000420210F8222001F82620D81C206001EB9C
:1067D000860299785170191D2160D8789070581DE3
:1067E00020604A491B790868D3701BF091FC31E79F
:1067F000474B1B78DB073FF556AFFFF7E3FBFFF78F
:10680000EBFB012327E75A1C0A603B4E1B783372CF
:106810000846F3F796F8B0832046F3F792F83083F2
:106820002046F3F78EF8236870835A1C22601B7889
:10683000F374082D7FF60EAF2046F3F782F8F0844C
:106840002046F3F77EF80C2D30857FF603AF2368E2
:106850001A46591C216012F8021BB17722605B783E
:1068600086F820302046F3F76CF8102DB0847FF6C0
:10687000F1AE23685A1C22601B78F3722046F3F7AE
:1068800049F82368F0605A1C22601A783274162D79
:106890007FF6E0AE9A1C22605B7886F821300123F7
:1068A000D9E65A1C0A601B4A1B7813700123D2E6F2
:1068B0000846F3F746F8184D28602046F3F741F8EC
:1068C00068602046F3F73DF80123A860C3E6134D46
:1068D00000232B600846F3F71DF82B681843286047
:1068E0000123B8E6A440002025499224E09B002023
:1068F000CF790020C827002098450020E08800209C
:1069000098920308849203086C81002024210020BF
:106910006F3D002004230020243C0020C8530020A9
:106920005A1C0A601A780F2A3FF6BDAE991C2160E6
:10693000C2EBC202A04958788854D81C20600A448F
:1069400099785170191D2160D9789170591D216075
:106950001979D170991D216059791171D91D216062
:106960009979517103F108012160DB7993710EF07F
:106970006DFA01236FE60846F2F7E3FF8F4DA88119
:106980002046F2F7DEFF0123688164E619465A1CAF
:1069900022608B4A11F8020B1070216059785170F7
:1069A000D91C216099789170191D2160DB78D37012
:1069B000012350E60846F2F7C4FF824DA882204624
:1069C000F2F7BFFFE8822046F2F7BBFF01232883DE
:1069D00041E61A46591C216012F8020B2260DA1CAB
:1069E000597822609A7819F0EFFC00287FF432AED3
:1069F00059E61A46591C2160734912F8020B0870B7
:106A000022606E495A788A70DA1C22606F4A9B783D
:106A1000937001231FE66E4B6E4918684A2220F0DE
:106A20003DF8012317E619465A1C22606A4A11F8FC
:106A3000020B1070216059785170D91C21609B782D
:106A400093702046F2F77DFF644A0123D08002E66E
:106A50000846F2F776FF614D28802046F2F771FF75
:106A600068802046F2F76DFF0123A880F3E55C4FB4
:106A70003B78002B3FF4EEAD5A4E00252046F2F74E
:106A800060FF17F075FC3B78A6EC010A0135AB42BC
:106A9000F4DCDFE50F2D7FF406AE5A1C0A601D788A
:106AA000072D3FF600AE08464F4F05EB4505F2F7C0
:106AB00048FFAD007E19B0802046F2F742FFF0801B
:106AC0002046F2F73EFF236830811A46591C2160A8
:106AD00012F8021BB17222605B78F3722046F2F763
:106AE00019FF01237851B6E50846F2F72AFF012382
:106AF000B1E55A1C0A601878050600F1F0823B4B9C
:106B00001B78DC073FF5A6AD032828BF0020FFF760
:106B10003DFA01239FE55A1C0A6008461D78F2F7EA
:106B2000F9FE80462046F2F7F5FE07462046F2F7CA
:106B3000F1FE06462046F2F704FF2046F2F701FF79
:106B4000236801332360002D00F0B582102D7FF4FF
:106B500081AD274BC3F800805F600EB1254B1E60EE
:106B60002549264B0222081F1A7008F069FA0123F2
:106B700071E51E4B1B78D8073FF56CADFFF704FCA1
:106B8000FFF72AFA012366E5184B1B78DA073FF571
:106B900061AD1B4A137843F00403137001235AE5D7
:106BA000124B1B78D9073FF555AD164B4FF4C87201
:106BB0001A8001234FE500BF7C750020308D002036
:106BC000843D0020C44000200C9C0020488D002003
:106BD00024210020B4A80308288D002094880020D8
:106BE000859400209C870020887400206F3D002041
:106BF0008C2600207C23002090260020943F00203B
:106C00004E1F0020A88D0020092D7FF64CADB84FF7
:106C10001A46591C3E68216012F8021B317022602E
:106C20005A78B270DA1C22609A78642A03F104015F
:106C3000A8BF642272712160DA78642A03F1050129
:106C4000A8BF6422B27121601A79F2719A1D226084
:106C50005A79642A28BF6422D91D327221609A7938
:106C6000F27003F108022260DB7933712046F2F7FB
:106C700068FE0A2D708140F03C821BF0BBFA0123B4
:106C8000E9E49C4A1068DA1C01462133951E256010
:106C900012F8035C0D70551E256012F8025C4D70F1
:106CA000226012F8015C8D7003329A4201F10301F7
:106CB000ECD1B2E05A1C0A601A788F49002A00F021
:106CC000A8810A7842F00202981C0A708B4D20605D
:106CD0005B782B702046F2F71DFE68602046F2F7C5
:106CE00019FEA8602046F2F72CFEA8812046F2F794
:106CF00028FE834A6882137843F00203137001234D
:106D0000A9E4C5F34705122D3FF6CDACBDB10AABE2
:106D10000DF1020703EB45083E46A8F12608204680
:106D2000F2F70FFE26F8020FB045F8D1754B37F891
:106D3000022F23F8022FBE42F9D1112D09D8724A31
:106D40006D00AB1E13440021223223F8021F934230
:106D5000FBD16E4A012313707DE41A46591C216051
:106D60006B4E12F8021BB17022606A495A780A70A1
:106D7000DA1C2260684D9A782A711A1D2260DB782D
:106D8000092BA8BF09232046AB70F2F7DAFD236870
:106D900062682880D11A012905DD2046F2F7D1FD6D
:106DA000626823686882934240F05C81FEF748FF86
:106DB000236862689A423FF44DAC5A1C22601B78EB
:106DC000EB70012347E40846F2F7BBFD2046F2F7DB
:106DD000B8FD2046F2F7B5FD2368464F9A1C3E6881
:106DE00022605A7886F82F20DA1C22609A7886F87A
:106DF0003A201A1D2260DA7886F83B200733236098
:106E00002046F2F79EFDF08720463E68F2F799FD96
:106E1000112DB08700F21881386816F093FF012316
:106E200019E41A46591C21603C4912F8020BC8703B
:106E300022603B495A780A70DA1C2260394A9B78F2
:106E4000D370012307E41A46591C2160364D12F80D
:106E5000021B297022605B786B702046F2F771FD8F
:106E6000236868805A1C22601B782B712046F2F739
:106E700068FD2368E8805A1C22601B782B7201236E
:106E8000FFF7E9BBF3F754FB0123FFF7E4BB274A05
:106E900003F108000133236013F8011C02F8011FFD
:106EA0009842F7D1FFF7D6BB591C1A4621602049FA
:106EB00012F8020B887022605B784B700123FFF799
:106EC000CABB1C4A1278012A3FF6C4AB19465A1CA9
:106ED0002260194A11F8020B9070216059781170E4
:106EE000D91C21609B7853700123FFF7B4BB00BF0E
:106EF00028210020242100204E1F0020501F0020A8
:106F0000923F00204E7700205077002074770020B9
:106F10000C9C0020248D0020C4400020308D0020D7
:106F2000408D0020488D0020A88800209745002033
:106F3000548D0020F1790020F27900205A1C0A605B
:106F40001E78112E3FF6AFAB9A1C0A606F4D5B782E
:106F500005F816300846F2F7F4FC40F6CA039842EA
:106F6000A8BF184640F2EE239842B8BF1846684BB7
:106F7000A0F2EE2083FB002305EB4605C017C0EB13
:106F8000E30068700123FFF766BB5A1C0A60614F7B
:106F9000DFF894811B783E6888F805300846F2F7E0
:106FA000D0FC308420463E68F2F7CBFC052D70847F
:106FB00060D8FEF745FE1DF003FD386817F010F8A5
:106FC0000123FFF748BB0AEBC508204688F802609A
:106FD000F2F7B7FC21682AF835000B464A1C2260FC
:106FE00013F8022B88F8032023604B7888F80430CC
:106FF000CB1C23608B7888F806300B1D236009F1C9
:107000000109CA7888F805204F457FF43CABFFF7AB
:1070100021BB0A7802F0FD0256E601AE304608F0C8
:10702000C1F8BDF80430AB423FF4E1AA3A4B1B680B
:10703000002B3FF4DCAA1B689B69002B3FF4D7AA06
:1070400028469847FFF7D3BA23683868591C1A4670
:10705000216012F8021B80F8311022605B7880F802
:107060003230DAE65A1C22601B78003318BF012345
:10707000F3719BE62046F2F764FCA8F80A0020466C
:10708000F2F75FFCA8F80C0020463E68F2F759FCC6
:10709000B08420463E68F2F754FC0D2DF08488D968
:1070A0002046F2F74EFCA8F80E002046F2F749FC05
:1070B000A8F810007DE7194B1020C3F800805F602E
:1070C00011F062FE164A137843F001031370002E8C
:1070D0003FF4C0AA134A01231660FFF7BCBA00F0C0
:1070E0007F00032828BF002004F0A0FB0123FFF746
:1070F000B2BA23683A68591C2160197851720B2D75
:107100001FBF991C21605B785370B6E51079002091
:107110001F85EB5124210020A44000206021002085
:107120004E1F00207C2300200C9C00202DE9F04FF6
:107130002DED028B994A9A49137895B000F59C4839
:1071400008F120080990C1F80080002B00F0AC86FF
:1071500094490968884240F2948093490591D1F896
:1071600000B092489249934C0290013B13700BF48B
:10717000805303910893002B40F09280039B5B7D2A
:10718000002B40F0FD841BF4004F41F054801BF4B1
:10719000807F0BD0099A884BDFF850A29A429AF868
:1071A000022001F22682002A41F02782834B844D7F
:1071B00006931BF4805940F05F86039BB4F9066088
:1071C0005B8B9E42B4BF00260126DFF81882D8F8F8
:1071D000003013F0805370D0069A127812F001023A
:1071E00072D003987749808C91ED037A049107EE71
:1071F000900AF8EEE77AB4EEE77AF1EE10FA81F24F
:10720000F580002E68D1029991F8A410002963D16D
:107210006D486E49006890F8300000270F604F609D
:107220008F606B49002858D10870002A59D01BF094
:10723000100F56D0674A1278D20652D4B9F1000F17
:107240004FD1002B4DD11BF4800F4AD12F78002F46
:1072500002F09980604B9B78002E42F0DA803BB1BF
:107260005E4A5F4B12681B689B1A002BC2F2B78004
:10727000102011F05DFC029A2F78012382F8A530CE
:1072800030E0494B0593D3F800B0494B474A03938C
:107290000BF480530292474C0893002B3FF46EAFDF
:1072A00000215048F2F72DFF00287FF467AF14F05B
:1072B000C5F8059BD3F800B060E71BF4800F8BD1B5
:1072C000069A127802F001020298002180F8A410B8
:1072D0003C490491002E9BD03D4901200870002AB2
:1072E000A5D12F78039AB4F900C0518B928BB4F9D1
:1072F00002008C45CCBF4FF0800E4FF0000E4EF0D8
:1073000040039445A8BF73469B0843F0800E884213
:10731000C8BF734643F0400E9042B8BF73469B0807
:10732000B4F904E0B4F9060043F0800C8E45C8BF00
:10733000634643F0400C9645B8BF63469B0843F054
:10734000800E8842C8BF7346029943F0400E91F800
:10735000A6C09042B8BF73469C4500F07D864FF0B2
:10736000000C81F8A63081F8A7C0002F00F0E98753
:10737000059B1B6803F00403002B40F057850DF1BB
:10738000480B194D0023CBF8043005F15009129336
:1073900040F6330A192740F283362CE0F4810020AE
:1073A00018800020F0810020C8450020A42500207E
:1073B00098450020E0220020404B4C006F3D00200B
:1073C000841B0020649500202421002008810020D7
:1073D000682500204E1F0020548D0020EC7D0020E9
:1073E000207E0020F48C00206C81002038210020B9
:1073F00004354D4520D0AA78EB789A4217FB0261FC
:10740000F6D26A78043217FB036334F9122052452E
:10741000A8BF5246B2F5617FB8BF4FF46172914286
:10742000E6DA9A42E4DC29782329E1D85846043583
:10743000F2F758FE4D45DED15F4B9BE803001E7806
:1074400088E80300002E00F077845C4B07935C48CB
:107450000121F2F756FE002840F09782059B1B6839
:10746000D80500F18D82574F574D2B881EB226F05C
:1074700001061FFA86F94B45A5F8009000F05A86E0
:10748000524E4FF002080F204FF0140B4FF0FF0A3E
:1074900086F8008086F801B086F802A011F048FB5B
:1074A00041464748B5F80090F2F72BFE002841F01E
:1074B0002D8229F002039BB24B452B800BD0434B0E
:1074C0001421FF2202260F201E7059709A7011F0AD
:1074D0002FFBB5F800903E4BDFF800A11978DAF8E1
:1074E0000400089319F0030F08BF81F00201C1F3F3
:1074F0004001F1F779FB3B6813F00A0F1CD005211E
:107500002F48F2F7FEFD002800F006872E8872074C
:1075100041F174812A480621F2F7F3FD002800F0BA
:10752000E886730641F1628107212548F2F7E9FDFB
:10753000002840F046833B68980600F151832E886E
:107540001F480C21F2F7DDFD002800F03D8246F4D3
:107550008073B3422B8009D01C4B02261421FF22DA
:107560000F201E7059709A7011F0E2FA194B1B78B7
:10757000082B00F035820E2B00F03282059B1B6831
:1075800058055CD5144B1B79002B00F01781142192
:107590000B48F2F7B6FD002840F0158118F0C6FB45
:1075A000012011F0BDF9002849D0DFF83490002601
:1075B0004FF0CC0B19E000BF8B3F002028210020AA
:1075C000F48C0020BC8D002020210020E028002029
:1075D000B67D0020042300202C950020B87D0020DB
:1075E000344E0020DEB2022E29D80BFB06F8731CA5
:1075F00059F80870002FF5D1C378CB4A90F90200F2
:1076000052F8233001970322009201213A4610F0EC
:1076100071FB034606EB460000EB0010029353B1EA
:10762000394609EB8000CC2221F0B7FC029B49F8D7
:1076300008300136F6B21DF073F90028D3D1069B4D
:107640001E7816F0010600F0F881B84B01221A707E
:10765000079BB4F906101B68B5485A890127914267
:10766000077080F2D081B34B4FF07E521A60B24A5D
:10767000039BB4F900C01F8B92F9043092F801E02B
:107680001078002BACEB070314BF01224FF0FF3240
:10769000002B40F35D82B3F5FA7FC0F25F824FF4B6
:1076A000FA731B1A07EE903AF8EEE77A049B6745E7
:1076B000C3ED007A03DDF1EE677AC3ED007AB4F929
:1076C00002C0ACEB0703002B40F34E82B3F5FA7F08
:1076D000C0F250824FF4FA731B1A07EE903AF8EE9C
:1076E000E77A049B6745C3ED017A03DDF1EE677A23
:1076F000C3ED017AB4F90400C31B002BD8BF3B1AB9
:10770000B3F5FA7F80F20A827345D8BF4FF0000EBE
:1077100000F3068202FB0EF207EE902A049A059B04
:10772000F8EEE77AB842C2ED027ABCBFF1EE677AB2
:10773000C2ED027A1A6812F4805200F0F481B1F5B9
:10774000FA6FA8BF4FF4FA61B1F57A7FB8BF4FF472
:107750007A71A1F57A71794C794884FB013ECB1797
:10776000C3EB6E1303F1010E6FF0630C30F91EE0F2
:1077700030F913000CFB0313AEEB000103FB01F324
:1077800084FB0314DB17C3EB641303441BB207EE43
:10779000903A049BB8EEE78A83ED038A002A40F012
:1077A00057822B885A0624D4002E40F0B0801AF05D
:1077B00004FF15B0BDEC028BBDE8F08F069B1B7873
:1077C000D9077FF5EBAE3C200AF080F900283FF4A2
:1077D00036AF10F077FA3C200AF024F900283FF485
:1077E0002EAF10F06FFA3C200AF01CF90028F0D1FF
:1077F00025E7544B544AB3F904305449DFED546A39
:1078000009889FED547A82FB0302DB17C3EBA203C6
:107810005B1A1BB207EE903AF8EEE77A67EEA67AAB
:1078200077EE876ABDEEE66A16EE103A2033402BFB
